:020000040800F2
:10000000B88300209D010008C91C0008671400087F
:10001000C51C0008530300087526000800000000F6
:100020000000000000000000000000002121000886
:10003000D503000800000000E91D0008A722000801
:10004000B7010008B7010008B7010008B7010008B0
:10005000B7010008B7010008B7010008B7010008A0
:10006000B7010008B7010008B7010008B701000890
:10007000B7010008B7010008B7010008B701000880
:10008000B7010008B7010008B7010008B701000870
:10009000B7010008B7010008B7010008B701000860
:1000A000B7010008B7010008B7010008B701000850
:1000B000B7010008B7010008B7010008B701000840
:1000C000B7010008B7010008B7010008B701000830
:1000D000B7010008B7010008B7010008B701000820
:1000E000CD0D0008B7010008B7010008B7010008EE
:1000F000B7010008B7010008B7010008B701000800
:10010000B7010008B7010008B7010008B7010008EF
:10011000B7010008B7010008B7010008B7010008DF
:10012000B7010008B7010008B7010008B7010008CF
:10013000B7010008B7010008B7010008B7010008BF
:10014000B7010008B7010008B7010008B7010008AF
:10015000B7010008B7010008B7010008B70100089F
:10016000B7010008B7010008B7010008B70100088F
:10017000B7010008B7010008B7010008B70100087F
:10018000B7010008B7010008DFF80CD000F088F8CC
:1001900000480047F5490008B8830020064880471A
:1001A00006480047FEE7FEE7FEE7FEE7FEE7FEE75C
:1001B000FEE7FEE7FEE7FEE771230008890100087D
:1001C00040EA01039B0703D009E008C9121F08C0D9
:1001D000042AFAD203E011F8013B00F8013B521E59
:1001E000F9D27047D2B201E000F8012B491EFBD2D0
:1001F00070470022F6E710B513460A460446194632
:10020000FFF7F0FF204610BD10B5044604E00B7860
:1002100000F8013B03B1491C521EF8D2204610BD24
:1002200010B5002200E0521C835C8C5CA34201D11B
:10023000002BF8D1D8B2E1B2401A10BD30B5044657
:100240000020034600E05B1C934203D2E05CCD5CDF
:10025000401BF8D030BD30B505460020034600E015
:100260005B1C934205D2EC5CC85C201A01D1002CC7
:10027000F6D130BD30B50B460146002020220124C6
:1002800009E021FA02F59D4205D303FA02F5491B64
:1002900004FA02F52844151EA2F10102F1DC30BD7A
:1002A000064C074D06E0E06840F0010394E80700C3
:1002B00098471034AC42F6D3FFF76AFF3490000839
:1002C0005490000870B58C1810F8015B15F0070306
:1002D00001D110F8013B2A1106D110F8012B03E0DF
:1002E00010F8016B01F8016B5B1EF9D12B0705D4E7
:1002F0000023521E0DD401F8013BFAE710F8013B30
:10030000CB1A921C03E013F8015B01F8015B521E4B
:10031000F9D5A142D8D3002070BD2DE9F0410446A3
:100320000E46F82231462046FFF74AFFB4F8F65051
:100330000020A4F8F600F821204600F027F8074630
:10034000A4F8F650AF4202D10120BDE8F0810020B0
:10035000FBE700BFFEE700001CB50121084601F0E5
:1003600045FD00208DF804000820009000208DF845
:10037000060001208DF807008DF805006946024847
:1003800000F0F0FF1CBD00000000024070B5024606
:100390000B4641F221054FF6FF70002117E0565C35
:1003A00080EA062000240EE000F400462EB141F25F
:1003B000210686EA4006B0B203E04FF6FF7606EA71
:1003C0004000661CB4B2082CEEDB4E1CB1B2994260
:1003D000E5DB70BD704700007FB500F043F900F029
:1003E0003FFB012000F0B6FD00F062FD042001F0AB
:1003F00046FF684601F05AFD64220198B0FBF2F115
:10040000B1F1807F00D31DE021F07F40401E4FF00E
:10041000E022506150170F22002807DA13071D0E43
:10042000094B00F00F04241F1D5503E013071C0E99
:10043000064B1C5400BF00204FF0E02290610720C3
:10044000106100BF7FBD000018ED00E000E400E097
:100450002F480068006800F0004098B92C480068F8
:10046000006800F4807068B129480068294909686B
:100470004860284800688068401C264909688860F0
:100480000120704722480068006800F00040F0B981
:100490001F480068006800F40070C0B11C48006884
:1004A000006800F4807090B919480068194909681B
:1004B000086000201749096848600120154909684B
:1004C000886013480068C068114908601DE0104842
:1004D0000068006800F00040B8B90D480068006886
:1004E00000F4007088B90A480068006800F4807061
:1004F00058B9084800688068401C06490968886047
:1005000003480068C068024908600020B9E700009D
:10051000480100204C01002030B10749896941F0B1
:100520000201054A916105E00349896921F0020150
:10053000014A9161704700000090024070B50C467E
:1005400013460021124D286000BF18E000EB411255
:100550004FF00045156044F2F4555560C1EBC115EC
:1005600005EB450504EB850595605D1E8D4204D9BC
:1005700000EB41152035D56000E0D060491C994260
:10058000E4D3044DE860044D044E356070BD0000B6
:100590004801002000900240A87F00204C0100206C
:1005A00030B10749896941F40051054A916105E07C
:1005B0000349896921F40051014A916170470000A3
:1005C0000090024030B50C46134600210F4D2860C4
:1005D00000BF15E000EB41124FF480151560C1EB30
:1005E000C11505EB450504EB850595605D1E8D4243
:1005F00004D900EB41152035D56000E0D060491CDE
:100600009942E7D3024D286130BD0000440100202B
:100610000090024002680A430260704710B5012151
:10062000480601F0F3FB00214FF0007001F0EEFBF3
:1006300010BD01B581B0002000900198009002E04B
:100640000098401E009000980028F9D10CBD0000D1
:100650000348806940F480100149886170470000B8
:10066000009002401CB50121880301F0FFFB01212D
:10067000072001F0BBFB012001F054FD8620009013
:1006800003208DF8050002208DF8040000208DF86D
:1006900006008DF8070069461E4800F063FE0B2235
:1006A00001211C4800F0A6FE0B220221194800F08F
:1006B000A1FE0B220721174800F09CFE4FF460506A
:1006C00000906946144800F04DFE0B221146124876
:1006D00000F090FE0B220C210F4800F08BFE0B2245
:1006E0000D210D4800F086FE3220009069460B482F
:1006F00000F038FE0B220121084800F07BFE0B229F
:100700000421064800F076FE0B220521034800F084
:1007100071FE1CBD000002400004024000080240BF
:1007200000200449096801F0010109B1012000E03D
:1007300000207047009002401EB500210022009268
:1007400001920292114A12681268C2F30D42111FFF
:1007500000910F4A12689268012A05D90C4A126862
:1007600012689268019203E0084A12689268019246
:10077000064A12680292054A1268D268034B1A6050
:100780009DE81C0080E81C001EBD00004801002000
:100790004C0100202DE9F04186B004460F464FF091
:1007A0000008002500200590954E009095480569A9
:1007B00025F01C0501A801F079FB029E92488642B3
:1007C00005D39248864202D245F008051AE08F48C8
:1007D000864205D38A48864202D245F00C0511E0D4
:1007E0008748864203D38A48864200D20AE0884876
:1007F000864205D38748864202D245F0040501E0CF
:1008000045F010057F4805614FF40042002138464D
:1008100000F0A8FA18B9002006B0BDE8F0817E48C3
:10082000FFF707FF206800284ED000BF0098401C4B
:1008300000900121384600F0EBF900F0040018B9EF
:10084000764900988842F1D374490098884201D1D2
:100850000020E1E7002000904FF48052002138464C
:1008600000F080FA08B90020D6E700BF0098401CCD
:1008700000900121384600F0CBF900F0200018B9B3
:10088000664900988842F1D364490098884201D1B2
:100890000020C1E7002000901021384600F0B8F990
:1008A000804608F0040018B14FF40060206201E0B7
:1008B0000020206208F0020010B10020606116E004
:1008C0004FF48040606112E0206AC0F3CF0061699C
:1008D000C1F34F0140EA01020021384600F042FA1C
:1008E00008B9002098E76FF07F40FFF7A2FE454867
:1008F00005684B480540D4E901010843E168084315
:100900002169084361690843A1690843E169084313
:10091000216A0843616A0843A16A0843E16A0843FF
:10092000216B0843616B0843054336480560D4E9F1
:100930000E010843216C0843616C0843A16C084315
:10094000E16C0843216D0843616D08432D494860FF
:10095000A06D8860E06DC860084685694FF64170FB
:100960000540B4F86010606E40EA0140A16E084393
:10097000E16E0843216F0843616F08430543214836
:100980008561D4E91E0108431E49C861254885696F
:1009900025480540D4E920010843D4F888100843CD
:1009A000D4F88C100843D4F890100843D4F894106D
:1009B0000843D4F898100843D4F89C100843D4F89E
:1009C000A0100843054317488561D4E9290108436D
:1009D000D4F8AC100843D4F8B0100843D4F8B410DD
:1009E00040EA8100D4F8B810084340F400000D49F3
:1009F00008600846006840F08000086001200BE7AE
:100A00000087930300800240002D3101C00E1602C2
:100A100000E1F50580D1F008FFFF0F00FFFF0400A3
:100A20000F8120FF00900240233FDEF810B50B79C4
:100A30004C7943EA0422094B03441A64CB781B0621
:100A40008C7843EA04434C7843EA04230C7843EA65
:100A50000402024B03445A6410BD000000800240AF
:100A600000B5AFB001214FF0606001F0BFF9FFF7B2
:100A7000D5FD00F003F900BFFFF752FE0128FBD0BF
:100A8000684600F015F901200090002007904FF40F
:100A900000700A9000200B900E901190139014900B
:100AA000159020904FF000702190001123900020AD
:100AB0002590269004202890C005299040122A9065
:100AC00080012B9040122C9040002E90012168460E
:100AD000FFF760FE014908602FB000BD84000020D0
:100AE00030B10749096841F00401054A116005E089
:100AF0000349096821F00401014A116070470000B0
:100B00000080024030B10749096841F00801054AF8
:100B1000116005E00349096821F00801014A1160EC
:100B2000704700000080024070B502460023002597
:100B3000002435480068006800F0004008B100203B
:100B400070BD3148016840F2F450824208DD92FBEA
:100B5000F0F392FBF0F600FB162010B15B1C00E0F6
:100B60000123012B1AD128480068006840F040504A
:100B7000254E36683060C2F30C00234E3668706034
:100B800021480068006840F000401F4E3668306021
:100B90001D480068C0681C4E306028E0002422E038
:100BA0003CB919480068006840F08050164E36681D
:100BB000306040F2F4504860581EA0420DD10868E1
:100BC00040F000500860581EC0EBC01000EB400021
:100BD000A2EB8005C5F30C004860086840F00040B7
:100BE0000860C968641C9C42DAD307480160074862
:100BF000406900F0040020B10420044E7061002020
:100C0000706001209CE70000440100200090024039
:100C100018B502460B4600210020009015480169D6
:100C200001F01C014FF4784000EAC22001434FF468
:100C3000F86000EA8310014321F0020141F0010154
:100C40000C48016100BF0098401C009009480169F0
:100C500001F0010018B1084C0098A042F3D3064CF3
:100C60000098A04201D1002018BD0248406980B21E
:100C7000FAE7000000800240FFFF0400034800681C
:100C800040F00100014908607047000000900240F8
:100C900000B50120FFF736FFFFF7DAFC0120FFF770
:100CA0001FFF0120FFF77CFC0120FFF735FC00BD92
:100CB00001210160002141608160C16001614FF448
:100CC0008041416100218161C1614FF40061016295
:100CD000002141628162C162016341638163C1633A
:100CE000402101642021416400218164C1640165C7
:100CF00041658165C165016680214166002181668B
:100D0000C166016741678167C1674FF08061C0F8C4
:100D100080104910C0F884100021C0F888104FF4EA
:100D20000011C0F88C100021C0F89010C0F8941089
:100D3000C0F89810C0F89C10C0F8A0104FF00071D7
:100D4000C0F8A4104912C0F8A8108901C0F8AC106E
:100D50004912C0F8B0100021C0F8B410C0F8B810A3
:100D60007047000038B503460C4600210020009073
:100D70001448016901F01C014FF4784000EAC320D7
:100D800001434FF4F86000EA8410014341F002018E
:100D900041F001010B484261016100BF0098401C15
:100DA00000900848016901F0010018B1064D009853
:100DB000A842F3D3044D0098A84201D1002038BDC9
:100DC0000120FCE700800240FFFF040010B54FF453
:100DD000804000F00FF830B1012000F0A9F84FF486
:100DE000804000F001F810BD014908607047000024
:100DF000143C0140014600200022074B1B6803EA17
:100E00000102054B14331B680B4013B10AB10120DA
:100E100000E0002070470000003C01400021234911
:100E20008279002A3AD00A46126803689A430B4630
:100E30001A600A1D126803689A430B1D1A60027932
:100E400011440A6803681A430A60184A0832126893
:100E500003689A43154B08331A601A1D1268036819
:100E60009A43124B0C331A604279102A0ED11A1F82
:100E7000126803681A430D4B08331A601A1D126872
:100E800003681A43094B0C331A600DE00749427995
:100E900011440A6803681A430A6005E002791144A4
:100EA0000A6803689A430A6070470000003C0140EA
:100EB00000B585B00121022000F098FF01218803D0
:100EC00000F0D4FF00208DF810008DF813004FF4CF
:100ED0008040039003A9154800F044FA0E21012038
:100EE00001F026F94FF48040019000208DF80800B1
:100EF0000C208DF8090001208DF80A0001A8FFF7E9
:100F00008DFF4FF4A06000F01DFF28208DF8000039
:100F100000208DF801008DF8020001208DF80300FB
:100F2000684600F0D3FE05B000BD0000000402409A
:100F300010B5044612212046FFF76AFE00F4005067
:100F400020B103480078C0430149087010BD00007B
:100F50008800002070B50546002411212846FFF7BF
:100F600057FE044644F00304224611212846FFF7A9
:100F7000F9FE08B9002070BD12212846FFF748FE8F
:100F8000044644F02004224612212846FFF7EAFED8
:100F900008B90020EFE70120EDE7000070B5044636
:100FA0000A460026082502B909E0012A01D11602E5
:100FB00005E0022A01D1160201E04FF4407600F06C
:100FC000DBF80546082D28D11548006820F440704C
:100FD0001349086008460068304308600846006806
:100FE00020F0F80008600846006844F00201084359
:100FF0000B4908600846006840F48030086000F043
:10100000BBF805460648006820F002000449086065
:101010000846006820F0F8000860284670BD00000F
:10102000103C024008201049096801F48031B1F5F4
:10103000803F01D1012015E00B49096801F0100142
:1010400009B105200EE00849096801F0EF0109B176
:10105000062007E00449096801F0020109B10720F0
:1010600000E00820704700000C3C024070B50446C8
:1010700025460C48854210D802212020FFF78EFF1C
:1010800002212820FFF78AFF02213020FFF786FF88
:1010900002213820FFF782FF01E0012070BD00200F
:1010A000FCE700000000080810B500F053F810BD80
:1010B0002DE9F04104460E461746002500BF16E014
:1010C00056F82510206800F01DF808280CD120687B
:1010D000006856F82510884202D00220BDE8F08151
:1010E0002068001D206001E00120F7E76D1CBD4273
:1010F00003D2206802498842E2D90020EEE70000CE
:10110000FBFF070830B502460C46082500F034F80E
:101110000546082D19D10E48006820F440700C498E
:1011200008600846006840F40070086008460068DF
:1011300040F001000860146000F01EF80546044805
:10114000006820F0010002490860284630BD000018
:10115000103C02400548006800F0004028B10448F7
:1011600002490C390860034808607047103C02408F
:1011700023016745AB89EFCD08B508200090FFF744
:1011800051FF009002E0FFF74DFF00909DF8000036
:101190000128F8D09DF8000008BD000070B5044695
:1011A0004FF400710B4800F051F9032000F09CFF50
:1011B000201200F099FFE0B200F096FF002000F04E
:1011C00093FF05464FF40071024800F041F92846AC
:1011D00070BD00000004024070B504460D464FF497
:1011E0000071134800F032F9062000F07DFF4FF443
:1011F00000710F4800F02CF942F6E06001F0D7FCD6
:101200004FF400710A4800F021F9022000F06CFF51
:10121000201200F069FFE0B200F066FF284600F0FF
:1012200063FF4FF40071024800F012F970BD000036
:101230000004024000B587B00121880300F0F6FDEC
:101240000121062000F0D2FD02208DF818008DF853
:10125000190000208DF81A008DF81B000C20059055
:1012600005A92F4800F07EF802208DF818008DF8AF
:10127000190000208DF81A008DF81B004FF48060D3
:10128000059005A9274800F06DF801208DF8180099
:1012900002208DF8190000208DF81A004FF400701C
:1012A000059005A91F4800F05DF8052202211C48A1
:1012B00000F0A0F805220321194800F09BF8052250
:1012C0000A21184800F096F84FF40071154800F014
:1012D000BFF80020ADF80000ADF80400ADF806003E
:1012E000ADF808004FF40070ADF80A002020ADF80A
:1012F0000C000020ADF80E004FF48270ADF8020033
:101300006946094800F0C2FE0121074800F0A4FE2A
:101310004FF48071044800F0D7FE07B000BD000014
:101320000008024000040240003800401CB50121C2
:10133000084600F05BFD00208DF804004FF480604B
:10134000009000208DF8060002208DF80700012093
:101350008DF805006946024800F004F81CBD000045
:1013600000000240F0B50A4600210023002400BF1F
:101370003DE0012505FA01F3156805EA03049C42E6
:1013800034D105684F000326BE40B543056015798A
:101390004E00B5400668354305601579012D02D031
:1013A0001579022D16D185684F000326BE40B5433E
:1013B000856055794E00B54086683543856045683F
:1013C00001268E40B5434560456896798E40B6B299
:1013D00035434560C5684F000326BE40B543C56030
:1013E000D5794E00B540C6683543C560491C102903
:1013F000BFD3F0BDF0B5002300244D07ED0E02FA77
:1014000005F3CE1000F1200555F826504E07F70ED3
:101410000F26BE40B543CF1000F1200646F82750F6
:10142000CE1000F1200555F8265045EA0304CE10F1
:1014300000F1200545F82640F0BD02460020136962
:101440000B400BB1012000E0002070474183704742
:10145000018370474FF6FF710160002101714171F6
:101460008171C171704700BFFEE700002DE9F041B6
:1014700005460C46002700262848007828B316E0C9
:10148000701C844209D9A95D244802780078401C68
:10149000224B18702248815408E0FF211F4802782F
:1014A0000078401C1D4B18701D488154761C1B4849
:1014B00000780328E4DD012219491A48FFF7F8FDF6
:1014C0000020164908703544A41B4FEA940804F024
:1014D0000307D7B11448006814490968884212D03C
:1014E00000200E4908700BE02819C01B01780B483A
:1014F00002780078401C094B1870094881547F1EFF
:10150000002FF1D101E008F101081FFA88F2294605
:101510000448FFF7CDFDBDE8F08100003400002055
:1015200030000020280000202C0000202400002093
:1015300010B505F045F9044650220749204604F04D
:1015400049FAFF21204605F0D3F804460349204616
:1015500004F0DCF910BD0000708F0008D9340008D9
:1015600070B505460C46204603F0FCFB284606F005
:10157000D7FD284606F0BEFE002203490348006856
:1015800006F0B4FE70BD00006116000818000020CF
:1015900001464878704770B504462546688803F0D0
:1015A00067FE70BD2DE9F04107460D461646002442
:1015B0004FF40A7003F030FC044654B919A11D48D9
:1015C00001F0A4F821463846FFF7CAFF0020BDE825
:1015D000F081022020602868C4F80C02C4F8106270
:1015E0000020C4F81402C4F81802224612493846F2
:1015F00006F07CFE002011490860FFF755FD1048F9
:10160000FFF734FD0E480F49086032462946384638
:10161000D4F8143200F0BCF80BA1064801F076F8BB
:101620000020D4E74D656D6F7279206572726F721C
:101630000000000054010020A51800081C00002034
:1016400000000108140000200D0A20537461746525
:101650003A2050726F6772616D6D696E672E2E0051
:101660002DE9F04F95B014469946DDF878B006F0B4
:101670002FFE8246BAF1000F06D126A12A4801F0BA
:1016800045F815B0BDE8F08F00222849504606F015
:101690000FFD074627B126A1234801F037F8F0E7F0
:1016A0006068FFF775FF0646022E07D025A11E4889
:1016B00001F02CF8504606F01DFE25E0D4F8048019
:1016C00008F10208002500E06D1C18F8050000284C
:1016D000FAD16A1C41460BA8FEF796FD1EA11248DE
:1016E00001F014F80BAA22A101A801F02DF801A91C
:1016F0000D4801F00BF821A10B4801F007F85A46FC
:1017000049465046FFF74EFF204603F05AFF00BF00
:10171000B7E7000043616E206E6F742063726561ED
:10172000746520706362000054010020708F00080F
:1017300043616E206E6F742062696E642070636214
:10174000000000004261642054465450206F7063D2
:101750006F646520000000000D0A202049415020E0
:101760007573696E672054465450202000000000B5
:101770000D0A46696C653A20257300000D0A537402
:101780006174653A2045726173696E672E2E2E0072
:101790002DE9F84380460D4616461F46002000906E
:1017A0000421684600F039F8B9B2684600F02CF818
:1017B00003220421002003F061FD04463CB90BA183
:1017C000104800F0A3FF4FF0FF30BDE8F8836068D9
:1017D00000990160B3B22A462146404606F0AAFDB0
:1017E0008146204603F0EDFE4846EEE743616E2059
:1017F0006E6F7420616C6C6F6361746520706275CC
:10180000660D0A005401002070B504460D462646B8
:10181000284601F05AFE708070BD002202704170AF
:101820007047000070B5452506F052FD0F4908606D
:101830000846006820B90EA1124800F067FF70BD8D
:10184000AAB211490948006806F032FC044634B9CE
:1018500000220E490548006806F048FD03E00CA18F
:10186000084800F053FF00BFE9E70000180000201F
:1018700043616E206E6F74206372656174652070C1
:101880006362000054010020708F00086116000898
:1018900043616E206E6F742062696E6420706362B3
:1018A000000000002DE9F047ADF50A7D06460F4621
:1018B00014469846DDF848A235464FF00009608985
:1018C0002189884207D04CA1514800F01FFF0DF537
:1018D0000A7DBDE8F0874FA14D4800F017FF6089F1
:1018E000042840DD6068FFF756FED5F81412491C45
:1018F000884238D16089001F82B204230AA9204699
:1019000003F016FE6089001F4949096808444849E8
:1019100008606189081FC11700EB9171C1F38F093D
:101920006189081FC11700EB91718910A0EB81013B
:1019300019B109F101001FFA80F93EA1344800F005
:10194000E5FE4A460AA94048FFF7B2FBD5F8140263
:10195000401CC5F814026089001FD5F8181208440D
:10196000C5F8180210E06068FFF715FED5F81412EC
:10197000491C884208D1D5F81402401CC5F814024D
:1019800032A1234800F0C2FE34A1214800F0BEFE7F
:10199000524641463846D5F81432FFF7F9FE6289BF
:1019A00035A11B4800F0B2FE6089B0F5017F1DDA59
:1019B00029463846FFF7D4FD204603F002FE33A146
:1019C000134800F0A3FE1A48026836A1684600F0EA
:1019D000BBFE69460E4800F099FE35A10C4800F0A8
:1019E00095FE39A10A4800F091FE03E0204603F07D
:1019F000E8FD6CE700BF6AE70D0A496E76616C6925
:101A0000642064617461206C656E67746800000016
:101A1000540100200D0A4941505F7772715F726571
:101A200063765F63616C6C6261636B200000000031
:101A30001C0000200D0A464C4153485F49665F5721
:101A40007269746520000000140000200D0A6172A4
:101A500067732D3E626C6F636B2B2B000D0A49413F
:101A6000505F746674705F73656E645F61636B5F13
:101A70007061636B657400000D0A706B745F627552
:101A8000662D3E6C656E203D202564000D0A546F66
:101A90007420627974657320526563656976656444
:101AA0003A0000000D0A25642062797465732000F5
:101AB0000D0A53746174653A2050726F672046694D
:101AC0006E697368656420000D0A202020526573DA
:101AD00065742074686520626F6172642020000064
:101AE0001CB501208DF804001020009000208DF816
:101AF000060002208DF8050069460548FFF732FC14
:101B00002020009069460248FFF72CFC1CBD000015
:101B10000000024000B58DB003F04CF903F09AFAD2
:101B2000424909780A0641490988C1F3072142EA76
:101B300001423E490968C1F3074142EA01213B4A9B
:101B4000126841EA126001F0B3FC0C903849097840
:101B50000A0637490988C1F3072142EA014234499C
:101B60000968C1F3074142EA0121314A126841EA9A
:101B7000126001F09DFC0B902E4909780A062D4950
:101B80000988C1F3072142EA01422A490988C1F3C1
:101B9000072142EA0121274A1288C2F3072241EABB
:101BA000020001F085FC0A9020480068000E8DF8C4
:101BB00024001E480068000C8DF825001B48008892
:101BC000000A8DF82600194800788DF827009DF846
:101BD00024009DF82510CDE900109DF826309DF8D1
:101BE000272015A104A800F0AFFD17A11D4800F0A3
:101BF0008DFD04A91B4800F089FD1BA1194800F0C8
:101C000085FD1A481A4900220AABCDE9002102904D
:101C10000BAA0CA9174803F065FA164803F0B2FAAC
:101C2000144803F009FB0DB000BD0000580000206F
:101C3000600000205C000020202025642E25642EFA
:101C400025642E25640000002020537461746963AC
:101C500020495020616464726573732020200D0A4E
:101C600000000000540100200D0A00007D31000832
:101C7000E93100085402002001B50C4900980968B8
:101C8000401AFA2804D309490098086006F062F95E
:101C9000074900980968401A41F28831884204D304
:101CA00003490098086001F019FA08BD7800002087
:101CB0007C00002010B5024801F0AEFA10BD000013
:101CC0005402002000BFFEE77047000070B50021FD
:101CD00000230F22C4781CB3174C246804F4E0647A
:101CE000C4F5E064C4F30721C1F10404E3B20A417E
:101CF00044789C40E1B28478144021430C07210EC3
:101D00000E4C05786155047804F01F050124AC40A1
:101D100005786D11AD0005F1E025C5F8004109E039
:101D2000047804F01F050124AC40054D06787611B7
:101D300045F8264070BD00000CED00E000E400E036
:101D400080E100E002490143024A1160704700004F
:101D50000000FA050CED00E02DE9FC470546884639
:101D60000024A1464FF0010A002600201C4908600B
:101D700000BF0BE0281910221A49FEF76CFA20B9AF
:101D800004F110001649086002E0641C4445F1D3D8
:101D900000BF13480068F8B10024114800682F18EC
:101DA00008E0385D0DF80400641C0D480068401C14
:101DB0000B490860385D0D28F3D16CB1661E09E04F
:101DC0001DF80600303800FB0A990AEB8A004FEA3A
:101DD000400A761E002EF3DA4846BDE8FC87000074
:101DE00038000020668E00087047000029B1064ABE
:101DF00012680243044B1A6004E0034A12688243EB
:101E0000014B1A60704700003038024029B1064A81
:101E100012680243044B1A6004E0034A12688243CA
:101E2000014B1A60704700001038024029B1064A81
:101E300012680243044B1A6004E0034A12688243AA
:101E4000014B1A60704700004038024029B1064A31
:101E500012680243044B1A6004E0034A126882438A
:101E6000014B1A60704700002038024029B1064A31
:101E700012680243044B1A6004E0034A126882436A
:101E8000014B1A60704700004438024029B1064AED
:101E900012680243044B1A6004E0034A126882434A
:101EA000014B1A607047000024380240F0B5002151
:101EB00000220024022500260223324F3F6807F04B
:101EC0000C0121B1042905D0082937D105E02E4F96
:101ED000076036E02D4F076033E02A4F3F1F3F6811
:101EE000C7F38056274F3F1F3F6807F03F036EB18F
:101EF000264FB7FBF3F7DFF88CC0ACF1040CDCF82D
:101F000000C0CCF3881C07FB0CF40CE01E4FB7FBA1
:101F1000F3F7DFF870C0ACF1040CDCF800C0CCF3D0
:101F2000881C07FB0CF4174F3F1F3F68C7F301479E
:101F30007F1C7D00B4FBF5F7076002E0124F0760DD
:101F400000BF00BF0F4F3F6807F0F0010909104FB5
:101F50007A5C0768D74047600A4F3F6807F4E05152
:101F6000890A0B4F7A5C4768D7408760054F3F6806
:101F700007F46041490B064F7A5C4768D740C76059
:101F8000F0BD0000083802400024F40000127A007E
:101F9000310100202DE9F04705460F4690463E46A8
:101FA0004FF00009002408E03046761C03F038FCAE
:101FB0002855285D8144601C84B24445F4DB3046DA
:101FC000761C03F02DFC04463046761C03F028FCFA
:101FD00004EB002084B289EA040010B90120BDE8B6
:101FE000F0870020FBE700002DE9F04106460F4690
:101FF0001446A046002508E0404608F1010803F019
:102000000FFC0E494855681C85B2F82DF4D30B49D6
:102010003046FEF782F918B109A000F085FB0BE00D
:10202000F82239463046FEF7CBF82146304600F01C
:102030004FFB0020BDE8F0810120FBE78802002073
:10204000526573746F72652073657474696E67731B
:10205000206F6B210D0A000021B1028842F040027E
:10206000028004E002884FF6BF731A400280704776
:102070000246002013890B400BB1012000E0002034
:1020800070470146888970478181704710B50022EA
:10209000028802F441520B884C8823438C882343E6
:1020A000CC8823430C8923434C8923438C892343C5
:1020B000CC8923431A430280838B4FF2FF74234061
:1020C00083830B8A038210BD4FF6FF62914204D0D6
:1020D000028842F48072028004E002884FF6FF63B7
:1020E0001A4002807047000010B5044600BF02216C
:1020F0000A48FFF7BDFF0028F9D021460748FFF73F
:10210000C3FF00BF01210548FFF7B2FF0028F9D047
:102110000248FFF7B6FFC0B210BD00000038004013
:10212000704700000149086070470000DC0027424A
:1021300030B500228B071C0F0F2303FA04F20B4B60
:102140008C1053F824309343084C8D1044F82530FC
:1021500023468C1053F824308C07240F00FA04F423
:102160002343024C8D1044F8253030BD083801401F
:102170000CB50020019000903348006840F4803096
:102180003149086000BF3048006800F4003000901A
:102190000198401C0190009818B90198B0F5A06F03
:1021A000F1D12948006800F4003010B101200090FE
:1021B00001E0002000900098012844D122484030DE
:1021C000006840F080502049403108601F48006896
:1021D00040F480401D4908601B48083000681A49D7
:1021E000083108600846006808600846006840F446
:1021F000805008601648091F0860081F006840F0FA
:102200008070091F086000BF0F48006800F0007070
:102210000028F9D040F205600E4908600A480830ED
:10222000006820F00300084908310860084600688B
:1022300040F00200086000BF03480830006800F06A
:102240000C000828F8D10CBD003802400070004096
:1022500008324306003C024070B504460D4600209B
:10226000A4F8F600F8212046FEF790F80646A4F8F8
:10227000F660F82221462846FDF7A2FF70BD04282B
:1022800008D14FF0E021096941F004014FF0E0224C
:10229000116107E04FF0E021096921F004014FF0DE
:1022A000E0221161704710B500F096F810BD0000F3
:1022B00070B500200022022300240221274D2D6842
:1022C00005F00C0020B1042806D0082834D107E01E
:1022D000234D244E356033E0234D224E35602FE0F0
:1022E0001E4D2D1F2D68C5F380541C4D2D1F2D68CC
:1022F00005F03F0154B11C4DB5FBF1F5174E361FEB
:102300003668C6F3881605FB06F209E0144DB5FBE6
:10231000F1F5124E361F3668C6F3881605FB06F235
:102320000E4D2D1F2D68C5F301456D1C6B00B2FBD2
:10233000F3F50C4E356003E0094D0A4E356000BFE1
:1023400000BF064D2D68C5F30315084E705D054DA1
:102350002D68C540034E356070BD0000083802404E
:102360000024F4000000002000127A000400002085
:1023700010B51548006840F4700013490860134810
:10238000006840F001001149086000200F49083141
:1023900008600E4800680E4908400C4908600D4866
:1023A000091D0860081F006820F48020091F0860CC
:1023B000002006490C310860FFF7DAFE4FF000609C
:1023C00001498039086010BD88ED00E00038024006
:1023D000FFFFF6FE10300024024800680A30014971
:1023E000086070476800002000B587B00121102008
:1023F000FFF73CFD01210846FFF7F8FC05A8FFF7B1
:1024000029F802208DF818000002059002208DF8AE
:10241000190000208DF81A0001208DF81B0005A975
:102420002148FEF79FFF02208DF81800400205901A
:1024300002208DF8190000208DF81A0001208DF877
:102440001B0005A91848FEF78DFF07220921164831
:10245000FEF7D0FF07220A211348FEF7CBFF002129
:10246000124800F025F8114800F02EF80121102044
:10247000FFF7FCFC4FF4612001900020ADF808004C
:10248000ADF80A00ADF80C00ADF810000C20ADF866
:102490000E0001A9054800F07FF80121034800F073
:1024A00007F807B000BD0000000002400010014026
:1024B00021B1828942F40052828104E082894DF682
:1024C000FF731A408281704710B504462548844244
:1024D00008D101211020FFF7D9FC00211020FFF7BF
:1024E000D5FC3EE02048844209D101214804FFF791
:1024F000ADFC00214FF40030FFF7A8FC31E01B4891
:10250000844209D101218804FFF7A0FC00214FF487
:102510008020FFF79BFC24E01548844209D101216B
:10252000C804FFF793FC00214FF40020FFF78EFC56
:1025300017E01048844209D101210805FFF786FC05
:1025400000214FF48010FFF781FC0AE00A48844222
:1025500007D101212020FFF799FC00212020FFF75F
:1025600095FC10BD001001400044004000480040B0
:10257000004C004000500040001401400246002082
:10258000B1F5007F00D100BF13880B400BB10120D3
:1025900000E00020704700002DE9FF4705460E4689
:1025A0000024A14600BFA046B08900B100BF2C8A1C
:1025B00024F44054F08804432C82AC8941F20C602E
:1025C0008443B08831890843718908430443AC814E
:1025D000AC8A24F44074B0890443AC826846FFF7A7
:1025E00065FC2048854202D01F48854202D1DDF8B3
:1025F0000C9001E0DDF80890A88900F4004040B19B
:1026000009EBC90000EB091031684900B0FBF1F794
:1026100007E009EBC90000EB091031688900B0FB45
:10262000F1F76420B7FBF0F004012009642101FBFD
:102630001078A88900F4004040B1322000EBC800B7
:10264000B0FBF1F000F00700044308E0322000EB9B
:1026500008106421B0FBF1F000F00F0004432C815E
:10266000BDE8FF870010014000140140C1F30802DB
:102670008280704700BFFEE72DE9F0470546884697
:1026800091464646002700240CE0285D0744295D5A
:102690003046761C05F040FF10B90020BDE8F087F9
:1026A000601C84B24C45F0DBF9B23046761C05F074
:1026B00033FF08B90020F1E73046761CC7F3072145
:1026C00005F02AFF08B90020E8E70120E6E700004E
:1026D0002DE9F04106460D462F460B493046FFF7DF
:1026E000BBFD00240BE0084A115D38467F1C05F055
:1026F00013FF10B90020BDE8F081601C84B2F82CF3
:10270000F1D30120F7E70000880200200FB4024651
:1027100010B504A9034B039800F03AF810BC5DF81B
:1027200014FB0000313400080FB4054B10B503A9A9
:10273000044A029800F02CF810BC5DF814FB00006D
:1027400031340008580100200FB4084B10B504A91B
:1027500002AA039800F01CF8044602A9002000F029
:10276000F3F8204610BC5DF814FB0000492900086E
:1027700002E008C8121F08C1002AFAD1704770474A
:10278000002001E001C1121F002AFBD170470000A8
:102790002DE9FF4F8BB09A460F460546002606E00E
:1027A00025280BD052460D9990476D1C761C287831
:1027B0000028F5D10FB03046BDE8F08F0024A046C8
:1027C0000122604900E0044315F8013F203B02FA72
:1027D00003F00842F7D128782E2817D115F8010FF9
:1027E00044F004042A280ED06FF02F022878A0F1BC
:1027F000300109290AD808EB880102EB410100EBFE
:1028000001086D1CF2E757F8048B6D1C28786928C5
:102810003ED006DC0028CDD063280BD0642804D13C
:1028200036E0732810D075284BD052460D9990474A
:10283000761C85E017F8040B8DF8000000208DF859
:102840000100E946012003E057F8049B4FF0FF30F8
:1028500061074FF0000401D40AE0641C44450DDA1E
:102860008442FADB19F804100029F6D106E0641C52
:102870008442FCDB19F804100029F8D1264404E056
:1028800019F8010B52460D999047641EF8D257E093
:1028900001CF4FF00A0B002802DA40422D2102E05E
:1028A000210504D52B218DF82410012103E0E10737
:1028B00005D02021F7E70DF1200908910CE0002157
:1028C000F9E701CF4FF00A0BF9E75946FDF7D2FCC3
:1028D00001F1300209F8012D0028F6D1ADEB090015
:1028E00000F1200B600701D44FF00108D84502DD4C
:1028F000A8EB0B0000E000208046002406E009A8B9
:102900005246005D0D999047641C761C08988442DD
:10291000F5DB04E0302052460D999047761CB8F163
:102920000001A8F10108F5DC05E019F8010B524699
:102930000D999047761CBBF10001ABF1010BF4DC63
:102940006D1C34E7092801000A68531C0B601070E5
:10295000704700001FB504460122074B206ACDE9ED
:10296000000304F12703CDE90202044A1946204678
:1029700000F010FB04B010BDB68F0008B08F000847
:102980007FB504460D46206A002850D0206A0079A1
:1029900000284CD094F827008DF800002820005D16
:1029A0008DF801002920005D8DF802002A20005DCD
:1029B0008DF803002B20005D8DF804002C20005DB5
:1029C0008DF80500D5F80E000390A8690290206AE2
:1029D0000079012806D0206A0079022817D1206AE0
:1029E0004079A0B90398216A096888420BD00298FF
:1029F000216A0968884219D1062205F10801684652
:102A0000FDF71CFC90B1204600F05BF80EE0039847
:102A1000216A0968884209D1062205F10801684641
:102A2000FDF70CFC10B1204600F034F800BF7FBD6C
:102A30002DE9F04105460E462B214A5D2C21495DCA
:102A400042EA0121104A881800F032FD074602F0E0
:102A500009FC0446286A407A0444A0B20B4940EAC3
:102A600001040948844201D204F57E4408488442A6
:102A700001D9A4F57E4400BF00BF204600F018FD38
:102A80003060BDE8F08100000001FEA90000FEA951
:102A9000FFFEFEA970B50446012575B1206A007AD3
:102AA000002803DD204600F00CF809E02046FFF77F
:102AB00051FF6420216A087202E0204600F001F80C
:102AC00070BD70B505462C6A0026284602F040FB12
:102AD00010B1284602F05CFB00206860A860E86046
:102AE0006CB90A2002F098F9044614B94FF0FF308F
:102AF00070BD00202060606020812C6205E0002015
:102B00002071E08060712060207221462846FFF726
:102B10008FFF607A401C6072284600F002F8304651
:102B2000E6E710B5016A01220A7100224A712C22DF
:102B3000125C13062A22125C43EA02432922125C29
:102B400043EA02222B231B5C1A43036A13B1036A74
:102B50005B7A00E000231A440A23B2FBF3F403FB80
:102B60001422CA804A7A0A2A02DD4FF41672CA80F9
:102B700010BD70B505460C460021284602F028FF1E
:102B80000021284605F018F80021284604F0A8FE88
:102B9000204602F0E7F8284602F096FF70BD70B5B7
:102BA00004460E462546284602F0DCF870BD00BFFC
:102BB0000100A0F10100FBD1704700002DE9FC5F8E
:102BC00006468946174600BF0EB9BDE8FC9F00BF08
:102BD00078892A2803DA384602F0F3FCF5E7D7F8BB
:102BE000048008F10E04012000F06FFC2188884267
:102BF00015D140F2046000F068FCA18888420ED133
:102C00004FF4006000F061FC6188884207D140F613
:102C1000060000F05AFCB8F80C10884203D0384681
:102C200002F0CFFCD1E721463046FFF7A9FED4F8E9
:102C30000E000190A0690090706810B94FF0000A72
:102C400007E000987168884201D1012000E000206F
:102C50008246BAF1000F07D0012304F1080201A94E
:102C6000304605F0E3FB06E0002304F1080201A969
:102C7000304605F0DBFBE08800F027FC012802D09D
:102C800002283AD138E0BAF1000F33D0022000F028
:102C90001CFCE080D4F80E00A0617068C4F80E003F
:102CA00000BF00BF0625306A20B1306A007908B144
:102CB000154801E004F10800834614E0681EC5B21F
:102CC00004F10800415D0A3041551BF8050008F881
:102CD000050019F8051004F10800415519F8051010
:102CE00008F106004155002DE8DC39463046B2694E
:102CF000904700E000BF01E000E000BF00BF3846A1
:102D000002F05FFC00BF60E7B08F00082DE9F041E2
:102D100004460F4600BF0CB9BDE8F08100BF7D68D6
:102D200005F10E06F068A1680840D4E901121140CF
:102D3000884200D0F0E70023AA1D06F10C012046CE
:102D400005F074FB00BFE7E72DE9FC4104460E46A1
:102D500015460E21304602F06BFC18B16FF00100F1
:102D6000BDE8FC8100272146284601F02CF808B177
:102D7000254F40E04FF0704002F074FA296800EAF5
:102D800001084FF0604002F06DFA80451DD101202E
:102D90008DF8000000208DF801005E208DF8020003
:102DA000286802F05FFAC0F306408DF80300286837
:102DB00002F058FA000A8DF80400286802F052FA6E
:102DC000C0B28DF805006F4615E02868A16808407C
:102DD000D4E901121140884207D0E06810B104F133
:102DE0000C0502E06FF00300BAE7324629462046A0
:102DF00000F00CF8B4E73B4604F1270231462046C8
:102E000000F04AF9ACE70000B08F00082DE9F84F58
:102E100081460F46164609F1270A4FF0FF30009011
:102E20004946384600F0CFFF78B94FF0704002F0C5
:102E300019FA396800EA01054FF0604002F012FA11
:102E4000854202D00FB1386818B96FF00900BDE8AB
:102E5000F88F0121384600F0F5F90446002C01DA1C
:102E60002046F4E704EB8400494901EB8000807BB5
:102E700030B9012004EB8401454A02EB81018873DB
:102E800000BF00BF04EB8400414901EB8000807B60
:102E9000012800D02EB93946484600F0E7F80090E6
:102EA00000BF002E71D004EB8400394901EB800093
:102EB000807B02280CD104EB840001EB800000F140
:102EC000080352463146484600F0E6F800905CE0C0
:102ED00004EB84002E4901EB8000807B012854D153
:102EE0004FF0000B354608E000BF00BF287B0128EB
:102EF00002D04FF0010B02E02D68002DF4D100BF8D
:102F0000BBF1000F10D029890022032002F0B6F98E
:102F100005466DB13146284602F0AFFA40B1284669
:102F200002F04FFB002503E03546284602F0FBFB8C
:102F300055B3062002F0C0F88046B8F1000F1FD04C
:102F40000020C8F80000C8F8045004EB84001049C1
:102F500051F8200060B104EB84010D4A52F82100C1
:102F600000E0006801680029FBD1C0F8008004E09F
:102F700004EB8400064941F820800020009002E024
:102F8000284602F01EFB00BF00BF00985FE700006C
:102F9000184200202DE9FF4F83B0074689469A4624
:102FA000DDF840B00020029000222A21032002F028
:102FB00065F98046B8F1000F04D14FF0FF3007B03B
:102FC000BDE8F08F00BF00BFD8F8046006F10E0521
:102FD000139800F07AFAE88000BF00BF0624386A30
:102FE00020B1386A007908B11F4800E005980190C7
:102FF00012E0601EC4B21AF8041005F10800015571
:103000001198015D05F1120001550198005D3055E0
:1030100019F80410B01D0155002CEADCDBF80000A3
:10302000C5F80E0012980068A861012000F04DFA62
:1030300028804FF4006000F048FA688040F2046095
:1030400000F043FAA88040F6060000F03EFAB08196
:1030500041463846BA6990470290404602F0B1FABC
:103060004FF000080298AAE7B08F00087FB5044629
:103070000D460121064A201D04F127038DE8250095
:103080000391044A19462046FFF784FF04B070BD3F
:10309000B68F0008B08F00082DE9F04706460F46AE
:1030A000904699467D6800BF00BF062408E0601E78
:1030B000C4B219F80400285518F80410A81D0155C9
:1030C000002CF4DC4FF4006000F0FFF9A8813946D1
:1030D0003046B2699047BDE8F087000010B5002483
:1030E00046E004EB8400244901EB8000C07B401CD7
:1030F00004EB8401204A02EB8101C87304EB8400D5
:10310000114601EB8000807B022806D104EB84008D
:1031100001EB8000C07BF0280EDA04EB8400164936
:1031200001EB8000807B012820D104EB840001EBBF
:103130008000C07B022819DB04EB84000E4951F8A3
:10314000200060B104EB84010B4A52F8210000F02A
:1031500081F9002004EB8401074A42F82100002095
:1031600004EB8401044A02EB81018873601CC4B241
:103170000A2CB6DB10BD0000184200202DE9F041FA
:1031800004460D466668B08900F09FF90746B7F51A
:10319000006F03D0A7F60600E8B915E021462846DF
:1031A000FFF7B4FD6FF00D01204602F041FA30B197
:1031B00000BF00BF204602F004FA002403E02946C5
:1031C000204600F0CDFE0BE0224605F127012846FF
:1031D000FFF7F4FC04E0204602F0F3F9002400BFFE
:1031E00000BF0020BDE8F08110B5044600BF00BF5D
:1031F000732084F82E0074212F200155044860614B
:103200000448A061204601F0B5FA002010BD00007E
:10321000492D0008B948000870B50446204601F061
:10322000F5FA064616B94FF0FF3070BD214630461C
:103230002269904705461DB1304602F0C2F90026CA
:103240002846F2E72DE9FC5F05460F464FF00A08D5
:10325000C1460A260024A34600200190B2460090F1
:10326000CDB17148007800EB8000704901EB80001F
:10327000807B02280FD128686B49097801EB810116
:103280006A4A02EB81014968884204D166480078A5
:1032900040B2BDE8FC9F002473E00A2E08D104EB85
:1032A0008400624901EB8000807B08B966B266E069
:1032B00004EB84005D4901EB8000807B012836D15E
:1032C00065B1286804EB8401584A02EB8101496822
:1032D000884203D15448047060B2DAE704EB8400FA
:1032E000524951F8200088B104EB840001EB8000C2
:1032F000C17B0098814242DB4FFA84FA04EB8400E0
:103300004A4901EB8000C07B009038E004EB840068
:10331000464901EB8000C07B584530DB4FFA84F80A
:1033200004EB840001EB800090F80FB027E004EB81
:1033300084003E4901EB8000807B02281FD165B1EB
:10334000286804EB8401394A02EB8101496888420C
:1033500003D13548047060B29BE704EB8400334925
:1033600001EB8000C17B0198814208DB4FFA84F9B0
:1033700004EB84002D4901EB8000C07B0190601CB0
:10338000C4B20A2C89DB0A2E02D107F0010010B169
:1033900007F0020010B14FF0FF307AE70A2E01DA91
:1033A000F4B222E0B9F10A0F03DA09F0FF0400BF1A
:1033B0001BE0B8F10A0F02DA08F0FF0415E0BAF1D9
:1033C0000A0F0FDA0AF0FF0404EB8401174A52F8DF
:1033D000210000F03FF8002004EB8401134A42F87A
:1033E000210002E04FF0FF3053E700BF00BF002094
:1033F00004EB84010D4A02EB8101887345B105B9E4
:1034000000E0286804EB8401084A02EB810148606F
:10341000002004EB8401054A02EB8101C8730248D5
:10342000047060B235E7000030010020184200202F
:1034300070B504460D4600BF40210548FFF79EF8D1
:103440000028F9D0E1B20248FFF710F9204670BD1C
:103450000010014070B5044600BF00BF00BF00BFB0
:103460000AE02546246800BF00BF686802F0A9F89A
:103470002946062001F0DEFD002CF2D170BD0000CF
:1034800070B506460D46094C0BE030466168FCF706
:10349000C7FE28B9A0682860E0686860012070BD98
:1034A0002468002CF1D10020F9E70000448E0008C8
:1034B0000146080601F47F4240EA022001F47F023F
:1034C00040EA122040EA1160704701460806000CED
:1034D00040EA1120704700002DE9F04106460D46F4
:1034E0001746082001F098FC04461CB94FF0FF3045
:1034F000BDE8F0810020206060602146284602F08F
:1035000067FA0749284604F0EBF90649284602F015
:103510006BFD0A220449284603F002FC0020E7E77D
:10352000493500089F2B00082D35000870B504466A
:103530000D461CB9284602F0C7FA03E0214628468A
:1035400002F077F9002070BD2DE9FF4F8FB0834660
:10355000904600250020009001905E4612980028B9
:1035600038D1B8F1000F35D0B8F80810109804F031
:10357000D1F93068002878D1D8F80470B8F808502C
:103580000522F7A13846FCF766FE002845D1112236
:10359000F5A13846FCF75FFEE8B9F8480078022844
:1035A00019D10320F54908706946F5A0FFF768FFB7
:1035B0000098306001987060404602F002F8314691
:1035C000109802F036F90120F0490870F04910987F
:1035D00004F0F2FAC2E1EF48007838B10020E74980
:1035E00008706946ECA0FFF74BFF06E00120E349B5
:1035F00008706946EBA0FFF743FF00983060019820
:103600007060404601F0DDFF3146109802F011F97C
:10361000DF49109804F0D0FAA0E11422E5A1384661
:10362000FCF719FE00283CD1D4480078002838D196
:10363000002433E038190922E4A1FCF70CFE00282D
:103640002BD1E5A3E4A2E6A102A8FFF77DF8381983
:103650001D2202A9FCF7FFFD40B90120C7490870EF
:103660006946D0A0FFF70CFF07E070E10020C349D6
:1036700008706946C8A0FFF703FF00983060019802
:103680007060404601F09DFF3146109802F0D1F87D
:10369000BF49109804F090FA02E0641CAC42C9DB08
:1036A0005CE11022D4A13846FCF7D5FD18B1D7480B
:1036B000006800287CD0B1480078012878D14FF00C
:1036C0000009D248006890BB0020D1490860D14968
:1036D0000860B8F808103846FEF73EFBCE4908608F
:1036E000002409E038190D22CC49FCF7B4FD10B9CB
:1036F00004F1100902E0641CAC42F3DB00BFB9F135
:10370000000F0ED1C1480068401CC049086001206C
:10371000BF490860404601F054FF002013B0BDE8E7
:10372000F08FBF480068001D281ABA490860B748E2
:103730000068012803D1B6480068012807D0B348C3
:103740000068002872D1B24800680028FAD1AF485A
:10375000006840B9AE48006828B9AC480068401C11
:10376000AA49086020E0A948006801281CD1A8489F
:103770000068012818D1002409E038190D22A74952
:10378000FCF769FD10B904F1100902E0641CAC42B9
:10379000F3DB00BF9F48006828449E4908609B48AF
:1037A0000068401C994908604FF0000A00240AE0B4
:1037B000C5E0381909229BA1FCF74DFD10B904F1B1
:1037C0000A0A02E0641CAC42F3DB00BF0024BAF139
:1037D000000F10D005E007EB0A00005D0AA90855AC
:1037E000641C07EB0A00005D222801D00D2CF2DBDF
:1037F00000200AA90855D4B901206049087069461B
:1038000068A0FFF73DFE0098306001987060404668
:1038100001F0D7FE3146109802F00BF85C49109881
:1038200004F0CAF900207949086077E71CE080A11C
:103830008548FEF76BFF0AAA84A18348FEF766FF5E
:1038400086A18148FEF762FF00208A490860FDF7E3
:103850002BFC8948FDF70AFC87488849086088A145
:103860007948FEF753FF04E06A4800682844694934
:10387000086007EB09000E90A5EB09057D4800687C
:1038800028447C4908600846006884490968401A51
:10389000B0F5205F07D9774800688049086080A1AB
:1038A0006948FEF733FF5B4800685B490968884256
:1038B0003CD1042400E0641CB8F808103944081B0B
:1038C00004227849FCF7C7FC0028F4D12D1B694875
:1038D0000068001B674908601DB129460E98FDF776
:1038E000C5FD002049490860624802686EA156483B
:1038F000FEF70CFF75A15448FEF708FF79A1524866
:10390000FEF704FF02201D490870694676A0FFF704
:10391000B7FD00983060019870603146109801F052
:1039200088FF1B49109804F047F904E01DB12946AF
:103930000E98FDF79BFD404601F043FE0EE0404629
:1039400001F03FFE31461098FFF713F906E04046BC
:1039500001F037FE31461098FFF70BF90020DDE645
:10396000474554202F000000474554202F726573AF
:1039700065746D63752E6367690000004C0000205C
:103980002F72657365742E68746D6C0035000020AD
:10399000FD3A0008640000202F696E6465782E6887
:1039A000746D6C002F75706C6F61642E68746D6C33
:1039B00000000000504F5354202F636865636B6C08
:1039C0006F67696E2E63676900000000757365722A
:1039D0006E616D653D00000069736B7261000000EF
:1039E000757365726E616D653D25732670617373C5
:1039F000776F72643D257300504F5354202F7570BC
:103A00006C6F61642E636769000000002000002075
:103A10003C0000202C00002024000020588E0008CC
:103A20003800002066696C656E616D653D000000C0
:103A30002020494150207573696E672048545450C6
:103A400020200D0A00000000540100202046696C6F
:103A5000653A202573200D0A000000002053746190
:103A600074653A2045726173696E672E2E2E0D0AB9
:103A70000000000040000020000001082800002095
:103A80002053746174653A2050726F6772616D6D76
:103A9000696E672E2E2E0D0A0000000048000020DF
:103AA000B1000000548E000820546F7420627974B5
:103AB00065732052656365697665643A20256420E4
:103AC0006279746573200D0A0000000053746174FC
:103AD000653A2050726F672046696E697368656445
:103AE000200D0A000D0A00002F75706C6F61646470
:103AF0006F6E652E68746D6C000000002DE9F0415A
:103B000004460D4617462646706820B131462846C1
:103B100001F08FFE18E031462846FFF72AF80C48DE
:103B20000078012810D100BFBFF34F8F094800680B
:103B300000F4E06008490843001D06490860BFF32F
:103B40004F8F00BF00BFFEE70020BDE8F0810000FE
:103B5000350000200CED00E00000FA0570B50546C8
:103B60000C4622460321284600F0B9F870BD2DE925
:103B7000FF5F054689466C68208801F079FBC0F339
:103B800003204FEA8008C8F10001284601F050FDEB
:103B900010B92889042800D298E0686890F800A03D
:103BA000BAF1080F7CD101264FF0704001F05AFBAA
:103BB000216900EA010B4FF0604001F053FB83459F
:103BC00000D10026494604F1100000F0FCF800B1D5
:103BD000002626B9284601F0F4FCBDE8FF9F28899D
:103BE000082800D272E0284600F0C2F818B1284632
:103BF00001F0E7FCF1E72221284601F019FD48B366
:103C00004146284601F014FD10B100BF00BF61E03D
:103C100029890022022001F031FB064606B959E04D
:103C200000BF00BF2946304601F027FC10B100BF9D
:103C300000BF4FE07468C8F1000001B2304601F0E7
:103C4000F7FC10B100BF00BF44E0284601F0B9FC0A
:103C5000354608E06FF02101284601F0E9FC10B17B
:103C600000BF00BF36E06F68E06803902069E06045
:103C700003982061002038707880208901F0F8FADC
:103C8000C0B240F47F463046FFF71FFC2081002081
:103C900060814146284601F0CBFC10B100BF0EE028
:103CA0000EE001200021FF230A46CDE90109009121
:103CB00004F10C01284600F03BFA064600BF00E084
:103CC00000BF00BF284601F07CFC86E7284601F0D3
:103CD00078FC82E7284601F074FC00BF7DE72DE9FF
:103CE000FC4706460F46904600222421012001F0A1
:103CF000C5FA05460DB9BDE8FC8700BF00BFD6F880
:103D000004906C68277084F801800020A080E08017
:103D100071686A6802F108001C22FCF751FA002061
:103D200060806989204600F019F860800120002138
:103D3000FF2309F10C02CDE90010284600F0DEF95E
:103D4000284601F03EFC00BFD5E770B505460C469D
:103D500022460B212846FFF7C2FF70BD70B504460E
:103D60000D462946204600F0C3FDC04380B270BD19
:103D70002DE9F041064600240027354617E0698901
:103D8000686800F0B5FD0444A0B200EB14446889F3
:103D900000EBD0714910A0EB410139B1C7F101002E
:103DA000C7B2E0B2C4F3072141EA00242D68002D18
:103DB000E5D127B1E0B2C4F3072141EA0024E04392
:103DC00080B2BDE8F08130B503461A68D04300B137
:103DD0000AB9012030BD91F82D0000F0020008B9A9
:103DE0000020F7E74868904201D10020F2E7186808
:103DF0008C682040D1E901452C40A04208D1886858
:103E000022EA00008D68EC43A04201D10120E1E7E5
:103E10000020DFE72DE9F74F86B08846B8F8240088
:103E200005901420019002220021104601F026FA8C
:103E3000054625B94FF0FF3009B0BDE8F08F059871
:103E400068812881454820F0030068606C68069806
:103E5000142241682046FCF7B3F9E08801F008FA23
:103E60000746C7F30C00049007F40050039006982F
:103E70000089143886B20599A1F11400C11700EB2E
:103E80005171C1F3CF0B61E005981438B04201DBEA
:103E9000012000E0002002900498C0F30C00039978
:103EA00040EA0107029808B947F40057029808B1A0
:103EB000304601E04FEACB001FFA80FA524604F187
:103EC0001401019B069801F033FB0199084480B26C
:103ED00001903846FFF7F9FAE0800AF1140188B240
:103EE000FFF7F3FA60800020608114212046FFF77D
:103EF00035FF6081029828B106F1140081B228468E
:103F000001F0D5FB00221146022001F0B7F98146ED
:103F1000B9F1000F0DD02946484601F09AFAD8F8B9
:103F2000143049464046089A9847484601F049FBF4
:103F300005E0284601F045FB4FF0FF307CE7A6EB9B
:103F40000A0086B20498584480B20490002E9BD197
:103F5000284601F036FB00206EE7000083030020B6
:103F60002DE9F04706460F467468208801F080F975
:103F70000421B1EB203F05D0304601F022FB0020A8
:103F8000BDE8F087208801F073F9C0F303294FF6EC
:103F9000FF7000EA8909608801F06AF9804670893B
:103FA000484502DB3089404504DA304601F009FB20
:103FB0000020E5E74146304601F079FB4FF0010A69
:103FC0003D4600BF284601F0C3F870B1281D60B11E
:103FD000686850B120696968884205D0294604F1B3
:103FE0001000FFF7F0FE00B10DE0BAF1000F04D0B1
:103FF0004FF0000A3E48056800E02D68BD4200D140
:104000002D68002DDED100BF394604F10C00FFF70A
:10401000DAFE60B94FF0704001F024F9E16800EA7F
:10402000010A4FF0604001F01DF9824504D130468D
:1040300001F0C7FA0020A3E725B9304601F0C1FA24
:1040400000209DE743F6FF70FFF73FFAE188084044
:1040500038B1304600F0EAF806460EB900208FE786
:10406000746824480760244804603946304601F0EB
:10407000A3FBA8BB208901F0FBF8C0B201280DD03A
:10408000062806D011280ED13946304604F058F8DB
:1040900025E03946304601F0E7FF20E0394630465A
:1040A000FFF765FD1BE0394604F11000FFF78BFEBA
:1040B00088B94FF0704001F0D5F8216900EA010A93
:1040C0004FF0604001F0CEF8824504D074600221C8
:1040D0003046FFF743FD304601F073FA00BF00BFE2
:1040E0000020044908600449086000BF48E7000058
:1040F000B400002094000020980000202DE9FE4F1D
:1041000005460E4614461F46DDE90C89204600F0A0
:10411000CFFA5FEA000A02D1001FBDE8FE8F3B46DE
:104120002246314628468DE8000700F001F8F4E702
:104130002DE9F05F06460F4690469A460C9DB8F171
:10414000000F5BD04FF014091421304601F070FAD3
:1041500018B16FF00100BDE8F09F746800BF00BFA8
:10416000208901F085F86AF31F208346FFF7ADF937
:104170002081208901F07CF801120B9840EA012B84
:104180005846FFF7A2F92081B8F1000F01D10020B5
:1041900001E0D8F800002061CB464FEAE97109EB55
:1041A000917189104FF4804242EA01210A9A114329
:1041B00088B2FFF78AF920803089FFF786F960809E
:1041C0000020E08018480088FFF77FF9A08016489B
:1041D0000088401C144908800FB1386830B9281D88
:1041E00008B9002000E06868E06004E00FB9002032
:1041F00000E03868E0600020608102E0746804F14B
:104200001008A88C48B13089A98C884205DD424647
:1042100029463046FFF7FEFD9DE7424631462846D7
:104220006B69984797E700009C0000202DE9FC5F30
:10423000804600200090D8F80450288801F018F833
:10424000C0F303201421B1EB800F00D0B1E0E88867
:1042500001F00EF8C0F30C004FF6FF7101EAC00A3E
:10426000688801F005F88346288801F001F8C0F35A
:104270000320ABEB800080B20190404601F0F4F8DF
:1042800006464E48018888190A280ADD3146284624
:1042900000F0D0F920B14948008830440A2800DDF8
:1042A00087E04748046812E06069E968884209D1FC
:1042B000A0692969884205D1A089A988884201D1CD
:1042C000012000E0002000B103E000942468002CED
:1042D000EAD100BF34B93146284600F03DF9044622
:1042E00094B966E0E88800F0C3FFC0F30C0058B949
:1042F000E08900F0BDFFC0F30C0028B1142229466C
:1043000004F10800FBF75CFF2C48008830442B497F
:104310000880E88800F0ACFF00F4005030B9A07FBE
:1043200040F00100A07701985044A0834146204608
:1043300000F048F8D0B3A08B1430A08360684068C8
:10434000076860684568142204F108012846FBF7F5
:1043500037FFA08BFFF7B9F868800020E8806881FC
:1043600014212846FFF7FAFC6881D4F804800CE099
:10437000D7F804906FF01301384601F059F9394627
:10438000404601F04AF8D9F80070002FF0D12046DD
:10439000009900F0CBF8404601F066F8074909881B
:1043A000081A064908804046BDE8FC9FFFE7002048
:1043B000FAE7404601F005F90020F5E790000020FB
:1043C0008C0000202DE9FE4F81460E46002501207D
:1043D0000090D6F804A0BAF8020000F049FF834626
:1043E000BAF8000000F044FFC0F30320ABEB8000FC
:1043F00080B20190BAF8060000F03AFFC0F30C005A
:104400004FF6FF7101EAC000029000BF00BF746860
:10441000002020600298A080DDE901100844E080BF
:10442000D9F804802AE0D8F80470A088B9888842B6
:1044300010DAC4F8008055B1A088E988884203DB0F
:10444000E088B988884200DD60E02E6001E0C9F8AC
:10445000046016E0A088B988884200D156E0A088A0
:10446000F988884200DA51E02DB1E888B98888429D
:1044700001D000200090D7F800803D46B8F1000F31
:10448000D1D100BFB8F1000F0ED14DB100BF00BFB8
:104490002E60E888A188884206D00020009003E0C2
:1044A00000BF00BFC9F8046099F81E0000F00100C9
:1044B00050B3009828B3D9F804004068808810B140
:1044C000002000901DE02546D4F800800BE0D8F8CD
:1044D0000440E888A188884202D00020009005E0CE
:1044E0002546D4F80080B8F1000FF0D100BF009845
:1044F00038B100BF00BF00BF00BF00BF00BF00BF9A
:1045000000BF0098BDE8FE8F0020FBE7304600F0BA
:10451000ABFF05490988081A03490880304601F0B5
:1045200050F80020EEE700009000002070B504462F
:104530000D4608480068A04203D10649206808607B
:1045400003E000BF00BF206828602146052000F07E
:1045500071FD70BD8C00002070B505460E4605202B
:1045600000F0AAFD044664B93146284600F062F81E
:10457000B04203DB052000F09FFD04460CB900208B
:1045800070BD20212046FBF734FE0320E07706486B
:1045900000682060044804601422294604F10800E1
:1045A000FBF70EFE2046EBE78C0000202DE9F047DC
:1045B00004468846002600BF00BFB8F1000F01D0B6
:1045C00000BF00BF60684768B88898B965683868F8
:1045D0006060142204F108016868FBF7F1FD012115
:1045E0002846FFF7B2FB284600F03EFF0644284667
:1045F00000F0E7FF65680AE06F68A9463D68484635
:1046000000F032FF0644484600F0DBFF00BF002DFB
:10461000F2D141462046FFF789FF00BF00BF0448A2
:104620000088801B024908803046BDE8F087000002
:10463000900000202DE9F05F05468946002700BF65
:104640000026B346B246194804681DE06069E9686F
:10465000884207D1A0692969884203D1A089A98825
:10466000884201D0012000E0002048B10AF1010A8F
:104670000EB9264604E0E07FF17F884200DC264642
:10468000206800B1A3462468002CDFD12EB1594622
:104690003046FFF78BFF804647444F4502DABAF1B8
:1046A000010FCDDC3846BDE8F09F00008C000020F3
:1046B00070B50546104804680EE0204600F048FD3D
:1046C00048B12868A1680840D4E901121140884225
:1046D00001D1204670BD2468002CEED10748006847
:1046E00020B10648006800F033FD08B90020F1E76A
:1046F00002480068EEE70000B4000020B800002087
:10470000F0B502460C460023591E2FE01578302DD7
:104710000FDB1578392D0CDC002900DA0021157823
:10472000303D01EB810605EB4601FF291DDD002030
:104730001DE015782E2D0BD1042B09DA002901DAA2
:10474000002014E01D465B1C61554FF0FF310CE06A
:10475000157845B9032B06D1002901DA002001E0C4
:10476000E154012003E0012001E0521CCEE700BF2C
:10477000F0BD000070B50446062084F826001E48EF
:10478000007884F827001C484178282001551A48F1
:104790008178292001551848C1782A2001551648EA
:1047A00001792B200155144841792C20015504F141
:1047B00027010020FCF73AF940F2DC50A0843220B7
:1047C00084F82D0005220D490D48FBF7FBFE05225C
:1047D0000C490D48FBF7B2FE002507E0084901EB44
:1047E00045104FF44001FBF715FF6D1C052DF5DB5F
:1047F000FCF74EFA70BD000050000020E46100207C
:104800008043002020440020E04200202DE9F04FAA
:1048100087B083460027B846002601A8FBF78CFF27
:1048200001A807C804AB07C304981FFA80F9DDF894
:1048300014A003224946104600F020FD064666B14A
:10484000344608E062890AEB07016068FBF7B8FCB0
:10485000608907442468002CF4D1154800688068FA
:10486000012803D912480068056800E0069D4FF052
:10487000000805E04FF000402860ED6808F10108ED
:104880000B48006880684045F4D800200849096852
:1048900088600848406900F0800020B18020054908
:1048A000486100208860304607B0BDE8F08F000006
:1048B0004C010020009002402DE9F04180460E4658
:1048C00000250A4800688768344607E0628978193D
:1048D0006168FBF775FC608905442468002CF5D1FC
:1048E000A8B2FCF721F90020BDE8F08144010020C6
:1048F0002DE9F04180460E460024454608E0287820
:1049000007026D1C287807436D1C3C44B01E86B21C
:10491000012EF4DC002E02DD287807023C44A0B210
:1049200000EB1444200C000410B1A0B200EB1444BE
:10493000A0B2FEF7CAFDBDE8F081F0B502460C4614
:104940000023591E52E01578412D02DB15785A2DAF
:104950000BDD1578612D02DB15787A2D05DD1578D4
:10496000302D23DB1578392D20DC002900DA0021D9
:104970001578302D07DB1578392D04DC1578303D9E
:1049800005EB01110EE01578412D07DB15785A2D46
:1049900004DC1578373D05EB011103E01578573D30
:1049A00005EB0111FF2920DD002020E015782D2DD9
:1049B00002D015783A2D0BD1062B09DA002901DA3D
:1049C000002014E01D465B1C61554FF0FF310CE0E8
:1049D000157845B9052B06D1002901DA002001E040
:1049E000E154012003E0002001E0521CABE700BFCE
:1049F000F0BD000008B5FBF7AFFCFCF797FCFCF737
:104A000019FC00208549087008218548FCF715FD30
:104A1000012811D04FF480618148FCF70EFD012878
:104A20000AD0FDF7E1FC7FA18848FDF76FFE88A161
:104A30008648FDF76BFE89E0FDF7D6FC79A1834837
:104A4000FDF764FE8AA18148FDF760FE91A17F48D1
:104A5000FDF75CFE944C00252E460DE0934B944AE6
:104A6000D4E9001059405040014300D107E0D4E997
:104A700000104D40464008348E488442EED300BFBB
:104A8000002185EA01007140084304D08AA16F48E3
:104A9000FDF73CFE5AE08BA16C48FDF737FE8248DB
:104AA00000688A490840B0F1005F06D07E4800687F
:104AB00087490840B0F1805F01D1012000E000206B
:104AC0005649087083A16148FDF720FE04224FF487
:104AD00001716846FDF75EFA80B186490098884208
:104AE0000CD10020009084A15848FDF70FFE04224D
:104AF0004FF401716846FDF7BFFD27E081A15348DF
:104B0000FDF704FE00218248FDF7A6FA81A14F4877
:104B1000FDF7FCFD4148007898B16AA14B48FDF7CC
:104B2000F5FD614840688149086008460068804991
:104B300008605D49086880F3088800BF7C48006809
:104B400080475DA14148FDF7E1FD00BFFCF7C8FFCC
:104B5000002000902EE0009800F0010058B130488D
:104B6000408B40F010002E4948830846008B40F0EF
:104B7000200008830AE02A48008B40F010002849F2
:104B800008830846408B40F020004883002700E05F
:104B90007F1C68488742FBDB2148008B40F01000F7
:104BA0001F4908830846008B40F0200008830098C6
:104BB000401C009000980F28CDDBFDF779FB5EA12B
:104BC0002248FDF7A3FD00225F496048FDF70CFA7B
:104BD0005F495E48D030FFF7B0FE5E495B48FFF7A3
:104BE0008FFD5D4959482030FFF78AFD5B495748E2
:104BF0001030FFF785FDFBF7EFFBFCF78BFFFCF7B1
:104C000097FCFCF70FFE08E0FBF722FC08B1FDF76C
:104C100051F853480068FDF72FF8F5E764000020CD
:104C200000000240426F6F742073797374656D20C9
:104C300073746172742C2076657273696F6E203A9A
:104C400020322E30322E2E2E0D0A0000540100206C
:104C5000436865636B20626F6F7420627574746F54
:104C60006E202E2E2E204163746976650D0A000099
:104C7000436865636B20626F6F7420627574746F34
:104C80006E202E2E2E2052656C65617365640D0AB0
:104C900000000000436865636B2043524320524F7D
:104CA0004D202E2E2E000000000001089CD9E6D8D1
:104CB0003A4DD4D2FFFF07084641494C45440D0AFE
:104CC000000000004F4B0D0A000000000000FE2F06
:104CD0000000FF1F436865636B20626F6F7420667E
:104CE0006C616720696E20656570726F6D202E2E75
:104CF0002E20000055AA55AA4163746976650D0AF5
:104D000000000000496E6163746976650D0A000059
:104D100000380040436865636B20524F4D20636F3D
:104D20006E746578742E2E2E200000007400002012
:104D300070000020A0860100426F6F7420737461C0
:104D400072742E2E2E0D0A00788E00085C01002051
:104D500050000020580000205C000020600000206F
:104D60006800002070B5054605B970BD00BF00BFE2
:104D700000BF00BF0C480068854203D30B480068A1
:104D8000854200D3F1E7A5F1080400BF00BF002071
:104D9000207107480068844201D20548046020461B
:104DA00000F0C6FC00BFE0E7A4000020A80000203F
:104DB000AC00002000BF00BF124921F00301124ADD
:104DC0001160114608684FF4805101800021418034
:104DD00001711146096801F580510C4A11600121E9
:104DE000126811710903094A12681180074A126892
:104DF00051800121064A117003490968054A116072
:104E00007047000063090020A4000020A8000020D3
:104E1000B0000020AC00002070B502460AB90020A6
:104E200070BDD01C20F0030082B20C2A00DA0C22E4
:104E3000B2F5805F01DD0020F2E730480088304E97
:104E40003688801B83B253E02D480068C11808796A
:104E500000284AD10E8803F10800301A904244D34A
:104E60000E8803F10800361A02F11400864218D3A6
:104E700003F10800104485B221480068441900205D
:104E800020710888208063800D80012008712088AF
:104E9000B0F5805F07D02088194E366830444580D1
:104EA00001E00120087115480068814214D107E033
:104EB000124800680088124E366830440F4E306049
:104EC0000E480068007928B10C4800680D4E36681D
:104ED000B042EDD100BF00BF00BF00BF00BF00BFA8
:104EE00000BF00BF01F108009AE705480068C35AF7
:104EF000C2F580509842A7DC002091E7AC0000206A
:104F0000A4000020A80000202DE9F04106460A4632
:104F1000D01C20F0030082B20C2A00DA0C22B2F579
:104F2000805F02DD0020BDE8F08100BF00BF3E4889
:104F30000068864203D33D480068864201D330466C
:104F4000F1E7A6F1080438480088201A85B22088C5
:104F5000401B083887B200BF00BFBA4201DD002005
:104F6000E1E7BA4201D13046DDE72088DFF8B8C07A
:104F7000DCF800C000EB0C01087980BB088805F163
:104F8000080C94441FFA8CF3DFF8A4C0DCF800C0CE
:104F90008C4508D1DFF890C0DCF800C09C44DFF8F5
:104FA0009080C8F800C0DFF880C0DCF800C00CEBCF
:104FB00003014FF0000C81F804C008804D8023806D
:104FC000B1F800C0BCF5805F08D0B1F800C0DFF8D0
:104FD0005880D8F80080C444ACF8023022E0FFE7E3
:104FE00002F11400B8421DD805F10800104483B244
:104FF0000D480068C1180E480068814201D20C4873
:10500000016000200871208808804D802380088876
:10501000B0F5805F06D00888DFF80CC0DCF800C06F
:105020006044438030467EE7A4000020A8000020B2
:10503000AC00002001B9704700BF00BF0A46044B16
:1050400053F820301360024B43F8202000BFF2E7F2
:105050007419002010B5002001E0431C98B2092803
:10506000FBDB114B23F00301002019E000230F4C60
:1050700044F8203000220CE00C4B53F820300B6039
:105080000A4B43F820100A4B33F810301944531CD4
:105090009AB2084B33F810309342EDDC431C98B2BF
:1050A0000928E3DB10BD00009B19002074190020C3
:1050B000788F00088A8F0008024600BF092A01DBAA
:1050C0000020704700BF064850F8221031B1044B51
:1050D000086843F8220000BF00BF00BF0846F0E7A1
:1050E000741900202DE9F04704460D4616461F4668
:1050F000DDE909A9DDF8208000206060A060E060A3
:1051000084F82D002062C4F81C800F48007884F8D1
:1051100030000D480078401C0B490870C4F810900E
:105120003B4632462946204600F018F82046D04734
:1051300010B10020BDE8F0870448006820600348F3
:1051400004602046F6E70000BC000020B400002008
:10515000014691F82D0000F0010070472DE9F04163
:1051600006460F4614461D463946304600F022F8E2
:105170002146304600F05AF82946304600F014F82F
:10518000BDE8F0810149086070470000B8000020C8
:1051900090F82D1001F0010129B190F82D1021F0A7
:1051A000010180F82D10704709B9002200E00A685B
:1051B000C26070472DE9F04107460D4628687968BE
:1051C000884201D1012000E0002018BB1548066884
:1051D0000CE030687968884207D1D6F80C8001214C
:1051E000304600F045FB464600E0F668002EF0D160
:1051F0000D4804680CE054B1206840B1206879681B
:10520000884204D10DB9002000E028682060E468DD
:10521000002CF0D10DB9002000E028687860BDE8CE
:10522000F0810000FC000020F800002009B90022F5
:1052300000E00A688260704710B5044694F82D00BB
:1052400000F0010068B914F82D0F40F00100207043
:1052500014F82D0900F0200018B1211D2046FDF79B
:1052600005FF10BD00B503461846FEF721F900BD45
:1052700000B502461046FEF728F900BD2DE9F05FA3
:1052800083460F4690460026BBF1000F09D0BBF1C4
:10529000010F0AD0BBF1020F0BD0BBF1030F0DD1F0
:1052A0000BE006F1140086B200BF06F1140086B2CE
:1052B00000BF06F10E0086B205E004E000BF00BFAB
:1052C0000020BDE8F09F00BFB8F1000F68D0B8F132
:1052D000010F74D0B8F1020F72D0B8F1030F70D182
:1052E0000820FFF7E9FE04460CB90020E9E784F83E
:1052F0000C800020206006F110002044C01C20F02B
:105300000300606000BF00BF2781F01C20F0030095
:10531000C0F5BE60B84201DD384604E0F01C20F064
:105320000300C0F5BE60608100BF00BF00BF00BFCA
:105330000120E081A2466089A7EB00092CE008204B
:10534000FFF7BAFE054625B9204600F03AF90020DD
:10535000B7E785F80C80002068732860CAF8005011
:1053600000BF00BFA5F808901FFA89F0B0F5BE6F26
:1053700002DA1FFA89F001E04FF4BE60688105F19E
:105380001000686000BF00BF00BF00BF0120E881BF
:105390006889A9EB0009AA46B9F1000FCFDC35E016
:1053A00006F1130121F00302F91C21F0030111445D
:1053B00088B2FFF731FD044624B9002081E711E0EF
:1053C00011E01FE004F110003044C01C20F0030085
:1053D0006060278167810020206084F80C8000BF16
:1053E00000BF13E000BF0720FFF766FE04460CB9BC
:1053F000002066E70020606027816781206084F8D4
:105400000C8003E000BF00BF00205AE700BF01206E
:10541000E08100206073204653E710B5024600BFCC
:1054200002B101B910BD00BF104604E003890C8928
:105430002344038100680368002BF7D100BF00BF3D
:1054400000BF00BF03890C8923440381016000BFB2
:10545000E8E730B505460C4621462846FFF7DDFF54
:10546000204600F060F930BD0146002002E0421CF9
:10547000D0B209680029FAD170472DE9F0410546FC
:105480000C460026002700BF25B11CB128892189C0
:10549000884203DA6FF00900BDE8F08100BF00BF69
:1054A00000BF00BF6889801B6189C91B884204DB7B
:1054B0006089C01B1FFA80F803E06889801B1FFA0F
:1054C00080F86268D1196A6890194246FAF778FE46
:1054D00006EB080086B207EB080087B200BF00BFEA
:1054E0006889B04201D100262D6800BF00BF6089E5
:1054F000B84201DC0027246854B1608921898842C0
:1055000006D100BF206810B16FF00800C4E700BFEB
:1055100055B168892989884206D100BF286810B131
:105520006FF00800B8E700BF002CB9D10020B3E746
:105530002DE9F05F8046894616461D464FF0000B68
:1055400000BFB8F1000F02D10020BDE8F09F00BFFE
:1055500000BFB9F1000F01D10020F6E700BF4FF006
:10556000000AB8F1000F02D0B9F1000F01D10020FC
:10557000EBE7444620E035B16089A84203DC60894E
:10558000281A85B217E06089401B87B2B74200DD58
:1055900037466268511909EB0A003A46FAF710FEDD
:1055A0000BEB07001FFA80FB0AEB07001FFA80FADB
:1055B000F01B86B2002524680EB1002CDBD15846C2
:1055C000C3E72DE9F041044624B900BF00BF002025
:1055D000BDE8F08100BF00BF002625E000BF00BF8E
:1055E000E089401E1FFA80F8A4F80E80B8F1000F81
:1055F00018D12768257B032D04D121460820FFF709
:1056000019FD0BE0012D01D0022D04D12146072008
:10561000FFF710FD02E02046FFF7A4FB701CC6B2A6
:105620003C4600E0002400BF002CD7D13046CFE735
:1056300070B5024600BF00BF01B10AB9002070BDBD
:10564000002908DA484284B200BF5089A04201DA3A
:105650000120F4E700E08CB2137B55680BB1032BFB
:105660000AD15068401A506002F110005668864214
:1056700015D255600120E2E7022B01D0012B0AD19F
:10568000002906DA5089A04203DB5068401A5060B6
:1056900005E00120D3E700BF00BF0120CFE750891C
:1056A000084450811089084410810020C7E72DE983
:1056B000F04106460F4600BF00BF00BF00BF308963
:1056C000B84201DCBDE8F0813089A7EB00083D4617
:1056D00034460AE06089281A85B200BF00BF2089DD
:1056E00040442081246800BF00BF6089A842F1DBEC
:1056F000207B60B96089A84209D0A088001B28449B
:1057000081B22046FFF700FC044600BF00BF658160
:1057100060892081206810B12068FFF752FF0020C7
:10572000206000BFCEE710B1C189491CC18170471C
:1057300030B500BF00BF00BF00BF00BF00BF00BF4B
:1057400000BF0388194C24681919884215D00B79B9
:105750009BB9174B1B6899420FD0164B1B688B42A5
:1057600001D1144B18600B880380104B1B88C31A9F
:105770000C880E4D2D682C44638043880B4C2468A4
:105780001A19824211D013797BB90A4B1B688342E4
:1057900001D1084B1A6003881380044B1B88D31A6D
:1057A0000488024D2D682C44638030BDA400002085
:1057B000A8000020AC0000202DE9F04705468A46ED
:1057C0004FF000086F683889FFF752FD00F0FF09BD
:1057D00000261248046819E0207C484514D160690D
:1057E00090B107F10C032A462146D4E905C0E047F1
:1057F00050B100254FF0010836B1E068F06007486D
:105800000068E060054804602646E468B8F1000FCF
:1058100001D1002CE0D14046BDE8F087C000002057
:1058200070B504460025A0B2FBF7B8FC0546284633
:1058300070BD2DE9F04106460C46B6F86E00616871
:10584000884202D2B6F86E5001E0A08885B20023EB
:105850002A463046216802F0B3FB07462FB920687C
:10586000284420606068401B6060BDE8F081000053
:105870002DE9FF5F04460E46207C0A2808D1214608
:10588000204801F001FA21460220FFF7D3FB37E060
:10589000A76DD4F824800CB9002000E020680290A5
:1058A000201D08B9002000E060680390B4F818A03B
:1058B000B4F82090D4F89050D4F814B0214612488F
:1058C00001F0E2F9A06F10B1A06F02F029F9606F4A
:1058D00010B1606F02F024F921460220FFF7AAFB05
:1058E00000BF1DB16FF004015846A84700BF3EB18C
:1058F00003AB02AA41463846CDE900A902F0ABF855
:10590000BDE8FF9F00010020FC000020C16170473E
:1059100003466FF00400704770B506460220FFF79B
:10592000CBFB04467CB900F02BFE0220FFF7C4FB42
:1059300004463CB9304600F0F7FD0220FFF7BCFBFF
:10594000044600BF00BF002C39D0A0212046FAF742
:1059500050FC4020183404F8070C41F2D060A4F841
:1059600056000020A4F8580041F2D06020826082E6
:10597000002004F80E0CFF2004F80D0C4FF4067004
:105980002084062020860020A0850620E085C01FF8
:10599000E0830120608700F055FF0546E56425643B
:1059A0006563256507480068A061002020770648E8
:1059B000E0660648E067002084F88500183C204631
:1059C00070BD0000F0000020E778000800DD6D00E9
:1059D000416170472DE9F04107460D46164600BF6C
:1059E000387C18B16FF00C00BDE8F08100BF16B92B
:1059F00000F0ECFE06463048046810E0208BB04210
:105A00000CD144B1206830B12DB1286818B120689C
:105A10002968884202D16FF00A00E5E7E468002CAB
:105A2000ECD12648046810E0208BB0420CD144B180
:105A3000206830B12DB1286818B1206829688842E3
:105A400002D16FF00A00CFE7E468002CECD11C48CB
:105A5000046810E0208BB0420CD144B1206830B112
:105A60002DB1286818B120682968884202D16FF0EA
:105A70000A00B9E7E468002CECD1124804680AE097
:105A8000208BB04206D120682968884202D16FF08D
:105A90000A00A9E7E468002CF2D11DB1286808B11A
:105AA000286838603E8300BF05480068F8600448F5
:105AB000076000BF002097E7F8000020FC000020EE
:105AC000F40000200001002070B50546287C08285D
:105AD00064D2DFE800F004323D485163635A002489
:105AE00000BF34480068A84205D132480068C06849
:105AF0003049086018E02F4800682F4908600EE020
:105B00002D480068C068A84204D12B49E86809689C
:105B1000C86008E028480068C0682749086026482F
:105B200000680028ECD100BF0020E86000BF2946D3
:105B30000220FFF77FFA002533E0002429461F48A2
:105B400001F0A2F829460320FFF774FA002528E0A7
:105B5000002429461A4801F097F829460220FFF749
:105B600069FA00251DE00121284601F0E8FF0446FE
:105B70000CB90520287414E00121284601F0DFFF4C
:105B800004460CB9052028740BE00121284601F0D9
:105B9000D6FF04460CB90920287402E00024002531
:105BA00000BF00BF1DB114B9284600F059FE2046C1
:105BB00070BD0000F400002004010020F800002067
:105BC000FC0000202DE9F04105460E463046FEF768
:105BD0006FFD044654B1A08C40B1A08C283887B228
:105BE000BD4201DA284600E0384605462846BDE8B1
:105BF000F0812DE9FF4F87B005469A4600BF09980E
:105C000048B9159838B90AF0030020B96FF00900B7
:105C10000BB0BDE8F08F00BF00BF099820B908980D
:105C200010B16FF00900F3E700BFB5F86E100998E6
:105C3000814208DA95F8220040F0800085F82200C1
:105C40004FF0FF30E4E70998049008980290159807
:105C500000F0010008B1042100E00021159800F0D7
:105C6000020008B10C2000E0002001EB0009A86E42
:105C70000590B5F87080B8F1040F03DA4FF6FC70A8
:105C8000804508DD95F8220040F0800085F822006C
:105C90004FF0FF30BCE7B8F1000F01D000BF01E0CA
:105CA00000BF00BF00242746264600200390C6E020
:105CB000288FA0EB09010498814203DA288FA0EB1A
:105CC000090000E0049880B203900420FFF7F4F983
:105CD000044604B976E10020206060600FB92746D1
:105CE00002E000BF00BF34602646149800F00100B7
:105CF000F8B10398484481B200221046FFF7BEFA7B
:105D0000606000B95EE100BF00BF6068FFF7ACFBF8
:105D100040441FFA80F8089838B16168496801EB7F
:105D20000900DDE90212FAF74BFA60684068A060EA
:105D30002CE0002249461046FFF7A0FA606000B947
:105D400040E16068FFF790FB40441FFA80F8049838
:105D500000281BDD012203200399FFF78FFA06902C
:105D600028B96068FFF72DFC002060602AE108F187
:105D700001001FFA80F80699029848600298A06016
:105D800060680699FFF749FB00200690B8F1040F00
:105D900003DC4FF6FC70804500DD13E10398A08121
:105DA00014216068FFF744FC00B10BE160684068B3
:105DB0002061288BFDF789FB21690880288CFDF77D
:105DC00084FB216948800598FDF772FB21694860D2
:105DD0000020216948824FF6C070FDF776FB2169EB
:105DE000898900EA010B5046FDF76FFB4BEA000B77
:105DF0002069A0F80CB01598A07321698889FFF775
:105E000037FA00F03F01CB464FEAE97009EB90709A
:105E10008010401D41EA003080B20190FDF755FB33
:105E200021698881DDE90310401A80B2049003994A
:105E3000059808440590DDE9020108440290002F0E
:105E40003FF436AF049800283FF732AF686F08B9C7
:105E5000002605E06E6F00E0366830680028FBD150
:105E6000002E74D031698889FFF702FA00F0030030
:105E700008B1012000E00020B1890844002866D064
:105E800031698889FFF7F4F900F00300E8BB0AF0F4
:105E9000030010B1BAF1010F59D1B089B989084492
:105EA000298F884253DCB07BB97B88424FD131695E
:105EB0004868FFF7D7F9B18900EB010B39694868E9
:105EC000FFF7D0F9834542D109F1140251427868B5
:105ED000FFF7AEFB10B100BF00BF73E078684089E8
:105EE00078B9D7F804B07868006878600020CBF8FB
:105EF0000000A8F101001FFA80F85846FFF761FB87
:105F000000BF0AF0010060B100E020E000BF00BF68
:105F10000120FDF7DAFA31698989084331698881FE
:105F20000BE000BF00BF79687068FFF776FAB089B0
:105F3000B9890844B08138683060BC4202D1344627
:105F4000B089039039460420FFF774F803E00EB9D6
:105F50006F6700E037600AF0020010B90AF0010034
:105F600018B10998401C80B209900AF0010028B1CC
:105F700095F8220040F0200085F8220055F8681FAF
:105F8000099808442860E9880998081AE880A5F863
:105F900008802889683D08B100BF00BF84B103981C
:105FA00000280DDD206958B1149800F0020038B9BE
:105FB0000820FDF78AFA21698989084321698881C7
:105FC000002025E695F8220040F0800085F82200A8
:105FD00017B1384601F0A4FDB5F8700008B100BF54
:105FE00000BF4FF0FF3013E6C0F89010704700007C
:105FF00070B51C48046831E0E06FC0B100BFD4F850
:10600000840040B100232146D4F88460E26F6069C7
:10601000B047054606E0002321461846E26F01F02E
:1060200062FC054600BF0DB90020E06700BF94F890
:10603000220000F0010080B100BF94F8220040F07F
:10604000020084F82200204600F00AFC00BF94F809
:10605000220020F0030084F82200E468002CCBD159
:1060600070BD0000FC0000202DE9FC5F06468A465A
:10607000FE497068086009680888FFF7F9F8C0F3FE
:106080000320716801EB8000F9490860F74909684D
:106090000888FFF7EDF8C0F303208000C0F1000B83
:1060A00059463046FFF7C4FA10B93089142804D293
:1060B0003046FFF786FABDE8FC9F5146EB48006882
:1060C0001030FDF780FE70B94FF07040FFF7CAF84E
:1060D000E6490968096900EA010B4FF06040FFF7E3
:1060E000C1F8834503D13046FFF76BFAE3E7E04997
:1060F00009688889FFF7BCF84FEA20394FEA890020
:1061000041423046FFF794FA18B13046FFF759FA8A
:10611000D1E7D74909680888FFF7AAF8D449096880
:106120000880D34909684888FFF7A2F8D049096870
:106130004880CF4909684868FFF794F8CC49096856
:106140004860CC490860CA4909688868FFF78AF83E
:10615000C74909688860C8490860C5490968C8898D
:10616000FFF786F8C2490968C881C149096888896A
:10617000FFF77EF800F03F00C049087030890978C9
:1061800001F0030109B1012100E000210844BC49EC
:1061900008800027BB4804682CE000BF00BF00BF98
:1061A00000BF00BF00BF208CB14909680988884240
:1061B0001ED1208BAE4909684988884218D1AB4965
:1061C00060680968C968884212D1A84920680968CE
:1061D000096988420CD100BF00BF37B1E068F860A0
:1061E000A8480068E060A748046000BF00BF03E063
:1061F0002746E468002CD0D100BF002C4CD1A24827
:10620000046821E000BF00BF208C99490968098813
:10621000884218D1208B964909684988884212D152
:10622000924960680968C96888420CD18F49206822
:1062300009680969884206D1204601F031FE3046DE
:10624000FFF7BFF937E7E468002CDBD100278F4860
:1062500005681FE03DB1286828B1844928680968AD
:106260000969884214D1288B814909684988884284
:106270000ED137B1E868F86084480068E860834868
:106280000560284600F09AF93046FFF79AF912E7C0
:106290002F46ED68002DDDD1002C75D000207C4903
:1062A0000860308988817068886008464660704858
:1062B0000068086100207749086077490870E06F3E
:1062C000F0B100BFD4F8840040B100232146D4F8D7
:1062D00084C0E26F6069E047804606E00023214603
:1062E0001846E26F01F0FFFA804600BFB8F1000FD8
:1062F00002D10020E06703E03046FFF762F9DAE6FA
:1063000066480460204600F011FD804608F1050053
:10631000002817D06048007800F0080098B100BF4E
:10632000D4F8900028B16FF00501D4F8902060698E
:10633000904700BF2146534800F0A6FC21460220AA
:10634000FEF778FE71E05448007800F0100040B18C
:1063500021464C4800F098FC21460220FEF76AFED8
:1063600063E04FF00008B4F86C00002810DD00BFB7
:10637000D4F8800048B1B4F86C202146D4F88030BD
:1063800060699847804602E05DE04FF0000800BF7A
:106390004048006848B33948007800F0080038B138
:1063A0003C480068407B40F001003A490968487366
:1063B00000BFD4F8840048B100233649D4F884C023
:1063C00060690A682146E047804607E000233148BB
:1063D00021460268184601F086FA804600BFB8F1EF
:1063E000000F02D02B480068E0672B48007800F0CF
:1063F0002000A0B100BFD4F8840040B100231A46A9
:106400002146D4F884C06069E047804606E0002356
:106410001A462146184601F066FA804600BF002061
:106420001E490860204600F01BFA00201B49086046
:1064300017484068A0B316494868FFF7C2F8002023
:10644000134948603CE00A4909688889FEF710FF53
:1064500000F0040088BB0648006800880449096809
:106460004988CDE90010034800681AE014010020B3
:1064700010010020180100201C0100202001002034
:1064800022010020FC00002000010020F800002074
:106490000442002028010020240100202C010020BB
:1064A0000EE0094A12888118084803680C33026814
:1064B00010320748006801F0CEFA3046FFF781F845
:1064C00000BF00BF00BFF6E522010020140100203C
:1064D0001C0100202DE9FC4104460022142101206A
:1064E000FEF7CCFE05460DB9BDE8FC8100BF00BF3C
:1064F000A16D481EFCF7DCFF07463B4600222946FB
:10650000204600F003FB064606200021CDE90010DE
:10651000E37A221D21462846FDF7F0FD2846FFF7C5
:1065200050F800BFE0E700002DE9F04106464FF0CB
:106530007F08002700251048046813E0607CB04203
:106540000FDC607C40450CDC0C49206B0968081AA4
:10655000B84206D30949206B09680F1A254694F8FA
:106560001180E468002CE9D11DB101212846FFF714
:106570007FF9BDE8F0810000FC000020F000002061
:1065800070B5002600250B4804680BE00A49206B13
:106590000968081AB04204D30749206B09680E1A2B
:1065A0002546E468002CF1D11DB101212846FFF7F2
:1065B0005FF970BD00010020F00000207CB50546A9
:1065C0004448007800F01000B8B1434800680088E3
:1065D000414909684988CDE9001040480068404AAF
:1065E000128881183F4803680C33026810323E4815
:1065F0000068401C01F02FFA69E03648007800F08E
:106600000200002863D0687CFFF786F9044614B9BD
:106610004FF0FF307CBD33480068103008B90020CF
:1066200002E03048006800692060288B20832D48F4
:1066300000680C3008B9002002E02A480068C068F1
:106640006060254800680088208403202074234867
:106650000068401C6062606AE0621F480068C08990
:10666000A4F85C00B4F85C00A4F854001B4800686F
:10667000401E206668696061E869E061288940F22F
:1066800099110840208100BF18480068E060174851
:10669000046000BF204600F07FFA208F211DFFF725
:1066A00091FA20870120002112230A46CDE900102B
:1066B0002046FFF79EFA06462EB100212046FFF73E
:1066C000D7F83046A6E7204600F0CAF8A2E7002037
:1066D000A0E7000020010020100100201801002088
:1066E00022010020140100201C010020FC000020D9
:1066F00070B504460E4600BF207C08B1002070BD76
:1067000000BF207C012801D12046F8E70320FEF7D6
:10671000D3FC05460DB90020F1E760696861208B64
:1067200028830120287420892881288940F00200CC
:106730002881E07AE872A07AA8720CB9002000E003
:106740002068286000BF1A480068A04205D1184898
:106750000068C0681649086018E0154800681549C7
:1067600008600EE013480068C068A04204D11149D7
:10677000E0680968C86008E00E480068C0680D4914
:1067800008600C4800680028ECD100BF0020E060E1
:1067900000BF21460220FEF74DFC0748E86100BF1C
:1067A00006480068E8600548056000BF2846A6E77F
:1067B000F40000200401002011590008F800002016
:1067C00010B54020FFF7A8F810BD000000BF194821
:1067D0000088401C80B2174A1080B0F5004F02DBE1
:1067E0004FF4805010801448016806E0088B114A6D
:1067F0001288904200D1EAE7C9680029F6D10F4813
:10680000016806E0088B0B4A1288904200D1DEE74F
:10681000C9680029F6D10A48016806E0088B054AD4
:106820001288904200D1D2E7C9680029F6D1014808
:10683000008870470A010020FC00002000010020B1
:10684000F800002004480068044909680844024927
:1068500008600846006870470C010020F000002026
:106860002DE9F047044675480068A04202D1002097
:10687000BDE8F087B4F85C00B4F85210884202DA40
:10688000B4F85C0001E0B4F852008146656F94F8FA
:10689000220000F0020070B14DB129694868FEF78E
:1068A000E1FCE16C401AA9890844484503D9204617
:1068B00001F053F9DCE7A66F26B100E036683068D6
:1068C0000028FBD18EE000BF29698889FEF7D0FC43
:1068D00000BFA06F70B194F8220000F0440048B9E6
:1068E000606F48B1606F006820B9606F8089218F48
:1068F000884201DB012000E0002028B994F8220042
:1069000000F0A00000B979E028686067207C0228C8
:106910000DD01020FCF7D9FD296989890843296920
:10692000888194F8220020F0030084F82200214698
:10693000284600F085F829694868FEF793FC074669
:1069400029698889FEF794FC00F0030008B1012052
:1069500000E00020A989084407EB0008A06DB0EB17
:10696000080001D5C4F8588029698889FEF780FCA1
:1069700000F0030008B1012000E00020A9890844CC
:1069800000282BDD00202860A06F10B9A5672E46D7
:1069900027E029694868FEF765FC074631694868C1
:1069A000FEF760FC381A16D504F1780700E03F685E
:1069B000386860B1396809694868FEF753FC824657
:1069C00029694868FEF74EFCBAEB0000EFD438683E
:1069D00028603D6005E03560366802E0284601F039
:1069E0008FF8656F55B129694868FEF73BFCE16C8B
:1069F000401AA989084448457FF665AF00BFA5B194
:106A000094F89C0088B929694868FEF72BFCE16C72
:106A1000401AA9890844B4F85C10884205D90020BE
:106A2000C4F89800012084F89C0094F8220020F01B
:106A3000800084F8220000201AE700002C010020CA
:106A40002DE9FC4105460C46606AFCF731FD2969D9
:106A50008860608DFCF739FD2969C881618D606AA5
:106A60000844E062286900F11408A87B00F00100E6
:106A700030B12448FCF71CFDC8F8000008F10408F8
:106A80000CB1206860B9201DFDF712FE06460EB954
:106A9000BDE8FC81301D08B9002000E0706820606E
:106AA000B4F93600401C08B90020E086E06B38B924
:106AB00015480068E06329694868FEF7D3FB206445
:106AC000288A69688988401A87B268684089C01B2B
:106AD0006968488168680089C01B696808816968BD
:106AE000286948600020296908820621A07ACDE93A
:106AF0000001E37A221D21466868FDF7FFFA00BF16
:106B0000C6E70000B4050402F00000202DE9F047BC
:106B100005460F46164698467C68288BFCF7D5FC40
:106B20002080288CFCF7D1FC6080C4F80480686A5F
:106B3000FCF7BEFCA0604FF6C070FCF7C6FCA18954
:106B400000EA01091020FCF7C0FC49EA0009A4F89A
:106B50000C90688DFCF7B9FCE08100206082A08970
:106B6000FEF786FB00F03F01B146F01706EB907090
:106B70008010401D41EA00301FFA80FA5046FCF7B1
:106B8000A4FCA08100202082698D686A0844E86224
:106B90002046BDE8F08700002DE9F04780462B48ED
:106BA000006800F11405294909688889FEF760FB2F
:106BB0000521B1EB203F46DA244909688889FEF7B0
:106BC00057FB0521C1EB20304FF6FF7101EA80062B
:106BD000002436E015F80490B9F1000F06D0B9F1A1
:106BE000010F05D0B9F1020F21D104E0BDE8F08713
:106BF000601C84B224E0601C285C042802D1201DA3
:106C0000B04200DDF2E7E01C295CA01C285C41EAF0
:106C1000002740F2B450874200DC17B940F2B4506C
:106C200000E03846A8F83800201D84B208E0601C57
:106C3000285C00B9DAE7601C285C204484B200BFFD
:106C400000BFB442C6DB00BFD0E700001001002047
:106C500010B50446207CA8B1207C0A2812D0207CE4
:106C600001280FD0E06F20B1E06FFEF7AAFC0020F2
:106C7000E067606F00F054FFA06F00F051FF00204C
:106C80006067A06710BD000070B505460C4600BFE8
:106C90002868A04203D12868C068286017E01F490F
:106CA000286808600EE01D480068C068A04204D152
:106CB0001A49E0680968C86008E018480068C068B8
:106CC00016490860154800680028ECD100BF002074
:106CD000E06000BF2046FFF7BBFF207C0A2810D0F1
:106CE000207C01280DD094F8220000F0010040B172
:106CF00094F8220040F0020084F822002046FFF7BA
:106D0000AFFD207C012803D000BF00BF00BF00BF43
:106D10000020207400BF00BF70BD000004010020EF
:106D2000C0F88C1080F83520704700002DE9FC4138
:106D300004460027B846FC48007800F0040060B321
:106D4000207C022806D1F949A06D096888420FD13C
:106D500001270DE0F649606A0968081A08D4218DF8
:106D6000606A0844F2490968081A002800DC012713
:106D70008FB100BF00BFEF48007840F00800ED4938
:106D8000087094F8220020F0010084F822006FF0CF
:106D90000500BDE8FC810020FBE7E348007800F037
:106DA000020090B1207C02280FD0207C03280CD058
:106DB00000BF94F8220040F0020084F82200204630
:106DC000FFF74EFD00BF0020E3E7DB4800682063CB
:106DD000002084F89D002046FFF7DEFE207C801E08
:106DE00008286FD2DFE800F0049AF4F3F2F1F0EF34
:106DF000CD48007800F01000002873D0CA48007811
:106E000000F0020000286DD0A16F09694868FEF704
:106E100029FA401CC5490968884263D1B4F86E005C
:106E2000401CA4F86E00C2480068401C6062606AA2
:106E3000E062BE480068E064C0480068C089A4F809
:106E40005C00BB480068401E206604202074208F30
:106E5000211DFEF7B7FE2087208F00EB80004FF644
:106E6000FF7101EA4000A4F85400B4F85200012870
:106E700002D1208F400000E0208FA4F8520000BF14
:106E800000BFB4F87000401EA4F87000A56F286819
:106E9000A067A06F18B94FF0FF30E08603E0002034
:106EA000E08684F84A00284600F02AFE00BFD4F8A5
:106EB000880040B100222146D4F8883060699847A4
:106EC000804602E0E4E14FF0000800BF00BF94F804
:106ED000220040F0020084F822002046FFF7C0FCA8
:106EE0001BE0FFE79048007800F01000A8B193483D
:106EF00000680088914909684988CDE900108C48EC
:106F000000688F4A128881188E4803680C33026823
:106F100010328648006800F09EFDBAE18248007891
:106F200000F0100000286BD0E06C401C7F4909681D
:106F3000081A4ED47D49A06D0968081A002848DC5B
:106F40000420207400BF00BF00BFE06930B1002200
:106F50002146E36960699847804601E04FF00008E8
:106F600000BFB8F1000F06D001212046FEF780FCDB
:106F70006FF004000DE7B4F85260204600F098F975
:106F8000B4F86C0020B1B4F86C00401EA4F86C009A
:106F9000012E02D1208F400000E0208FA4F8520083
:106FA0006448007800F0200060B100BF94F822002F
:106FB00040F0020084F822002046FFF751FC00BF99
:106FC000072020742AE04FE10DE128E0C2E03DE017
:106FD00026E05A4800680088584909684988CDE980
:106FE000001053480068564A1288811855480368B3
:106FF0000C33026810324D48006800F02CFD0DE0A3
:107000004948007800F0020040B1606A401E4849DB
:107010000968884202D1204600F09FFC39E100BF98
:10702000204600F045F94348007800F0200060B1A8
:1070300000BF94F8220040F0020084F822002046AD
:10704000FFF70EFC00BF0720207422E1204600F06D
:107050002FF93848007800F0200088B332480078D3
:1070600000F0100068B33149A06D096888423FD133
:1070700000BF94F8220040F0020084F8220020466D
:10708000FFF7EEFB00BF2046FFF7E2FD00BF2E48F2
:107090000068A04205D12C480068C0682A490860F1
:1070A0001AE0294800682949086010E0274800686C
:1070B000C068A04206D12549E0680968C8600AE0B6
:1070C00024E015E021480068C068204908601F4896
:1070D00000680028EAD100BF0020E06000BF0A205D
:1070E000207400BF1A480068E0601948046019E085
:1070F00000BF94F8220040F0020084F822002046ED
:10710000FFF7AEFB00BF082020740BE006480078B4
:1071100000F0100030B10549A06D0968884201D126
:1071200006202074B5E00000200100201C01002092
:107130001801002024010020F00000201001002090
:107140002201002014010020FC0000200401002086
:1071500000010020204600F0ABF84F48007800F016
:107160002000E8B300BF94F8220040F0020084F849
:1071700022002046FFF774FB00BF2046FFF768FDA2
:1071800000BF46480068A04205D144480068C06876
:107190004249086018E041480068414908600EE033
:1071A0003F480068C068A04204D13D49E0680968D2
:1071B000C86008E03A480068C06839490860384843
:1071C00000680028ECD100BF0020E06000BF0A206A
:1071D000207400BF33480068E0603248046000E07B
:1071E00000E000BF55E0204600F062F82E4800782D
:1071F00000F01000B8B32D49A06D0968884232D163
:107200002046FFF725FD00BF24480068A04205D1B5
:1072100022480068C0682149086018E01F480068DB
:107220001F4908600EE01E480068C068A04204D1F3
:107230001B49E0680968C86008E019480068C06830
:1072400017490860164800680028ECD100BF0020EC
:10725000E06000BF0A20207400BF12480068E060B0
:107260001048046000BF14E0204600F021F80E48EA
:10727000007800F0100050B10C49A06D09688842F8
:1072800005D10548007840F010000349087000E07F
:1072900000BF00BF00207CE524010020FC0000208E
:1072A0000401002000010020200100201C0100201A
:1072B0002DE9FC5F044600200190F948007800F0B9
:1072C0001000002872D0B4F85C00616E00EB010978
:1072D000F449206E0968401A15D4F249206E0968F5
:1072E000884204D1F049606E0968401A0BD4EE4917
:1072F000606E096888421CD1EC480068C089B4F807
:107300005C10884215DDE9480068C089A4F85C007B
:10731000E44800682066E44800686066B4F85C00F1
:10732000002806DD94F89C00002802DD002084F887
:107330009C00DD49E06C0968081A002844DC002044
:10734000A4F86C00DA48008878BBB4F85C10606E72
:107350000844484532D1B4F9360000282EDBD24922
:10736000E06C0968884229D10120019094F850000E
:10737000401C94F85010884204DD94F85000401CE2
:1073800084F8500094F85000032810DDB4F852003F
:10739000218F084480B2B4F8521088420EDDB4F850
:1073A0005200218F0844A4F8520007E03AE194F813
:1073B0005000032802D1204600F0F7FA0198002877
:1073C00001D184F85000AFE0E06C401CB649096878
:1073D000081A7DD4B449A06D0968081A002877DC22
:1073E00094F8220000F0040038B114F8220F20F0C5
:1073F00004002070608E2086223C00203434A0756A
:10740000608AB4F9101000EBE10000B2A082208B7A
:10741000A5490988081A2087608F218F0844608752
:1074200000202077A0480068A06114F8240C343CA8
:10743000042824DBB4F85200B4F8541088420FDA60
:10744000B4F85200218F084480B2B4F85210884238
:1074500015DDB4F85200218F0844A4F852000EE064
:1074600034F8381F4943628B91FBF2F1114488B222
:10747000618B383C814201DAA4F8520000BF26E05B
:10748000A56FA06F0068A06700BF6868FDF7ECFFFC
:1074900000BFB4F86C0058B129698889FDF7E8FE8F
:1074A00000F0010020B1B4F86C00401EA4F86C009C
:1074B0006868FDF7D9FF34F8701F081A2080284645
:1074C00000F01EFB34F8700908B100BF00BF00E0F7
:1074D00027E0A06FC8B1A16F09694868FDF7C2FE37
:1074E0008346A16F09698889FDF7C2FE00F0030099
:1074F00008B1012000E00020A16F898908445844A8
:1075000069490968401A0028BADDA06F18B94FF020
:10751000FF30E08601E00020E086002084F834009F
:1075200002E00020A4F86C0026E0656F606F006840
:10753000606700BF6868FDF797FF00BFB4F86C0094
:1075400058B129698889FDF793FE00F0010020B148
:10755000B4F86C00401EA4F86C006868FDF784FF66
:1075600034F8701F081A2080284600F0C9FA34F851
:10757000700908B100BF00BF606FF0B1616F0969A9
:107580004868FDF76FFE8346616F09698889FDF7DA
:107590006FFE00F0030008B1012000E00020616FE1
:1075A00089890844584440490968081A05D43E4965
:1075B000A06D0968081A0028B7DDE06B90B33A495E
:1075C000206C0968401A2DD534F83C0F39490988D8
:1075D000081A0FFA80F8B4F90800A8EBE0000FFAD7
:1075E00080F82089404400B220813C3CB8F1000F73
:1075F00003DAC8F100000FFA80F83C34B4F90A004D
:10760000A8EBA0000FFA80F86089404400B26081C6
:107610006089B4F9081000EBE10000B2A0810020FD
:1076200044F83C092248008800287DDD1D48616A35
:107630000068401C081A5DD41A48616A00681C4A38
:1076400012881044401E081A002853DC1549606A4D
:107650000968471A1848466800BF00BF00BF00BF4E
:1076600040684089B84229DA00BF00BF124840682C
:107670000089C01B1FFA80FA06E070893F1AA6F83D
:1076800008A00020708136687089B842F5DB784226
:1076900001B23046FDF7CCFFC8B100BF17E00000D3
:1076A00020010020180100201C01002010010020F2
:1076B00022010020F0000020044200208349486895
:1076C000794209B2FDF7B4FF08B100BF00BF7F499E
:1076D0007068886008468089A18C7D4A1288891A62
:1076E000401A7A4988817A49606A0860774909694D
:1076F00048600FE07649606A0968081A0AD500BF39
:1077000094F8220040F0020084F822002046FFF79F
:10771000A7F800BF6E49606A0968081A7ED4218DF7
:10772000606A0844401E00E0B4E069490968081A2C
:10773000002873DC6649606A096888426FD1634932
:1077400009698889FDF794FD00F0030008B1012064
:1077500000E000205D49898908445E490880208D49
:107760000988884246DA594909698889FDF780FD08
:1077700000F00100C0B14FF6C070FBF7A6FE534900
:107780000969898900EA010B504909698889FDF76F
:107790006FFD00F03E000090FBF797FE4BEA000BF8
:1077A0004A480069A0F80CB0208D484988810969D1
:1077B0008889FDF75DFD00F0020020B14348808913
:1077C000401E42498881414A91895068FDF76FFF08
:1077D0003E4909698889FDF74BFD00F0030008B1B7
:1077E000012000E00020394989890844394908808E
:1077F00000BF00BF36480068364909880844606207
:1078000000BF00BF208D33490988401A20852046DB
:1078100000F0B2FB2D484068008901E036E031E01D
:10782000002806DD294840682B49086000202749C8
:107830004860264909698889FDF71AFD00F00100B2
:1078400028B12648007840F020002449087000BF85
:1078500094F8220000F0010068B114F8220F20F023
:1078600001002070207840F0020004F82209204630
:10787000FEF7F6FF05E094F8220040F0010084F8DE
:10788000220020E0204600F068F91CE0204600F0CD
:1078900064F918E00E49606A0968081A08D4218D55
:1078A000606A0844401E0A490968081A00280ADD6F
:1078B00000BF94F8220040F0020084F82200204625
:1078C000FEF7CEFF00BFBDE8FC9F00000442002091
:1078D000180100202201002028010020240100209E
:1078E000C0F8841070472DE9F04107460D46144654
:1078F0001E463CB12189284600F00CF82046FDF7D1
:1079000060FE05E026B92846FEF7DEF8BDE8F08106
:107910000020FBE770B504460E4600BF00BF208D77
:1079200030442085208D41F2D061884201DD084637
:107930002085204600F020FB054640F2B4508542E9
:107940000ADB00BF94F8220040F0020084F8220015
:107950002046FEF785FF00BF70BD2DE9F0410446CB
:10796000A06F08B9BDE8F081A66F3068A06704F188
:10797000740500E02D68286858B1296809694868CD
:10798000FDF770FC074631694868FDF76BFC381A53
:10799000F0D4286830602E6094F84A00401C84F8C7
:1079A0004A000020E06300BFDCE710B50446A06F8A
:1079B00098B394F8220000F0040070BB2046FFF753
:1079C000CCFFB4F85200B4F85C10884207DDB4F87C
:1079D0005C0000EBD0714910A4F8541006E0B4F834
:1079E000520000EBD0714910A4F85410B4F85400C0
:1079F000218F4900884204DA208F4004000CA4F84B
:107A000054002234608EE18A032202FB01002086AA
:107A1000207840F0040004F8220910BD70B5044637
:107A2000A06F00B970BDA56F00E02D682868002820
:107A3000FBD1606F2860A06F60670020A06794F89A
:107A40004A00401C84F84A000020E0632046FEF70C
:107A500007FF00BFE6E72DE9FC5F81460E461746AB
:107A60009846DDF830A0002214210120FDF706FC25
:107A700005460DB9BDE8FC9F00BF00BF6C685046CD
:107A8000FBF723FD20800D98FBF71FFD6080484623
:107A9000FBF70EFD60603046FBF70AFDA0604FF675
:107AA000C070FBF712FDA18900EA010B1420FBF75F
:107AB0000CFD4BEA000BA4F80CB041F2D060FBF7D0
:107AC00004FDE08100206082A089FDF7D1FB00F079
:107AD0003F0040F4A04B5846FBF7F7FCA081002084
:107AE000208206200021FF234246CDE900103946BE
:107AF0002846FCF703FB2846FDF763FD00BFB9E706
:107B000070B5044600254CB1606818B16068FDF797
:107B100058FD054621460420FDF78CFA284670BD25
:107B200070B50446002506E026682046FFF7E8FF0A
:107B30002844C5B23446002CF6D1284670BD7CB529
:107B400005460C460020012123460246CDE90010DF
:107B500001462846FEF74DF87CBD2DE9FC41044660
:107B6000002606F1140100220120FDF787FB0546DF
:107B700015B9B01EBDE8FC8194F8220020F0030086
:107B800084F82200A06DFBF793FC80464346324602
:107B900029462046FEF7BAFF07460621A07ACDE91E
:107BA0000001E37A221D21462846FCF7A7FA284661
:107BB000FDF707FD0020DDE7C0F8801070470000EA
:107BC0002DE9FC474FF0000AAF480068401CAE4961
:107BD00008600026AD48046828E100BF00BF00BF70
:107BE00000BF00BF00BF0025A846207C022806D1A8
:107BF00094F84A00062802D1681CC5B26AE094F8DD
:107C00004A000C2802D1681CC5B263E094F89C00BD
:107C100000281BDD54F8980F401C20602079216853
:107C2000983C401E9A4A105C814253D30020C4F80D
:107C3000980094F89C00072804D294F89C00401CFB
:107C400084F89C00204600F0DFF943E0B4F93600E8
:107C5000002803DBE08E401C00B2E086A06FC8B3B2
:107C6000B4F93600B4F94810884233DB207C02288E
:107C70000CD044346088B4F9001000EBE100A17925
:107C8000844A515C884000B2A080443C0020E086D9
:107C9000B4F85200B4F85C10884202DAB4F852002A
:107CA00001E0B4F85C0081464FEA6900A4F8540092
:107CB000B4F85400218F884206DA208F4FF6FF7106
:107CC00001EA4000A4F85400208FA4F85200204696
:107CD000FFF7A4FE207C062807D16B49206B0968BA
:107CE000081A282801D9681CC5B2207A00F00800BB
:107CF000B0B3207C042802D0207C072830D166490C
:107D0000D4F8940008444FF4FA71B0FBF1F05E4AE5
:107D1000216B1268511A884206D2681CC5B208F15C
:107D2000010000F0FF081BE094F89D1042F29F4212
:107D300011FB02F1D4F8940000EBC1004FF4FA718A
:107D4000B0FBF1F0504A216B1268511A884207D2F9
:107D50002046FEF7BFFB94F89D00401C84F89D0070
:107D6000207C032807D14849206B0968081A282875
:107D700001D9681CC5B2207C092807D14249206B73
:107D80000968081AF02801D9681CC5B265B32046F5
:107D9000FEF75EFF26B100BF00BFE068F06004E0C0
:107DA00000BF00BF3949E068086000BFD4F8900008
:107DB00028B16FF00401D4F890206069904700BFAB
:107DC000B8F1000F09D0208C218BCDE90010231DC4
:107DD0002246616AA06DFFF73EFEE7682146022059
:107DE000FDF728F93C4621E014F8340F401C2070C0
:107DF00020786178343C884216DB002084F8340017
:107E000000BFD4F88C0030B12146D4F88C206069D2
:107E10009047824601E04FF0000A00BFBAF1000F20
:107E200002D12046FEF71CFD2646E468002C7FF4B4
:107E3000D4AE00261948046822E000BF00BF002528
:107E40001149206B0968081AF02801D9681CC5B2CD
:107E5000A5B12046FEF7FCFE26B100BF00BFE068DA
:107E6000F06004E000BF00BF0C49E0680860E7680C
:107E700021460220FDF7DEF83C4601E02646E46894
:107E8000002CDAD1BDE8FC87F0000020FC000020C7
:107E9000A98F00089C8F0008B84C0A000001002040
:107EA0001CB504462448007800F0040008B1002006
:107EB0001CBD2148007800F0020020B31F49606A11
:107EC0000968081A27D4218D606A08441B4909688B
:107ED000081A00281FDC1A48006800881849096839
:107EE0004988CDE9001015480068164A12888118A3
:107EF000154803680C330268103214480068FFF715
:107F0000AAFD0020D4E70C48007800F0010010B171
:107F10000F48006820630B480088002809DD94F8AA
:107F2000220040F0020084F822002046FEF798FC70
:107F3000BEE70020BCE7000020010020180100205F
:107F40001001002022010020140100201C0100204B
:107F5000F000002010B5FEF74BF806480078401CF2
:107F6000C0B20449087000F0010008B1FFF728FE14
:107F700010BD00000801002010B501460B8D486AB5
:107F8000C218088F40F66834CB6AA04201DD204653
:107F900000E0088F1844101A04D4088D4885C86A78
:107FA000101A10BDCB6A486AC01A002802DD0020F2
:107FB000488503E0888D8B8CC01A48850020F0E747
:107FC0002DE9FC4104460F4615461E46207C042838
:107FD00008D0207C072805D0207C022802D0207CF5
:107FE00003280ED1002D0ADD002003462A4639461B
:107FF000CDE900602046FDF7FCFDBDE8FC810020D6
:10800000FBE76FF00700F8E72DE9FC470446A56F92
:1080100005B9656F0DB9BDE8FC8729698889FDF749
:1080200027F900F0010018B1A88908B9012000E083
:1080300000208046B8F1000F01D0142000E0152088
:108040008146002249460120FDF718F9064606B987
:10805000E1E700BF00BF286943680022314620469F
:10806000FEF754FD0746B8F1000F0ED04FF6C07072
:10807000FBF72BFAB98900EA010A1120FBF725FA70
:108080004AEA000AA7F80CA003E0A8680078716823
:10809000087506200021CDE90010E37A221D214653
:1080A0003046FCF72BF83046FDF78BFA00BFB2E7FD
:1080B00030B503460C4600251848016805E08B42A0
:1080C00002D100BF00BF0125C9680029F7D10CB952
:1080D000002000E020681860B2B94FF480520F48C9
:1080E000016808E0488A904204D1501C82B20B48D3
:1080F000016800E0C96819B147F6FF708242F1D10A
:1081000011B16FF00A0030BD5A8225B903480068EA
:10811000D860024803600020F5E70000A0000020BE
:10812000064909B9002101E00449096841600021BC
:108130008182017C21F0040101747047708F000876
:108140002DE9F34F85B0064675682888FDF790F84D
:10815000C0F30320082101EB8000318988420CDC48
:108160002888FDF785F8C0F303208000C0F1000BDC
:1081700059463046FDF75CFA18B13046FDF721FA52
:10818000A0E0D6F8049005F110000699FBF71BFE5D
:108190008046B9F80000FDF76BF80490B9F80200CA
:1081A000FDF766F8039000270020029082464748BA
:1081B000046835E000200290618A0398814216D15C
:1081C000B8F1000F02D144B1206830B120682969AC
:1081D000884202D0B8F1000F09D001200290BAF114
:1081E000000F04D1207C00F0040000B9A2460298E0
:1081F000A0B1A18A0498814210D1201D28B16068E5
:1082000018B16068E968884208D137B1E068F86061
:108210002E480068E0602D48046003E02746E468CB
:10822000002CC7D100BF04B9544624B90698406851
:108230002969884242D16FF007013046FDF7F8F90D
:1082400028B100BF00BF3046FDF7BBF93AE07CB172
:10825000A06948B10498009005F10C03324621460C
:10826000D4E906C0E0472CE03046FDF7AAF929E042
:10827000B8F1000F1ED14FF07040FCF7F3FF2969F1
:1082800000EA010B4FF06040FCF7ECFF834511D092
:108290002888FCF7EDFFC0F30320082101EB800BD9
:1082A00059463046FDF7C4F900BF00BF03213046F0
:1082B000FBF754FC3046FDF784F902E03046FDF749
:1082C00080F900BF07B0BDE8F08F0000A0000020DB
:1082D00010B50120FCF7F0FE04462CB12021204609
:1082E000F7F787FFFF20E072204610BD8161C26171
:1082F0007047000070B505460D480068A84205D1DA
:108300000B480068C0680A4908600CE00848046827
:1083100007E0E06820B1E068A84201D1E868E060C9
:10832000E468002CF5D129460120FCF783FE70BDDE
:10833000A00000202DE9F84306460F461446984653
:108340002046FCF7B5F905461DB96FF00300BDE8FE
:10835000F8834346224639463046009500F001F83E
:10836000F5E72DE9FF4F83B004460E469B46DDF846
:108370004080608A60B9628A21462046FFF798FEF5
:108380008246BAF1000F03D0504607B0BDE8F08F27
:1083900008213046FDF74CF970B100220821012078
:1083A000FCF76CFF054615B94FF0FF30EDE731469D
:1083B0002846FDF74EF800E0354600BF00BF6F6865
:1083C000608AFBF782F838805846FBF77EF87880A1
:1083D0000020F8800CB1206810B908F104090EE003
:1083E0002068D8F80410884208D0B54203D0284647
:1083F000FDF7E7F800256FF00800C6E7A1462889D9
:10840000FBF763F8B8801121A07A8DE80301E37AC5
:1084100049462846059AFBF78BFE8246B54203D0B3
:108420002846FDF7CEF800255046AEE72DE9F05F6F
:1084300007460D4690469A4600BF00BF9DB128688A
:1084400088B139462846FBF7BEFC60B94FF0704052
:10845000FCF708FF296800EA01094FF06040FCF7CB
:1084600001FF814503D16FF00900BDE8F09F51463F
:108470002846FAF7E7FE0446002C01DA2046F4E726
:10848000022004EB8401234A02EB8101887304EB90
:108490008400114601EB8000076106260AE0701E89
:1084A000C6B218F8061004EB84001A4A02EB8000EA
:1084B00008308155002EF2DC002004EB8401154ABF
:1084C00002EB8101C8731CE004EB8400114951F8F0
:1084D000209004EB84010F4AD9F8000042F82100F3
:1084E000D9F804B049460620FCF7A4FD434607F13D
:1084F000270259463846FAF7CFFD5846FDF761F88E
:1085000000BF04EB8400034951F820000028DBD1B0
:1085100000BFAAE71842002070B504460D46A0B27D
:108520002946F8F759FE012070BD00002F696E64DE
:1085300065782E68746D6C00485454502F312E307D
:1085400020323030204F4B0D0A5365727665723AF7
:10855000207549502F302E392028687474703A2FB6
:108560002F64756E6B656C732E636F6D2F61646124
:108570006D2F7569702F290D0A436F6E74656E74C7
:108580002D747970653A20746578742F68746D6CF9
:108590000D0A0D0A3C21444F43545950452048547C
:1085A0004D4C205055424C494320222D2F2F5733FC
:1085B000432F4454442048544D4C20342E302054F2
:1085C00072616E736974696F6E616C2F2F454E22F4
:1085D0003E0D0A3C68746D6C3E0D0A3C4D4554419D
:1085E00020485454502D4551554956203D20225085
:1085F0007261676D612220434F4E54454E543D22B7
:108600006E6F2D6361636865223E0D0A3C74697468
:108610006C653E2053544D333246347837204941FF
:1086200050207573696E672048545450203C2F7455
:1086300069746C653E0D0A3C626F64793E0D0A3CBC
:1086400068323E4C6F67696E3C2F68323E0D0A3CC3
:10865000464F524D204D4554484F443D504F535482
:1086600020414354494F4E3D222F636865636B6C34
:108670006F67696E2E636769223E0D0A3C703E0D7E
:108680000A3C666F6E742073697A653D2232223E21
:10869000203C7374726F6E673E20456E7465722065
:1086A0007573657220494420616E64207061737334
:1086B000776F72643A203C2F7374726F6E673E3C22
:1086C0002F666F6E743E0D0A3C42523E0D0A3C739B
:1086D00074726F6E673E20557365722049443C2F5B
:1086E0007374726F6E673E203C696E70757420748F
:1086F0007970653D2274657874222073697A653DCE
:1087000022323022206E616D653D22757365726E76
:10871000616D65223E0D0A3C7374726F6E673E2078
:1087200050617373776F7264203C2F7374726F6E35
:10873000673E20203C696E70757420747970653DC9
:108740002270617373776F7264222073697A653D5A
:1087500022323022206E616D653D22706173737725
:108760006F7264223E0D0A3C42523E0D0A3C696E15
:1087700070757420747970653D227375626D6974CB
:1087800022206E616D653D226C6F67696E222076D6
:10879000616C75653D224C6F67696E223E0D0A3C27
:1087A0002F703E0D0A0D0A3C2F666F726D3E0D0A4A
:1087B0003C2F626F64793E0D0A3C2F68746D6C3EED
:1087C0000D0A2F72657365742E68746D6C004854C1
:1087D00054502F312E3020323030204F4B0D0A5361
:1087E00065727665723A207549502F302E392028EF
:1087F000687474703A2F2F64756E6B656C732E639A
:108800006F6D2F6164616D2F7569702F290D0A439B
:108810006F6E74656E742D747970653A2074657826
:10882000742F68746D6C0D0A0D0A3C21444F43543B
:108830005950452048544D4C205055424C494320F6
:10884000222D2F2F5733432F2F4454442048544D6B
:108850004C20342E3031205472616E736974696F0C
:108860006E616C2F2F454E223E0D0A3C68746D6C74
:108870003E20202020200D0A20203C686561643EB7
:10888000202020202020200D0A202020203C6D6563
:10889000746120687474702D65717569763D22630A
:1088A0006F6E74656E742D747970652220636F6EBF
:1088B00074656E743D22746578742F68746D6C3BBA
:1088C00020636861727365743D77696E646F777356
:1088D0002D31323530223E202020202020200D0A4C
:1088E000202020203C7469746C653E53544D333213
:1088F00020494150207573696E67204854545020B8
:10890000202020200D0A202020203C2F7469746C28
:10891000653E20202020200D0A20203C2F68656124
:10892000643E20202020200D0A20203C626F6479C4
:108930003E20204D435520526573657420446F6E70
:108940006520212020202020200D0A20203C2F629D
:108950006F64793E0D0A3C2F68746D6C3E2F757004
:108960006C6F61642E68746D6C00485454502F31E4
:108970002E3020323030204F4B0D0A536572766511
:10898000723A207549502F302E392028687474703F
:108990003A2F2F64756E6B656C732E636F6D2F614C
:1089A00064616D2F7569702F290D0A436F6E7465B0
:1089B0006E742D747970653A20746578742F6874BC
:1089C0006D6C0D0A0D0A3C21444F4354595045200B
:1089D00048544D4C205055424C494320222D2F2FB6
:1089E0005733432F2F4454442048544D4C20342EA9
:1089F0003031205472616E736974696F6E616C2FCF
:108A00002F454E223E0D0A3C68746D6C3E0D0A20C7
:108A1000203C686561643E0D0A20203C6D657461F0
:108A200020687474702D65717569763D22636F6E70
:108A300074656E742D747970652220636F6E746531
:108A40006E743D22746578742F68746D6C3B20637E
:108A50006861727365743D77696E646F77732D31E9
:108A6000323530223E0D0A20203C7469746C653E1C
:108A700053544D3332463478372049415020757372
:108A8000696E6720485454503C2F7469746C653E7D
:108A90000D0A20203C2F686561643E0D0A20203CB1
:108AA000626F64793E0D0A202020203C666F726D53
:108AB00020616374696F6E203D222F75706C6F6149
:108AC000642E6367692220656E63747970653D2248
:108AD0006D756C7469706172742F666F726D2D6440
:108AE00061746122206D6574686F643D22706F73DC
:108AF00074223E0D0A20203C703E506C6561736507
:108B0000207370656369667920612062696E6172A5
:108B1000792066696C6520746F2075706C6F616474
:108B200020696E746F2053544D33324634783720A9
:108B3000666C6173683A0D0A202020203C62723E08
:108B40000D0A202020203C696E70757420747970A5
:108B5000653D2266696C6522206E616D653D22640B
:108B600061746166696C65222073697A653D22349F
:108B700030223E0D0A20203C2F703E0D0A20203C62
:108B80006469763E0D0A202020203C696E70757461
:108B900020747970653D227375626D697422207648
:108BA000616C75653D2255706C6F6164223E0D0AE3
:108BB00020203C2F6469763E0D0A3C2F666F726D53
:108BC0003E0D0A20203C2F626F64793E0D0A3C2F37
:108BD00068746D6C3E0D0A2F75706C6F6164646F04
:108BE0006E652E68746D6C00485454502F312E30D1
:108BF00020323030204F4B0D0A5365727665723A41
:108C0000207549502F302E392028687474703A2FFF
:108C10002F64756E6B656C732E636F6D2F6164616D
:108C20006D2F7569702F290D0A436F6E74656E7410
:108C30002D747970653A20746578742F68746D6C42
:108C40000D0A0D0A3C21444F4354595045204854C5
:108C50004D4C205055424C494320222D2F2F573345
:108C6000432F2F4454442048544D4C20342E30314F
:108C7000205472616E736974696F6E616C2F2F4539
:108C80004E223E0D0A3C68746D6C3E202020202050
:108C90000D0A20203C686561643E202020202020B1
:108CA000200D0A202020203C6D65746120687474BA
:108CB000702D65717569763D22636F6E74656E7493
:108CC0002D747970652220636F6E74656E743D2219
:108CD000746578742F68746D6C3B2063686172737F
:108CE00065743D77696E646F77732D31323530224C
:108CF0003E202020202020200D0A202020203C740F
:108D000069746C653E53544D33322049415020758F
:108D100073696E67204854545020202020200D0A8B
:108D2000202020203C2F7469746C653E2020202078
:108D3000200D0A20203C2F686561643E2020202001
:108D4000200D0A20203C626F64793E202046696C29
:108D5000652055706C6F616420446F6E6521202022
:108D6000202020200D0A202020203C62723E20205E
:108D70002020202020200D0A202020203C666F7219
:108D80006D20616374696F6E203D222F726573657B
:108D9000746D63752E6367692220656E63747970E4
:108DA000653D22746578742F706C61696E22206D48
:108DB0006574686F643D22676574223E2020202020
:108DC0000D0A2020202020203C696E7075742074CC
:108DD0007970653D227375626D6974222076616CCD
:108DE00075653D225265736574204D4355223E0DD5
:108DF0000A202020203C2F666F726D3E20200D0A35
:108E000020203C2F626F64793E0D0A3C2F68746D00
:108E10006C3E0000000000002C850008388500082A
:108E20008A020000148E0008C2870008CE8700085E
:108E30008F010000248E00085D8900086A890008FF
:108E40006D020000348E0008D78B0008E88B000804
:108E50002A0200000D0A2D2D6F637465742D737442
:108E60007265616D0D00436F6E74656E742D4C6597
:108E70006E6774683A2000003139322E3136382E50
:108E8000312E3132300000003235352E3235352E5C
:108E90003235352E300000003139322E3136382E41
:108EA000312E310000000000382E382E382E3800C8
:108EB0000000000000000000382E382E342E340050
:108EC00000000000000000006B6B6D2D7365727672
:108ED00065722D746573742E312D6F66642E7275F4
:108EE0000000000000000000000000000000000082
:108EF0000000000000000000000000000000000072
:108F00000000000000000000000000000000000061
:108F10000000000000000000000000000000000051
:108F20000000000000000000000000000000000041
:108F30000000000000000000000000000000000031
:108F4000000000000000000037382D43352D453566
:108F50002D45462D30342D30370000000000000034
:108F6000611E60EA3075307501000100911F00003C
:108F700000000000FFFFFFFF1C002000A0002000F9
:108F80001400200008001000000604000500020084
:108F90000200020005001E00020006000102030498
:108FA00005060707070707070703060C1830607850
:108FB000FFFFFFFFFFFF00000000000046494E5F7B
:108FC000574149545F31000046494E5F574149546B
:108FD0005F32000045535441424C495348454400D8
:108FE000434C4F534544000053594E5F524356443F
:108FF00000000000434C4F53494E47004C4153542E
:109000005F41434B000000004C495354454E000063
:1090100054494D455F57414954000000434C4F535C
:10902000455F57414954000053594E5F53454E54D4
:109030000000000054900008000000205C010000C7
:10904000C40200089C9000085C0100205C820000C3
:10905000802700088580F0FA020009B001020304AD
:109060000607080913E08F140808901B0828041A43
:10907000E80C1AD4041ABC041AC8041A1C141AF4F2
:10908000081AFC041A100C011B0427106E192D017C
:0C90900002030404051B06070809000089
:040000050800018965
:020000040801F1
:1000000020F8001069020108530201085502010896
:10001000590201085D0201086102010800000000A8
:100020000000000000000000000000009D01010829
:100030006502010800000000F1010108E9AA0108B9
:100040008302010883020108830201088302010878
:100050008302010883020108830201088302010868
:100060008302010883020108830201088302010858
:100070008302010883020108830201088302010848
:100080008302010883020108830201088302010838
:100090008302010883020108830201088302010828
:1000A0008302010883020108830201088302010818
:1000B0004D70010879700108830201082385010849
:1000C0004B860108830201088302010883020108AC
:1000D00083020108837F010883020108830201086B
:1000E00083020108830201088302010883020108D8
:1000F00083020108830201088302010883020108C8
:1001000083020108830201088302010883020108B7
:1001100083020108830201088302010883020108A7
:100120008302010883020108830201088302010897
:100130008302010845E501088302010883020108E2
:100140008302010883020108830201088302010877
:100150008302010883020108830201088302010867
:100160008302010883020108830201088302010857
:100170008302010883020108830201088302010847
:100180008302010883020108DFF80CD01DF040FF54
:1001900000480047D54E010820F800102A4B196886
:1001A0000868B0E8F04F80F30988BFF36F8F4FF015
:1001B000000080F3118870470000000006480068C6
:1001C000006880F3088862B661B6BFF34F8FBFF353
:1001D0006F8F00DF00BF00BF08ED00E0DFF80C000C
:1001E000016841F470010160704700BF88ED00E0D4
:1001F000EFF30980BFF36F8F134B1A681EF0100FD7
:1002000008BF20ED108A20E9F04F106008B44FF0CD
:10021000BF0080F31188BFF34F8FBFF36F8F0BF0D8
:10022000D7FB4FF0000080F3118808BC19680868FC
:10023000B0E8F04F1EF0100F08BFB0EC108A80F34A
:100240000988BFF36F8F7047FC050020EFF305802E
:100250007047704700BFFEE700BFFEE700BFFEE744
:1002600000BFFEE770470000064880470648004789
:10027000FEE7FEE7FEE7FEE7FEE7FEE7FEE7FEE756
:10028000FEE7FEE765030108890101080CB50020BF
:10029000019000907448006840F480307249086012
:1002A00000BF7148006800F4003000900198401CC5
:1002B0000190009818B90198B0F5A06FF1D16A4883
:1002C000006800F4003010B10120009001E000202F
:1002D00000900098012844D163484030006840F005
:1002E00080506149403108606048006840F48040B7
:1002F0005E4908605C48083000685B490831086066
:100300000846006808600846006840F480500860AD
:100310005748091F0860081F006840F08070091FD7
:10032000086000BF5048006800F000700028F9D055
:1003300040F201604F4908604B480830006820F0E7
:1003400003004949083108600846006840F002008F
:10035000086000BF44480830006800F00C0008281E
:10036000F8D10CBD10B54448006840F47000424913
:1003700008603D48006840F001003B4908600020EB
:10038000394908310860384800683C490840364916
:1003900008603B48091D0860081F006820F48020A1
:1003A000091F0860002030490C310860FFF76EFF1C
:1003B000344831498039086010BD70B500200022F2
:1003C000022300240221284D08352D6805F00C0079
:1003D00020B1042806D0082834D107E02A4D2B4E3E
:1003E000356033E02A4D294E35602FE01E4D2D1D1E
:1003F0002D68C5F380541C4D2D1D2D6805F03F015F
:1004000054B1234DB5FBF1F5174E361D3668C6F3D2
:10041000881605FB06F209E01B4DB5FBF1F5124EFF
:10042000361D3668C6F3881605FB06F20E4D2D1DE7
:100430002D68C5F301456D1C6B00B2FBF3F5134E3F
:10044000356003E0104D114E356000BF00BF064D12
:1004500008352D68C5F303150E4E705D0B4D2D68E4
:10046000C5400A4E356070BD003802400070004043
:1004700008324306003C024088ED00E0FFFFF6FE34
:1004800010300024000001080024F40000000010D7
:1004900000127A000400001070B5F94CF948007998
:1004A000401E00EB401000EB4000F74901EB001547
:1004B0004FF4C662294620461DF092F82078FF28A6
:1004C0000AD14FF4C66120461DF0B2F8EF4800781B
:1004D00020F00200ED490870012070BD2DE9F041C7
:1004E0000824E74D0026E7480079401E00EB401045
:1004F00000EB4000E44901EB001708F0D3FD0AE0EF
:1005000035F8021B384608F0EBFE0446082C00D0F4
:1005100004E0B61CBF1CB6F5C66FF1D300BF08F0EF
:10052000CEFD2046BDE8F08110B5082408F0BAFDE4
:100530000121382008F002FE044608F0C0FD2046E4
:1005400010BD10B5044604F10B0020F00700D0499F
:1005500009680844CE49086020461EF057FC10BDCB
:1005600070B50446254655F8040CC9490968081AAF
:10057000C749086020461EF021FC70BDF0B5024658
:10058000147804F5FA6153789578022B01DC0C336A
:10059000491E642691FBF6F6CF1701EB9777BF1043
:1005A00040F26D1C0CFB0177BE1B4FF4C87791FB2A
:1005B000F7F7F0195C1C04EB4404052694FBF6F4F1
:1005C0001E2606FB03442C442044B24C001BB24CB4
:1005D0006043D4784FF4616614FB06F416793C2727
:1005E00017FB06442044F0BD10B50121402009F05E
:1005F0004AFC012009F07EFD00BF012009F09CFDAE
:100600000028FAD009F085FD0446002009F072FDAB
:100610000021402009F037FC204610BD30B50B46C4
:10062000014637E01C787F2C0BDD1C78B02C08DAF3
:10063000D0240C70491C1C7810340C705B1C491CB5
:1006400028E01C78DF2C0BDD1C78F02C08DAD12494
:100650000C70491C1C78603C0C705B1C491C19E038
:100660001C78F02C07D1D0240C70491C81240C700C
:100670005B1C491C0EE01C78F12C06D1D1240C70B7
:10068000491C91240C705B1C491C1C780C70491C83
:100690005B1C00BF1400A2F10102C3D10C7030BD7D
:1006A0004FF4FA7400252BE00AF001FA7B48008829
:1006B000844202DD0CF05CF8054655B10CF058F8A8
:1006C00005F6B831884204D94FF4FA7073490880AE
:1006D0000025724804880AF0F9F97148408B40F00F
:1006E00010006F4948835CB120460BF071FF6C48E5
:1006F000008B40F010006A49088320460BF068FF29
:10070000D2E74FF4FA7400BF23E00AF0D0F965484D
:10071000007810B90020644908706348007808B96F
:10072000002401E0614804880AF0D0F95C48408B5D
:1007300040F020005A4948835CB120460BF048FF46
:100740005748008B40F020005549088320460BF0A5
:100750003FFFDAE70BE00821514808F096FF30B977
:100760004FF47A7006F09FFC64200BF031FFF2E743
:100770000146092903DD01F13700C0B2704701F1DC
:100780003000C0B2FAE700B503460A461809FFF781
:10079000EFFF107003F00F00FFF7EAFF507000202A
:1007A0009070104600BD2DE9F04786B00746884698
:1007B00015461E463E480BF0C9FF0BF018FF3DA141
:1007C0003D481EF03DF80BF01AFF00240EE00BF040
:1007D0000EFF385D01A9FFF7D6FF82465146364825
:1007E0001EF02EF80BF00BFF601C84B24445EEDBCC
:1007F0000AF05DF94FF0010900203080C7E0434660
:100800003A4604212D4807F0AFFD401C78B1284638
:1008100005F01AFC3080308840B90BF0E8FE28A1C2
:1008200025481EF00DF80BF0EAFE08E0B0E00BF0F2
:10083000DEFE2BA120481EF003F80BF0E0FE30484E
:100840000078A8B10BF0D3FE2E491B481DF0F8FF2D
:100850000BF0D5FE0AF03AF942F210700BF0B8FE38
:100860000AF025F926480078401E254908708EE0D8
:1008700000200A4908800AF029F90BF0B8FE43E08D
:100880008C99001055000020000006085C990010AB
:1008900084000020C9FA0A0080510100880000206D
:1008A0000000024045000020460000208A00002091
:1008B0000C0000200D2D3E00EC000010005C0040FC
:1008C0000D0A4552524F523A20464E2072656365DA
:1008D000697665206572726F722E2E2E0D0A0000E9
:1008E0000D0A4552524F523A20464E207472616EA4
:1008F000736D6974206572726F722E2E2E0D0A0050
:100900001F000020F4B10308F2A1FB481DF098FF7E
:100910000BF075FE0021F94808F0AFFFF74808F02A
:1009200007FF0121F54809F003F80021F34808F01A
:10093000FFFF0020ADF80C004BF6FF70ADF80E0085
:100940004FF48060ADF812000001ADF81400EC48DF
:1009500002900121E94808F0BCFF02A9E74808F02D
:1009600010FF0BF044FEE7A1E3481DF069FF0BF018
:1009700046FE06F091FE0121E04808F07EFF0420CB
:10098000EB4908700AF093F84FF0000900BF36E712
:1009900000BF0020E6490870B9F1000F04D14FF400
:1009A000FA70E44908800BE0F878302808D1E8783C
:1009B00000F07F0020B91E22291DDF481CF010FE28
:1009C0000AF084F80BF013FEDCA1CB481DF038FFD1
:1009D0000BF015FE00240EE00BF009FE285D01A9C6
:1009E000FFF7D1FE82465146C3481DF029FF0BF0A8
:1009F00006FE601C84B23088A042EDDCD0480BF0CB
:100A0000AEFE484606B0BDE8F0870EB50025A84604
:100A10004FF48069AA46002002904F46F0E3C9488F
:100A2000007800286FD0C848007805286CD2DFE82D
:100A300010F00500E8005E02DA02A504C349B1F82F
:100A4000EA000BF0C5FD0BF0D2FDC1A1AA481DF0D4
:100A5000F7FE0BF0D4FD0BF0CAFDC7A1A6481DF0B0
:100A6000EFFE0BF0CCFDCB4B00221146302005F001
:100A7000C1FAC9490880C94BC94A08460188C54816
:100A8000FFF791FEAC480078C0F34000002840D04A
:100A9000C4480088FF283FD1BE4B002211463220B7
:100AA00005F0A8FABC490880BC4BBD4A084601883D
:100AB000B848FFF778FEBA48047ABB480470B920FA
:100AC000B9494870042088700320B8490870B14BB8
:100AD00008460278B449442005F08CFAAE490880F3
:100AE000AE4BAF4A08460188AA48FFF75CFEAB4808
:100AF0000188AB4805F0C6FA8246BAF1000F04D16E
:100B0000A748007A02E0ADE36CE20020A549088026
:100B100002E0FF20A3490880A2480088FF2800D1F6
:100B200060E20BF064FD9F480288A1A172481DF0AD
:100B300087FE0BF064FD0298D0B9964B0022114657
:100B4000312005F057FA94490880944B944A08469E
:100B500001889048FFF727FE002405E09049201DFA
:100B6000085C9D490855641C102CF7DB012002909D
:100B700005F03AFA00208C49087001208B49087072
:100B8000844B084602788849212005F033FA8249CF
:100B90000880824B824A084601887E48FFF703FEA0
:100BA0007C4B00221146242005F024FA7A49088063
:100BB0007A4B7B4A084601887648FFF7F4FD00B976
:100BC000FAE376480188764805F05CFA8246BAF185
:100BD000000F03D101205C49087010E00BF007FD05
:100BE0006F48C2787DA144481DF02AFE0BF007FD36
:100BF00064200BF0EDFC00205349087000BF00BFDB
:100C0000CCE3644B00221146202005F0F3F9624941
:100C10000880624B624A084601885E48FFF7C3FDC0
:100C20005E4801885E4805F02DFA10F1240F4FD080
:100C300010F1230F3DD000284BD109F038FF1022CE
:100C40005749091D73481CF0CBFC09F03FFF54487D
:100C500005F065FAA0B1524805F061FA1FFA80FB71
:100C60000BF0C5FC5A466CA123481DF0E9FD0BF0C2
:100C7000C6FC02203449087064200BF0A9FC17E080
:100C800009F015FF4FF4FA706E4908802949088071
:100C900009F01CFF0BF0ABFC6BA117481DF0D0FD59
:100CA0000BF0ADFC00202849087064200BF090FC8C
:100CB0001BE10BF09CFC6FA10F481DF0C1FD0BF078
:100CC0009EFC00202049087064200BF081FC0CE1A0
:100CD000EAE0F8E00D0A4552524F523A20493243B9
:100CE00020736F6674776172652052657365742E28
:100CF0002E2E0D0A00000000EC000010005C0040E9
:100D0000A08601000D0A4552524F523A20464E200D
:100D1000686173206E6F7420726573706F6E736597
:100D200064212052657365742E2E2E0D0A0000007A
:100D30001F000020880000205C9900100D3C2D0051
:100D40000C000020340000208C000020C89F001000
:100D50000D0A4D4553534147453A2053746172740F
:100D6000206F6620776F726B696E67207769746891
:100D700020464E0D0A0000000D0A494E464F3A200B
:100D800052656164696E6720464E205374617475C4
:100D9000730D0A00F8000010220000202600002039
:100DA000E60800108E000020FE0400102400002041
:100DB0000D0A4D4553534147453A20464644207657
:100DC000657273696F6E206465746563742020308A
:100DD0007825580D0A000000EC0C00100D0A455251
:100DE000524F523A20436F6465206F6620726573DC
:100DF000706F6E73652066726F6D20464E2069734A
:100E0000206E6F6E206E756C6C3A20307825580D10
:100E10000A0000007C9900100D0A4D4553534147CC
:100E2000453A20464E206861732025642066696C2F
:100E3000657320746F207472616E736D69743A20EB
:100E40000D0A00008A0000200D0A4D45535341470A
:100E5000453A20464E20686173206E6F2066696CAB
:100E6000657320746F207472616E736D69742120D4
:100E70000D0A00000D0A4552524F523A2052657336
:100E8000706F6E73652066726F6D20464E20646FC2
:100E9000206E6F7420737461727420776974682097
:100EA00030783034210D0A000BF0A1FBEEA1FD4893
:100EB0001DF0C6FC0BF0A3FB0020FB49087064206A
:100EC0000BF086FB11E00BF092FBF848C278AFF212
:100ED000F401F4481DF0B4FC0BF091FB0020F24942
:100EE000087064200BF074FB00BF00BF56E209F0ED
:100EF000DEFDEF48067809F0E9FD002E38D0ED4917
:100F0000B1F8EC0005F012F9002831D10120EA49CE
:100F10000870EA490870EA4B08460278E649212041
:100F200005F068F8E7490880E74BE04A0846018881
:100F3000E348FFF738FCE4480188DC4805F0A2F8F4
:100F400018B90320D849087011E00BF050FBD748BE
:100F5000C278AFF27811D3481DF072FC0BF04FFB52
:100F60000020D149087064200BF032FB00BF39E04B
:100F700009F09DFD0020D549088009F0A7FD00205B
:100F8000CD4908700120CD490870CD4B0846027844
:100F9000C949212005F02EF8CA490880CA4BC34A26
:100FA00008460188C648FFF7FEFBC7480188BF48CE
:100FB00005F068F818B90020BB49087011E00BF083
:100FC00016FBBA48C278AFF2EC11B6481DF038FCF7
:100FD0000BF015FB0020B449087064200BF0F8FA00
:100FE00000BF00BFDAE1002609F061FD6420B749C7
:100FF000088009F06BFD64200BF0EAFA1BE105F0B4
:10100000E5F805464FF00008002D75DD2A20B049AF
:10101000087008204870412088700A20C87081201C
:101020000871A220487101208871AA48008868B11F
:1010300001280CD0022804D0032806D11020C87142
:1010400009E00520A249C87105E000BF00BF0020EB
:101050009F49C87100BF00BF0BF0C9FA9C48C27914
:101060009DA190481DF0ECFB0BF0C9FA002406E0AE
:10107000A448015D964A04F108001154641C102C28
:10108000F6DB93490D76280A4876142088760020EE
:10109000C876087748771E209B4908804D4501DDBA
:1010A000484600E0284687B23AE03A4641467F4843
:1010B00005F03AFA84490880084601887B4804F024
:1010C000E1FF0646CEB900240BE07849201D095CFB
:1010D0008D4802880088401C8B4B18807C488154C6
:1010E000641CBC42F1DBED1B08EB07001FFA80F823
:1010F000BD4215DAAFB213E08AE0714B002211460F
:10110000242004F077FF6F4908806F4B674A084638
:1011100001886B48FFF747FB00206349087001E036
:10112000002DC2DC00BF06B18DE0654B00221146E8
:10113000252004F05FFF63490880634B5B4A084643
:1011400001885F48FFF72FFB04F009FF064636B120
:1011500009F0ADFC6D490E7009F0B8FC73E00BF0BE
:1011600046FA6BA14F481DF06BFB0BF048FA0024C8
:101170000EE00BF03CFA5649085D01A9FFF703FBAE
:101180000146009047481DF05BFB0BF038FA641CE9
:101190005D4800888442ECDB01225B4801884C48B2
:1011A00005F03EFA064616BB05F0DDFA06467EB9A6
:1011B00009F07DFC00205549087009F087FC0BF010
:1011C00016FA57A137481DF03BFB0BF018FA32E036
:1011D00009F06DFC4D490E7009F078FC0BF007FA30
:1011E00055A130481DF02CFB0BF009FA2BE009F05B
:1011F0005EFC46490E7009F069FC0BF0F8F900E05E
:10120000DAE054A127481DF01BFB0BF0F8F91AE0B7
:1012100015F1110F06D015F1080F07D10020224952
:10122000087007E000202049087003E000201E49F4
:10123000087000BF00BF5FEA0B00ABF101011FFAAD
:1012400081FB7FF4DCAE00BF09F031FC4FF4FA7093
:101250001E4908804849088009F038FC00201249DE
:1012600008709BE09BE000000D0A4552524F523A35
:1012700020526573706F6E73652066726F6D2046C5
:101280004E20697320696E76616C696420647565AF
:1012900020746F20435243206D69736D61746368DD
:1012A000210D0A00EC0000108C000020E608001060
:1012B00045000020C89F0010FE04001024000020FC
:1012C000F800001022000020260000208A000020E4
:1012D0003D0D00108E0000200D0A4D45535341472F
:1012E000453A204646442076657273696F6E2069E0
:1012F0006E206865616465722020307825580D0A7B
:1013000000000000EC0C0010280000209E000020CF
:101310000D546F207365727665722D3E00000000DB
:101320000D0A4D4553534147453A2052656365695F
:101330007665206F6B0D0A000D0A4D4553534147EA
:10134000453A2052656365697665206661696C641B
:101350000D0A00000D0A4D4553534147453A2053AD
:10136000656E6420746F20736572766572206661A5
:10137000696C640D0A0000008800002005F0F3F994
:1013800040B90BF034F9AFF26801F8481DF058FA93
:101390000BF035F90020F649087000BF0BE00BF0A8
:1013A00026F9F449F1481DF04BFA0BF028F941F207
:1013B00088300BF00DF900BFFFF731BB00B50246D6
:1013C0000B461009FFF7D4F9187002F00F00FFF771
:1013D000CFF9587000BD0146302905DB392903DCFF
:1013E000A1F13000C0B27047612905DB662903DC3A
:1013F000A1F15700C0B2F6E7412905DB462903DC1D
:10140000A1F13700C0B2EEE71020ECE710B50246BC
:101410001078FFF7E0FF04465078FFF7DCFF034643
:1014200003EB0410C0B210BD10B5D348006810B172
:10143000D1481AF0EFFED0481AF0D4FE10BD37B5EF
:101440000C46BDF8080000B93EBD0222CB48018819
:10145000684605F06DFEC9480088801CC7490880B1
:1014600002220846018802A805F062FEC3480088EF
:10147000801CC2490880BDF8082008460188204623
:1014800005F056FEBD480088BDF808100844BB4969
:10149000088000BFD8E73EB504461022B84940F2A4
:1014A0001140FFF7CCFF0422B54910314FF48260A0
:1014B000FFF7C5FF21208DF8000004208DF8010002
:1014C000B048D0F80600000E8DF80200AD48D0F804
:1014D0000600000C8DF80300AA48C088000A8DF8A9
:1014E0000400A84880798DF805000622694640F27C
:1014F0003540FFF7A4FF0C22A34940F2FA30FFF772
:101500009EFF1422A049123140F20D40FFF797FFD1
:101510009B48401FFFF732F80290042202A94FF4C3
:101520007D70FFF78CFF04F0010040B19548008802
:101530000290042202A940F20E40FFF780FF04F05F
:10154000020030B104228F490A3140F21240FFF705
:1015500076FF04F0040030B101228A49103140F2D4
:101560001E40FFF76CFF04F00800B0B187484088C8
:101570000290042202A940F24940FFF760FF0422D2
:101580008249091D40F25C40FFF759FF05227F495F
:10159000083140F24A40FFF752FF3EBD2DED048B6B
:1015A0008EB04FF0000B002700200A900990804673
:1015B00003F0A1B9BBF1000F0CD0BBF1020F5FD05B
:1015C000BBF1030F01F03382BBF1040F43F08C81B8
:1015D00001F004BA6E48006800284FD000216D4821
:1015E00008F04BF940F206416B481CF021F86B48BB
:1015F00001886B4804F06DFD0746002064490860CF
:1016000017F1240F0BD017F1230F11D10AF0EFFFC0
:1016100064A156481DF014F90AF0F1FF2DE00AF01C
:10162000E6FF6FA151481DF00BF90AF0E8FF24E036
:10163000EA2F08D00AF0DBFF3A4674A14B481DF0B0
:10164000FFF80AF0DCFFE02F0CDBEA2F07D00AF0EE
:10165000CEFF7DA145481DF0F3F80AF0D0FF4FF012
:10166000020B09E00AF0C3FF83A140481DF0E8F82F
:101670000AF0C5FF4FF0030B00BF00BF03F037B9FE
:10168000A7F1E000202881F08B81DFE810F0200036
:101690001501640187019D01DF01FC01560355021C
:1016A0007A02AE02D70200038909890989099103E8
:1016B000B803DE033B04A004630528065E063F076B
:1016C0009F07EB0749089208D2083409F808344804
:1016D00000793349497900EB012080B20A90BDF8C6
:1016E000280007F0FEF870480078704908706E48CE
:1016F0000088001248706C48807888706A49486891
:101700001BF0D5FF0C900C9888B100200D900AE0DA
:10171000654840680D99415C644A0D98C01C11549D
:101720000D98401C0D90DDE90C108842F0DB002183
:101730005E4A0C98C01C11540C98001D5C4908802E
:10174000154B084602885949002004F053FC5949BA
:10175000088001210F4808F090F801210D4808F099
:10176000B8F84FF0000B01F036B90000EC000010A3
:101770008C00002038B20308408A00105C00002072
:10178000669900103A9900108E9A001080F00208B5
:101790004400001000540040AECA00104000001089
:1017A000A8C600100D0A4552524F523A20526563A6
:1017B0006569766564206D6573736167652066721F
:1017C0006F6D204B4B5420646F206E6F74207374C8
:1017D000617274207769746820307830340D0A00A3
:1017E0000D0A4552524F523A204352432066726FBF
:1017F0006D204B4B54206D657373616765206D6977
:10180000736D61746368210D0A0000000D0A4D4577
:1018100053534147453A204D6573736167652066B0
:10182000726F6D204B4B542069732072656365693C
:101830007665642E20436F6D6D616E64203D2030AF
:101840007825780D0A0000000D0A4D455353414795
:10185000453A204D6573736167652073686F756CD9
:1018600064206265206578656375746564206F6EB9
:10187000205043422E0D0A000D0A4D455353414757
:10188000453A204D6573736167652073686F756CA9
:101890006420626520726573656E64656420746F90
:1018A00020464E2E0D0A0000F0050020FE04001018
:1018B0002000002042000010FE480079FD494979CF
:1018C00000EB012080B20A90FA488179BDF8280027
:1018D00007F029F8F8480078F8490870F6480088B9
:1018E00000124870F44880788870F34948681BF00B
:1018F000DEFE0C900C9888B100200D900AE0EE48B6
:1019000040680D99415CED4A0D98C01C11540D982A
:10191000401C0D90DDE90C108842F0DB0021E74A05
:101920000C98C01C11540C98001DE5490880E54B2B
:1019300008460288E149002004F05CFBE249088087
:101940000121E24807F099FF0121E04807F0C1FFBB
:101950004FF0000B07E709F0AAF81422D549091D3A
:10196000DB48FEF75BFE0A22D2491831D9481BF04A
:101970000BFF09F0ABF8D34B00221146104604F0E0
:1019800039FBD14908800121D04807F076FF0121B9
:10199000CE4807F09EFF4FF0000BE4E64FF0000B3F
:1019A000052006F0BBFEC74B00221146104604F08E
:1019B00021FBC54908800121C44807F05EFF0121D1
:1019C000C24807F086FFCEE6BA484079B94989791E
:1019D00000EB012080B20A90B6480079062810D2A8
:1019E000DFE800F00D0B09070503BB4C0CE0BB4C16
:1019F0000AE0BB4C08E0BB4C06E0BB4C04E0BB4C2F
:101A000002E000200A9000BF00BFBDF8280028B106
:101A1000BDF828202146A9481BF0E2FDBDF82800AA
:101A2000A7490880A74B08460288A449002004F073
:101A3000E1FAA54908800121A44807F01EFF012111
:101A4000A24807F046FF4FF0000B8CE609F02FF894
:101A500007F069F908B9012000E000208246994B9F
:101A60000022114604F0C6FA9749088001219748E0
:101A700007F003FF0121954807F02BFF09F026F836
:101A80004FF0000B6FE632200D9012E009F00FF8D6
:101A9000974800780C9009F019F80C98022800DAA1
:101AA00008E064200AF094FD0D99481E0D9001B9DC
:101AB00000E0EBE700BF08F0FAFF00218D4814F0CA
:101AC00016FE81467B48007978B164208A490880F7
:101AD00000208A49087001208949087049F4006291
:101AE0000021844814F0E6FD11E04FF4FA708249B9
:101AF000088000207E4908700120804908708049D4
:101B0000087029F4006200217A4814F0D3FD6D4B6F
:101B100000221146104604F06DFA6B49088001213D
:101B20006A4807F0AAFE0121684807F0D2FE08F0D3
:101B3000CDFF4FF0000B16E608F0B9FF71480268C0
:101B400071495E481BF04CFD6E4800685C49088096
:101B500000206C49086008F0B9FF5A4B58480288C9
:101B60005649002004F046FA574908800121574899
:101B700007F083FE0121554807F0ABFE4FF0000B44
:101B8000F1E54C4840784B49897800EB012080B260
:101B90000A90BDF82800401E80B20A9008F087FF26
:101BA000BDF828204349091D58481BF019FD0020A5
:101BB0005649BDF828208854BDF8280054490860CB
:101BC00008F084FF3F4B00221146104604F012FA41
:101BD0003D49088001213D4807F04FFE01213B4867
:101BE00007F077FE4FF0000BBDE508F060FF06221E
:101BF0003049091D47481BF0F3FC42480068000AC1
:101C00002E4948703F480068087002202C4908801F
:101C100008F05CFF2B4B2A4802882849002004F07A
:101C2000E9F9294908800121284807F026FE012109
:101C3000264807F04EFE4FF0000B94E508F037FF02
:101C40001C4800791B49497900EB01203249A1F871
:101C5000F4000021304805F0FEFA4FF481712E485F
:101C600005F0F9FA174B00221146104604F0C2F9AC
:101C7000154908800121154807F0FFFD012113488F
:101C800007F027FE08F022FF4FF0000B6BE522481B
:101C9000B0F8F4000012094948701F4890F8F400A9
:101CA0000870022006490880064B0846028803494E
:101CB000002033E0A8C6001024070020FE04001016
:101CC00020000020AECA0010420000100054004066
:101CD000C0A00010E9A0001038E4020878E3020870
:101CE000D4E20208DEE10208A8E002082AE10208C4
:101CF0008C000020F80700208A000020340000201B
:101D0000350000202C0000209D7A00106D8200100C
:101D1000300000203D000020C89F001004F06AF948
:101D2000FE4908800121FE4807F0A7FD0121FC487B
:101D300007F0CFFD4FF0000B15E508F0B8FE4FF0AF
:101D400000600068F7490840B0F1005F07D04FF02D
:101D500000600068F4490840B0F1805F13D10021B1
:101D6000F24805F078FA4FF48171F04805F073FA03
:101D70004FF0040BEE4B00221146104604F03AF9E6
:101D8000E649088009E0EA4B00221146012004F0F0
:101D900031F9E24908804FF0000B0121E04807F0DB
:101DA0006CFD0121DE4807F094FD08F08FFEDAE4B7
:101DB000E0480068000EE049C870DE480068000C8A
:101DC0008870DC480088000A4870DA48007808709B
:101DD0000420DA490880D64B08460288D6490020FC
:101DE00004F008F9CD4908800121CD4807F045FDF0
:101DF0000121CB4807F06DFD4FF0000BB3E408F074
:101E000056FECF48007930B90020CE490870012035
:101E1000CD49087004E00120CA490870CA49087019
:101E2000C34B00221146104604F0E4F8BB49088079
:101E30000121BB4807F021FD0121B94807F049FD08
:101E400008F044FE4FF0000B8DE408F030FEBC4873
:101E50004078BB49897800EB012080B20A900021CC
:101E6000B74ABDF82800C01C11548021AF4850303B
:101E70001BF0DEFBB2490C31AC4850301BF039FC92
:101E8000AF480079AE49497900EB0120A749A1F894
:101E9000E800AB488079AA49C97900EB0120A34941
:101EA000A1F8EA00A648007AA549497A00EB01208A
:101EB0009E49A1F8EC00A248807AA149C97A00EBBA
:101EC00001209A49A1F8EE000021984805F0C3F9D5
:101ED0004FF48171954805F0BEF9954B00221146EB
:101EE000104604F087F88D49088001218C4807F0DE
:101EF000C4FC01218A4807F0ECFC08F0E7FD4FF034
:101F0000000B30E48948B0F8E80000128A494870B4
:101F1000864890F8E80008708448B0F8EA0000129B
:101F2000C870824890F8EA0088708048B0F8EC00E9
:101F3000001248717D4890F8EC0008717B48B0F8B9
:101F4000EE000012C871794890F8EE008871002008
:101F50000A900BE075485030BDF82810405C00B97D
:101F600008E0BDF82800401C80B20A90BDF82800A7
:101F70008028EFD300BF00200D900AE06B4850305E
:101F80000D99415C6C4A0D98083011540D98401C15
:101F90000D90BDF828100D988842EFDBBDF82800A1
:101FA000083066490880624B084602886249002072
:101FB00004F020F8594908800121594807F05DFCD8
:101FC0000121574807F085FC4FF0000BC2E408F0F0
:101FD0006EFD5B4800795549A1F8F20058484079F8
:101FE000A1F8F0005648807900065549C97900EB00
:101FF00001405349097A00EB01205149497A0844CC
:1020000009904A4909980EF044F94D48807A000633
:102010004B49C97A00EB01404949097B00EB01209B
:102020004749497B084409904049103109980EF00E
:1020300030F94348807B00064149C97B00EB0140F1
:102040003F49097C00EB01203D49497C0844099047
:102050003649203109980EF01CF93948807C000679
:102060003749C97C00EB01403549097D00EB01206F
:102070003349497D084409902C49303109980EF0C4
:1020800008F92F48807D00062D49C97D00EB0140ED
:102090002B49097E00EB01202949497E084409901B
:1020A0002249403109980EF0F4F8204CD034002039
:1020B0000D9010E00D991A31214A505C2146FFF72E
:1020C0007DF9A41C0D98052802D02D202070641CD9
:1020D0000D98401C0D900D980628EBDB0020207019
:1020E0000021124805F0B7F84FF481710F4805F050
:1020F000B2F80F4B00221146104603F07BFF074950
:1021000008800121064807F0B8FB0121044807F0C8
:10211000E0FB08F0DBFC4FF0000B17E04200001082
:10212000005400400000FE2F0000FF1FC89F001059
:10213000AECA001018000020FE040010200000208D
:10214000A8C600103400002035000020FF2006F053
:10215000E5FA22E4FA4890F8F200FA490870F848E3
:1021600090F8F000487009A9F5480EF04CF8F448D2
:10217000B0F8F20020B1F448007808B900200990C6
:10218000F049099848710998000A08710998000CEB
:10219000C8700998000E887009A9E94810300EF03F
:1021A00032F8E748B0F8F20020B1E748007808B903
:1021B00000200990E349099848720998000A0872BA
:1021C0000998000CC8710998000E887109A9DC48AB
:1021D00020300EF018F8DA48B0F8F20020B1DA48F2
:1021E000007808B900200990D649099848730998E1
:1021F000000A08730998000CC8720998000E8872CA
:1022000009A9CF4830300DF0FEFFCD48B0F8F000FE
:1022100020B1CD48007808B900200990C949099833
:1022200048740998000A08740998000CC873099842
:10223000000E887309A9C24840300DF0E4FFC04881
:10224000B0F8F00020B1C048007808B9002009902B
:10225000BC49099848750998000A08750998000C46
:10226000C8740998000E8874B548D030FFF7CEF8CE
:10227000B4498875B248D330FFF7C8F8B149C8757A
:10228000AF48D630FFF7C2F8AE490876AC48D9302F
:10229000FFF7BCF8AB494876A948DC30FFF7B6F841
:1022A000A8498876A648DF30FFF7B0F8A549C87678
:1022B0001C20A6490880A64B08460288A149002098
:1022C00003F098FEA34908800121A34807F0D5FA3E
:1022D0000121A14807F0FDFA4FF0000B7BE39F4876
:1022E000006858B10120974908709C480068007A3E
:1022F00048709A4800680079887005E0002091498C
:102300000870FF204870887095484078012801D1F6
:102310003F2001E0934800788A49C87004208B4927
:1023200008808B4B084602888649002003F062FE35
:10233000884908800121884807F09FFA01218648D2
:1023400007F0C7FA4FF0000B45E38448006830B14E
:102350008248006817F07AF9002080490860FFF78A
:1023600063F81CF09FFA002101607D4840787C49A9
:10237000897800EB0120401E0D9000210D98001D72
:10238000774A11541046007900F010081046007981
:1023900000F00800D8B110460079C0F3800000902A
:1023A000B8F1000F01D1012000E0002008B10220A7
:1023B00000E0052003466A48007900F003026848FF
:1023C0004179083017F043FB644908601AE064481B
:1023D0000079C0F380000090B8F1000F01D1012016
:1023E00000E0002008B1022000E0052003465C4820
:1023F000007900F003025A484179083017F015FBC4
:10240000564908601CF04EFA00685749087017F0EA
:10241000BAFC52480068E8B353480078D0BB0020AB
:102420000D90002640E04FF0000807200B900020A0
:102430000C9025E049480068C06848490968496827
:102440000C9A06FB0121405C00F001000B9A511E22
:10245000904040EA080000F0FF080B910B9800281C
:102460000BDA3E480068C1680D9A501C0D9001F8C7
:1024700002804FF0000807200B900C98401C0C9035
:102480003648006840680C998842D3DC0B980728CE
:1024900009D000E019E031480068C1680D9A501C6D
:1024A0000D9001F80280761C2C4800684068B0420C
:1024B000B9DC2A4909684968C81DC11700EB517188
:1024C000C910264A126891600CE02748007810B9BC
:1024D0000620254908702148006817F0B7F8002049
:1024E0001E4908601A4B002211461F48007803F06D
:1024F00081FD184908800121174807F0BEF9012124
:10250000154807F0E6F94FF0000B64E21348006845
:1025100060B3134800790C901048006840680C992B
:10252000884224DD0D4800680089084908800B486E
:102530000068C068054A12880C9901FB020422E079
:10254000C89F0010FE04001046000020200000205C
:10255000AECA0010420000100054004038000020B5
:10256000A8C600103C0000204400002015E0FB48F5
:1025700000680089F949096889884843F849088052
:10258000F6480068C468F74BF548028821460020E9
:1025900003F030FDF44908800DE00020F349087095
:1025A000EF490880EF4B08460288F049002003F00D
:1025B00021FDED4908800121ED4807F05EF9012178
:1025C000EB4807F086F94FF0000B04E2E948006899
:1025D00008B30120E5490870E6498868C11700EB97
:1025E0005171C1F3C701E14A5170E2498868C117CE
:1025F00000EB5171C910A0EBC10109B1012100E04C
:102600000021DA4A52781144D84A5170D948007BE7
:102610001146887005E00020D4490870FF204870FA
:102620008870D5484078012801D13F2001E0D34887
:102630000078CE49C8700420C9490880C94B0846B3
:102640000288CA49002003F0D5FCC749088001214F
:10265000C74807F012F90121C54807F03AF94FF0D1
:10266000000BB8E1BD48006830B1BC48006816F006
:10267000EDFF0020B9490860FEF7D6FE1CF012F904
:1026800000210160BC484078BB49897800EB0120FB
:10269000401E0D9000210D98001DB74A11541046A0
:1026A0000079B449C1F8A40E10464079086110467B
:1026B00080791146C97900EB01200D900D981BF02F
:1026C00085FA41EC190B9FEDAE0B53EC102B1BF070
:1026D0000EFA41EC180B1BF0E2FAA649C1F8A80E5D
:1026E000A5480830C1F89C0E08461AF043FDA148E1
:1026F00090F8B00EA44908709A4B00221146A248E7
:10270000007803F077FC984908800121984807F089
:10271000B4F80121964807F0DCF84FF0000B5AE1BD
:102720009448006860B3944800790C909149886897
:10273000C11700EB5171C1F3CF01894A11808D4956
:102740008868C11700EB5171C910A0EBC10109B134
:10275000012100E00021824A12881144804A118040
:102760008448016812880C9800FB02147D4B7C4859
:1027700002882146002003F03DFC7B4908800DE0E3
:1027800000207A49087076490880764B084602880E
:102790007649002003F02EFC73490880012174481B
:1027A00007F06BF80121724807F093F84FF0000B27
:1027B00011E108F07CF9704840786F49897800EBA6
:1027C0000120401E80B20A9000200D9009E00D9873
:1027D000001D6949085C6D490D9A88540D98401C8C
:1027E0000D90BDF828100D988842F0DB0020674955
:1027F000BDF8282088540B224FF40B71634804F075
:1028000097FC584B00221146104603F0F3FB564943
:1028100008800121564807F030F80121544807F09C
:1028200058F808F053F94FF0000BFF2005F076FF41
:10283000D1E000200D9008E054480D99405C4B49D0
:102840000D9A88540D98401C0D900D980A28F3DBC2
:102850000A2043490880434B084602884349002028
:1028600003F0C8FB404908800121414807F005F802
:1028700001213F4807F02DF84FF0000BABE008F0C6
:1028800016F9434800783949087042481AF00FFF9A
:102890000C900C9880B100200D9009E03D480D99F6
:1028A000415C324A0D98401C11540D98401C0D900B
:1028B000DDE90C108842F1DB08F008F900212B4A11
:1028C0000C98401C11540C98801C25490880254BFD
:1028D000084602882549002003F08CFB2249088025
:1028E0000121234806F0C9FF0121214806F0F1FF2C
:1028F0004FF0000B6FE0204840781F49897800EBCB
:102900000120401E80B20A900021BDF82800001D61
:10291000194A115409F06BFE1749091D1E481BF096
:102920008FFF09F06CFE09F062FE1CA11A481BF033
:1029300087FF09F064FE0B4B00221146104603F09E
:1029400059FB094908800121094806F096FF012139
:10295000074806F0BEFF4FF0000B3CE038000020B7
:1029600020000020AECA001042000010FE0400103B
:1029700000540040408A0010A8C600103C0000200F
:102980000000000000408F4044000020BC9F001069
:102990009E00002000A90010EC0000100D0A0000AD
:1029A00009F025FEF2A1F9481BF04AFF09F027FEC5
:1029B000F74B00221146012003F01CFBF54908806B
:1029C0000121F54806F059FF0121F34806F081FF87
:1029D0004FF0000B00BF00BF01F089BF08F067F89F
:1029E00072B6EE480D9004224FF401710DA804F068
:1029F000CBFB00BF00BF00BF00BF00BFBFF34F8FC6
:102A000000BF00BF00BFE648006800F4E060E54991
:102A10000843001DE249086000BF00BF00BFBFF3CC
:102A20004F8F00BF00BF00BF00E000BFFDE7DE48E2
:102A30000078F8B908F03BF86420DC49088008F019
:102A400045F8DB48C078032802D1FF20D949088027
:102A50000AABCF4AD8480188D548FDF7A4FE01212A
:102A6000CD4806F00AFF0121CB4806F032FF4FF0B7
:102A7000000BB1E7CE48C07820287DD01EDCA0F145
:102A80000200182881F02487DFE810F0E40A560BD2
:102A9000F9091F0A6705E80CE70CE70CE70CE70CDF
:102AA000E70CE70CE70CE70C4E058A06EF069305EA
:102AB00015066607E9076507F4086209402876D01D
:102AC00011DC312874D007DC212872D0262871D07F
:102AD000302841F0FD86FAE332286CD033286BD0E1
:102AE0003528F6D1F4E3442867D006DC41286FD0BE
:102AF00042286ED04328ECD1EBE3452805D0462888
:102B000073D06028E5D101F09BBEA9480079A8499F
:102B1000497900EB01200D90A848407868BBA74890
:102B2000D0F81A000D99884255D11820A349487051
:102B3000A348C089062818D005DC3FD2DFE800F0A2
:102B40003E0C0E1012140B2807D0152807D01F2892
:102B500007D0292832D106E000BF00BF00BF00BF68
:102B600000BF00BF00BF00BF00BF40F2D2209549A8
:102B700008800222811E01E0F9E32CE0924804F073
:102B8000EEFA002504209149088008460188904803
:102B90001AF04EFD8A48807B8D4908707C4B8B482B
:102BA0000288002003F026FA7A4908800FE057E2F5
:102BB000F0E3F0E3F0E3F0E3F0E3A5E2744B00228E
:102BC0001146082003F016FA7249088000BF0AE097
:102BD000F8E3F8E309E06E4B00221146022003F00F
:102BE00009FA6C49088001F073BE744840781828CF
:102BF0007ED17348C089062816D005DC60D2DFE894
:102C000000F05F600C0E10120B285BD0152805D069
:102C10001F2805D0292853D104E000BF00BF00BF02
:102C200000BF00BF00BF00BF67480088E0B3654831
:102C30000088801C81B20222664804F090FA654840
:102C40000088001D63490880084602885D480188A5
:102C50005F4804F084FA5B4800885E4909880844AC
:102C6000584908805B4800885849088058480078CF
:102C70005749497800EB0126554880785449C9786E
:102C800000EB01200B905048008852490988401AF7
:102C90004D4908803E4B4D4802884D49002003F0C5
:102CA000A9F93C4908800BE0FFE700204349487040
:102CB000374B00221146082003F09CF93549088063
:102CC000C4E100BF00BF25E005EB4500424901EB30
:102CD0008000408801280DD105EB45013E4A02EBFA
:102CE000810148681AF0E3FC18B9681C85B202E05B
:102CF000ADE111E010E03248C08901280AD105EBAE
:102D00004500354931F8200040F24D41884201D15B
:102D1000681C85B2272DD7DB00BF272D0BD10020E3
:102D2000264948701A4B00221146082003F062F928
:102D30001849088089E12948407808B1F02000E06E
:102D400083200C9000200D9064E02448407870B1FE
:102D500005EB4500204931F820000D9901EB4101B8
:102D60001F4A32F8211088423CD101203BE03DE06F
:102D70000D0A4552524F523A20556E6B6E6F776E68
:102D800020636F6D6D616E64210D0A00EC00001010
:102D9000AECA0010420000100054004055AA55AAC7
:102DA0000CED00E00000FA05430000208800002040
:102DB000A8C600108E000020400000105C99001092
:102DC0003A9900105C0000205E00002020000020E6
:102DD000FE0400106000002078EE02088C990010BC
:102DE00098F80208002006468EB117E005EB450072
:102DF000FE4931F82000FE490D9A31F83210884220
:102E000001D1012000E00020064606B106E00D9841
:102E1000401C0D90DDE90C10884296DB00BF16B90E
:102E2000681C85B24FE7F34C05EB4500EF4931F8DC
:102E300020000C9040F23C410C9888426AD1691CF9
:102E400001EB4101E94A02EB810148681AF02FFCCD
:102E50008246A91C01EB4101E44A02EB810148686A
:102E60001AF025FC0AEB000606F10800E24908808A
:102E7000BDF830002080A41C084600882080A41CD7
:102E800040F23D400C90BDF830002080A41C691C2D
:102E900001EB4101D54A02EB810148681AF007FCB9
:102EA0000B90BDF82C002080A41C681C00EB400097
:102EB000CE4A02EB8000416820460B9A1AF090FB44
:102EC0000B98044440F23D400C90BDF83000208047
:102ED000A41CA91C01EB4101C44A02EB8101486812
:102EE0001AF0E5FB0B90BDF82C002080A41CA81C58
:102EF00000EB4000BD4A02EB8000416820460B9A7F
:102F00001AF06EFBBC480088001DBB490880E81C15
:102F100085B291E00C98B0F57D7F1FD105EB45019E
:102F2000B24A02EB81014868FDF728FB08900420B3
:102F3000B1490880BDF830002080A41C08460088F4
:102F40002080A41C0846028808A920461AF048FBE5
:102F5000A9480088001DA84908806BE040F235416F
:102F60000C98884233D10620A3490880BDF8300070
:102F70002080A41C084600882080A41C21208DF8F5
:102F8000040004208DF805009C48D0F81406000EBB
:102F90008DF806009948D0F81406000C8DF807004B
:102FA0009648B0F81406000A8DF80800934890F887
:102FB00014068DF809000846028801A920461AF077
:102FC0000FFB8D480088001D8B49088032E005EB1F
:102FD0004500864901EB8000408801280AD105EBB5
:102FE0004501824A02EB810148681AF060FB824980
:102FF000088007E005EB45007C4901EB8000008973
:103000007D490880BDF830002080A41C7A480088E3
:103010002080A41C05EB4500744A02EB8000416847
:103020007548028820461AF0DBFA73480088001DB4
:1030300071490880681C85B2714B6F4802886D49E0
:10304000002002F0D7FF6F49088000BF07E06C4BFB
:1030500000221146022002F0CDFF6A490880C2E535
:1030600032224FF42571684804F0B9F866480078B8
:1030700006282BD005DC31D2DFE800F0301418210F
:103080002319152817D004DC072823D00B2825D1B5
:1030900004E01F2814D0292820D113E030205649FD
:1030A00008801BE02F205449088017E000BF0F2044
:1030B0005149088012E016204F4908800EE000BFF9
:1030C00000BF00BF13204C49088007E02D204A496B
:1030D000088003E01B204849088000BF00BF464825
:1030E0000088801C444908800846028846494148B7
:1030F0001AF076FA424B404802883E49002002F01E
:1031000079FF404908806EE54048B0F80100022888
:1031100009D100200D903D4800793C49497900EBE8
:1031200001200C9009E0394800790D90374840792A
:103130003649897900EB01200C90354800790D99CA
:10314000884252D100202C4908800D90FDE00D9856
:1031500000EB4000254931F820000C9988427DD1D0
:10316000244C40F23C410C98884278D10D99491C7E
:1031700001EB41011D4A02EB810148681AF097FA00
:1031800082460D99891C01EB4101184A02EB81012D
:1031900048681AF08CFA0AEB000606F10800164996
:1031A0000880BDF830002080A41C06F108000B90B8
:1031B000084600882080A41C40F23D400C90BDF8D9
:1031C00030002080A41C0D99491C01EB4101074AE5
:1031D00002EB810148681AF06AFA0B90BDF82C00E6
:1031E0002080A41C0D98401C14E0CAE078EE020870
:1031F00080F40208FE040010200000208C990010CA
:10320000AECA00104200001008990010A8C60010B5
:103210005500002000EB4000F64A02EB80004168B8
:1032200020460B9A1AF0DCF90B98044440F23E4019
:103230000C90BDF830002080A41C0D99891C01EB76
:103240004101EC4A02EB810148681AF030FA0B9018
:10325000BDF82C002080A41C0D9801E072E010E065
:10326000801C00EB4000E34A02EB800041682046EE
:103270000B9A1AF0B5F9E0480088001DDE49088075
:103280005FE0DE4C0C98B0F57D7F23D10D9901EB0A
:103290004101D84A02EB81014868FDF76FF90890B7
:1032A0000420D5490880BDF830002080A41C0846C1
:1032B00000882080A41C0846028808A920461AF02D
:1032C0008FF9CD480088001DCB49088039E006E120
:1032D00056E164E00D9800EB4000C64901EB800028
:1032E000408801280BD10D9901EB4101C14A02EB45
:1032F000810148681AF0DBF9BF49088008E00D98A1
:1033000000EB4000BB4901EB80000089BA4908800E
:10331000BDF830002080A41CB74800882080A41C81
:103320000D9800EB4000B34A02EB80004168B248C0
:10333000028820461AF054F9AF480088001DAE49B3
:10334000088006E00D98401C0D900D982728FFF688
:10335000FEAE00BFA848008850B1A94BA64802881D
:10336000A649002002F046FEA649088011E017E1B8
:10337000A34B00221146082002F03CFEA149088020
:1033800007E09F4B00221146082002F033FE9D49C2
:10339000088028E4ACE0EAE097E0B3E0BBE09A48BC
:1033A0000078C0F3400020B197480078C0F3800057
:1033B00050B1934B00221146022002F01BFE9149AE
:1033C000088070E082E06FE09048B0F8010010B92A
:1033D00000200D9002E08D4800790D908C48007916
:1033E0000D99884257D1854C8A48D0F80F11216039
:1033F00090F813012071641D8748016821604168BD
:1034000061608068A0600C34142283491231204628
:103410001AF0E6F814347F4890F80E012070641C0E
:103420007C4890F82B017B4991F828110844794990
:1034300091F82C11491C8840764991F84311891C58
:103440008840744991F82A11C91C8840714991F843
:103450002D11091D884040010D900D982070641CAD
:103460006C4890F82C012070641C6A48D0F8000663
:103470002060241D6748D0F81406206030205E4983
:1034800008805F4B084602885C49002002F0B2FDCC
:103490005C49088007E05A4B00221146082002F0E0
:1034A000A9FD58490880DAE50020544908704870A1
:1034B000022051490880524B084602884F4900209B
:1034C00002F098FD4F490880C9E500BF4C4B00222F
:1034D0001146082002F08EFD4A490880BFE5484B9E
:1034E0001E224949002002F085FD46490880B6E5C4
:1034F000434B102244490A31002002F07BFD414930
:103500000880ACE53E4B05224149002002F072FDE7
:103510003C490880A3E53A4B11224049002002F0C3
:1035200069FD384908809AE5344C05203249088005
:103530003548C07820703A480088A4F8010038481F
:103540004089A4F803002E4B08460288214600203B
:1035500002F050FD2B49088081E500202A4948707F
:103560001E2240F24121284803F00EFE00BF244BEA
:1035700000221146104602F03DFD224908806EE50A
:1035800000201E49087001201B4908801C4B08467A
:1035900002881A49002002F02DFD1A4908805EE5D4
:1035A000174B10221F49002002F024FD1549088006
:1035B00055E515484078B8BB1348C078A0B3012042
:1035C0000A9000200D9048E00F48401D0D99415C85
:1035D0000D98001D0D4A105C814200D13AE00A4866
:1035E000401D0D99415C0D98001D084A105C8142F8
:1035F0001BDA35E078EE020820000020FE040010FF
:10360000AECA0010420000105C990010A8C600105D
:10361000550000208C9900108E9A00106AF0020864
:103620003A99001080F002083CE0FE480D99415C98
:103630000D98001DFC4A105C81420ADDFB4B002204
:103640001146072002F0D6FCF949088000200A90B4
:1036500006E000BF0D98401C0D900D980528B3D3CF
:1036600000BFBDF8280028B30820EE49491F487064
:1036700040F2D220EF490880EF48EB494A680260E7
:10368000097A01711E2240F24121E648401F03F0F1
:103690007BFDE64B00221146104602F0ABFCE449EC
:1036A000088007E0E14B00221146022002F0A2FC54
:1036B000DF490880D3E4DB48401F4078082866D102
:1036C0000520DE49C8810846D0F80200401CC1F838
:1036D00002000020C1F80A00FCF786FFD749C1F8B4
:1036E000060012224FF41E71D44803F04DFD002055
:1036F000CC49491F4870C870D048D0F80200C1F8C2
:103700001A000846CC490A68C0F8052009794172B8
:103710001E2240F2412103F037FDC948C6490A681C
:10372000C0F8022009798171C448D0F80210C44859
:10373000C0F80710C148D0F80610C148C0F80B10F7
:10374000BE480188BE48A0F80F10BC48807BBC4929
:10375000087032224FF42571B94803F015FD00209E
:10376000FDF799FEB3480088A0F2D22080B20A90FB
:1037700002224FF434710AA803F0DAFCAB4B0A22A0
:10378000AE49002002F036FCA949088007E0A74BAB
:1037900000221146022002F02DFCA54908805EE4BB
:1037A000A048401FC078E0BB01200A9000200D9087
:1037B0002BE09C480D99415C0D98001D9A4A105CC5
:1037C000814200D11EE097480D99415C0D98001D83
:1037D000954A105C814200DA1AE092480D99415CEA
:1037E0000D98001D904A105C81420ADD8F4B00222B
:1037F0001146072002F0FEFB8D49088000200A9048
:1038000006E000BF0D98401C0D900D980528D0D300
:1038100000BFBDF8280038B302208249491F487014
:1038200000E019E040F2D2208249088082487E49B7
:103830004A680260097A01711E2240F241217948EA
:10384000401F03F0A1FC794B00221146104602F004
:10385000D1FB7749088007E0744B00221146022013
:1038600002F0C8FB724908804DE46E48401F407862
:10387000022867D17149C8810846D0F80200401C6F
:10388000C1F8020008460088401C0880FCF7ACFE26
:103890006A49C1F8060012224FF41E71674803F00E
:1038A00073FC00205F49491F48700120C8706348BD
:1038B000D0F80200C1F81A0008465F490A68C0F84B
:1038C0000520097941721E2240F2412103F05CFC7F
:1038D0005B4859490A68C0F8022009798171574844
:1038E000D0F802105648C0F807105448D0F8061017
:1038F0005348C0F80B10514801885148A0F80F10E8
:103900004E48807B4E49087032224FF425714C4856
:1039100003F03AFC0120FDF7BEFD46480088A0F206
:10392000D22080B20A9002224FF434710AA803F028
:10393000FFFB3E4B0A224149002002F05BFB3C4961
:10394000088007E0394B00221146022002F052FBAA
:10395000374908801DE500BF3248401F407880BBD2
:103960003048401FC07860B301200A9000200D90BD
:103970002CE02C480D99415C0D98001D2A4A105CE2
:10398000814200D11FE027480D99415C0D98001D30
:10399000254A105C814200DA1BE022480D99415C07
:1039A0000D98001D204A105C81420BDD1F4B002248
:1039B0001146072002F01EFB1D49088000200A90D6
:1039C00007E043E000BF0D98401C0D900D980528BE
:1039D000CFD300BFBDF82800A0B31348C078172884
:1039E00004D114200F49491F487003E004200D49F9
:1039F000491F487040F2D2200E4908800E480A49FB
:103A00004A680260097A01711E2240F2412105488C
:103A1000401F03F0B9FB054B00221146104602F08F
:103A2000E9FA10E061990010A8C60010AECA0010B3
:103A3000420000105C000020500000203A99001065
:103A4000089900100AE0FE49088007E0FD4B0022BB
:103A50001146022002F0CEFAF949088099E4FA48AA
:103A6000407804280BD0F8484078142807D0F6484E
:103A70004078142803D0F4484078152869D10120F3
:103A80000A9000200D902BE0F0480D99415C0D98B4
:103A9000001DEF4A105C814200D11EE0EB480D99F9
:103AA000415C0D98001DEA4A105C814200DA1AE080
:103AB000E6480D99415C0D98001DE54A105C814275
:103AC0000ADDE04B00221146072002F093FADC49A0
:103AD000088000200A9006E000BF0D98401C0D9061
:103AE0000D980528D0D300BFBDF8280080B3D84872
:103AF000407AD8490882002006900790D448D0F830
:103B00000A100691807B8DF81C0003AADDE90601EE
:103B100005F0E2F99DF80C200DF10D014FF47F70D6
:103B2000FDF78DFCC8484078042806D0112805D040
:103B300014280FD0152818D10DE000BFC64890F802
:103B40002A0108B9032000E00420C249C8810CE022
:103B50008FE086E000BFC04890F82A0108B91F2016
:103B600000E02920BB49C88100BF00BFB948D0F898
:103B70000200401CB749C1F802000846D0F80A000C
:103B8000401CC1F80A00FCF72FFDB249C1F806003D
:103B900012224FF41E71AF4803F0F6FA0020AA4932
:103BA0004870AC48D0F80200C1F81A000846A7498E
:103BB0000A68C0F80520097941721E2240F24121AD
:103BC00003F0E2FAA548A1490A68C0F80220097981
:103BD0008171A048D0F80210A048C0F807109D4895
:103BE000D0F806109D48C0F80B109A48817B9B487E
:103BF000C173974C0A34216801612179017592489B
:103C00004078964908709348807B087032224FF4C0
:103C10002571924803F0B8FA0720FDF73CFC904864
:103C20000088A0F2D22080B20A9002224FF43471B0
:103C30000AA803F07DFA874840898A4908808548A8
:103C4000D0F80200C1F802008248D0F80600C1F89E
:103C500006007C4B0A22002002F0CCF9784908804B
:103C600007E0784B00221146022002F0C3F97449A4
:103C7000088018E474484078C8BB73480078C0F3E3
:103C80004000A0B370480078C0F3800078BB0120EA
:103C90000A9000200D902FE06B48401D0D99415C6B
:103CA0000D98001D6A4A105C814200D121E06648EF
:103CB000401D0D99415C0D98001D654A105C8142C4
:103CC00000DA1CE06048401D0D99415C0D98001D14
:103CD0005F4A105C81420BDD5A4B002211460720DF
:103CE00002F088F95649088000200A9007E026E093
:103CF00000BF0D98401C0D900D980528CCD300BF37
:103D0000BDF8280018B317204F49487040F2D22060
:103D1000534908804D484E494A680260097A01714A
:103D20001E2240F24121484803F02EFA454B002262
:103D30001146104602F05EF94149088007E0414B08
:103D400000221146022002F055F93D49088016E490
:103D50003D484078172871D115203E49C881084652
:103D6000D0F80200401CC1F80200FCF73DFC3949C4
:103D7000C1F8060012224FF41E71364803F004FA0F
:103D80000020314948703348D0F80200C1F81A00C9
:103D900008462E490A68C0F80520097941721E229A
:103DA00040F2412103F0F0F92C4828490A68C0F894
:103DB0000220097981712748D0F802102748C0F8FD
:103DC00007102448D0F806102448C0F80B10002132
:103DD000C0F80F101F48807B20490870084600215A
:103DE000C0F81310C17532224FF4257103F0CCF9DD
:103DF0000820FDF750FB1A480088A0F2D22080B2BC
:103E00000A9002224FF434710AA803F091F9114884
:103E1000D0F80200134908600E48D0F80600486048
:103E2000002088600846002181818173054B0F22A4
:103E30000146002002F0DEF8014915E016E000001E
:103E400042000010AECA00105C9900105000002023
:103E5000A8C600103A9900108C990010089900101B
:103E60005C0000204C990010088007E0F64B00220F
:103E70001146022002F0BEF8F44908801AE4F44822
:103E8000C078C8B9F2480078C0F34000A0B1F0484B
:103E90000078C0F3800078B91020ED49487040F2F6
:103EA000D220EC490880E84B00221146104602F06F
:103EB000A1F8E649088007E0E34B00221146022002
:103EC00002F098F8E149088069E4E1484078102858
:103ED0007ED100200D902FE0DD48401D0D99415C02
:103EE0000D98001DDC4A105C814200D121E0D848C9
:103EF000401D0D99415C0D98001DD74A105C814210
:103F000000DA1CE0D248401D0D99415C0D98001D5F
:103F1000D14A105C81420BDDCB4B002211460720B9
:103F200002F068F8C94908800020C949487006E0D5
:103F300000BF0D98401C0D900D980528CCD300BFF4
:103F40000620C649C8810846D0F80200401CC1F8C6
:103F50000200FCF749FBC149C1F8060012224FF4E8
:103F60001E71BE4803F010F90020B9494870BB48E3
:103F7000D0F80200C1F81A000846007820F00400CA
:103F8000001D08700846B4494A68C0F80520097A3F
:103F900041721E2240F2412103F0F6F8B048AC49CC
:103FA000D1F80520C0F80220497A8171AB48D0F8D9
:103FB0000210AB48C0F80710A848D0F80610A8486F
:103FC000C0F80B100F30A7494A6902608A6900E007
:103FD00037E04260C96981601422A24914310C3073
:103FE00019F0FEFA9D48807B9D49087032224FF4FB
:103FF00025719B4803F0C8F80020FDF74CFA95485E
:104000000088A0F2D22080B20A9002224FF43471CC
:104010000AA803F08DF8082093490880934C8F4834
:10402000D0F8020020608D48D0F806006060864B12
:10403000084602882146002001F0DCFF8349088001
:1040400007E0814B00221146022001F0D3FF7F4997
:10405000088002E27E480078C0F38000F0BB84480C
:10406000C078D8B37A480078C0F3400020B17848CF
:104070000078C0F3800008B1FCF756FA7648407823
:104080007549897800EB0120401E0C900C9818B9F6
:1040900000207849087003E06F480079754908707E
:1040A0006B480078C0F3400038B169480078C0F32D
:1040B000800010B96F48007860B165480078C0F39F
:1040C000400020B162480078C0F3800068B16948C0
:1040D000007850B15C4B0022114600E023E0022042
:1040E00001F088FF5949088025E059480078C0F35D
:1040F000400040B156480078C0F3800018B9132042
:104100005349487002E001205149487040F2D220E2
:10411000504908804C4B00221146104601F06AFFBE
:104120004A49088007E0484B00221146022001F06E
:1041300061FF46490880CBE345484078012803D019
:104140004348407813287CD1434C241D01200A9019
:104150003F480078C0F3400090B33D480078C0F37A
:10416000800068BB00200D902FE03948401D0D995C
:10417000415C0D98001D384A105C814200D121E05D
:104180003348401D0D99415C0D98001D324A105C6A
:10419000814200DA1CE02E48401D0D99415C0D98CB
:1041A000001D2D4A105C81420BDD274B0022114679
:1041B000072001F01FFF2549088000200A9007E032
:1041C00007E000BF0D98401C0D900D980528CCD33A
:1041D00000BFBDF82800A8B31D482168C0F805102D
:1041E000217941720078C0F3400040B1184800784E
:1041F000C0F3800018B91F480078012849D1102267
:1042000013490A311C4819F0EBF91648801C54F880
:10421000051F016061684160A1688160641F14220C
:1042200004F11101123019F0DBF914482168C0F8CB
:104230000F11217980F813110E48007801281FD141
:104240001FE002E109E10000AECA001042000010C8
:104250005C9900105C000020A8C600103A9900107C
:10426000089900108C9A001020000020FE04001015
:10427000550000205A000020909F00108C990010DB
:104280000020F74981F818061221F64819F0D0F9F4
:1042900004E094F82700F24981F8180614F8250F75
:1042A000EF4981F80E0160780D90607800F0010010
:1042B00081F82B016078C0F3400081F82801607814
:1042C000C0F3800081F82C016078C0F3C00081F851
:1042D00043016078C0F3001081F82A016078253C22
:1042E000C0F3401081F82D01DF484078012800D14B
:1042F00000E00B20DB49C8810846D0F80200401CD2
:10430000C1F80200FCF770F9D649C1F80600122284
:104310004FF41E71D34802F037FFD248D0F80200A4
:10432000CF49C1F80006CF48D0F80600C1F81406FE
:104330000020CD494870CB48D0F80200C1F81A00DF
:104340000846007820F00200801C08700846C74923
:104350004A68C0F80520097A41721E2240F24121C4
:1043600002F012FFC2480079401CC149087108469A
:10437000C078401EC870052240F26921BC4802F096
:1043800003FFBC48B849D1F80520C0F80220497A9B
:104390008171B448D0F80210B648C0F80710B1488F
:1043A000D0F80610B348C0F80B100F30B2494A6974
:1043B00002608A694260C96981601422AE49143181
:1043C0000C3019F00DF9A64890F80E11A94880F8A4
:1043D0002F100D98C1B2A74880F83010A04890F86F
:1043E0001816A44880F831109E48807BA1490870B7
:1043F00032224FF425719F4802F0C6FE0020FDF7DF
:104400004AF89E480088A0F2D22080B20A90022288
:104410004FF434710AA802F08BFE72B6FCF75EF816
:1044200062B6082096490880964C8E48D0F8020063
:1044300020608C48D0F806006060934B08460288E4
:104440002146002001F0D6FD07E08F4B00221146E7
:10445000022001F0CFFD8D49088039E28248407882
:10446000002871D0814840788049897800EB01208C
:10447000401E0C907D4C241D804800880C990844F7
:10448000B0F5006F0CDA0C9882B27C4801882046A7
:1044900002F04EFE794800880C990844774908805C
:1044A00071484078012803D06F484078132879D1AB
:1044B000B0E160880D90208840F22642811A904237
:1044C0007BD032DC40F20C42A0EB020190426BD078
:1044D00018DCB0F57D7F75D00ADCB0F57A7F50D05E
:1044E000A0F2E93088B301287CD0082849D1FBE04C
:1044F000A0F2F53050B304286CD0052856D0082817
:104500003FD1DEE00C2941D008DC012963D0042929
:1045100072D0052971D00A2933D116E1142975D03A
:1045200015296CD018292CD1F4E07E2968D015DC2F
:10453000302966D00BDC0F2972D0162971D02E29B4
:1045400073D02F291DD185E071E164E0AFE03729F8
:1045500069D0402968D07D2913D1D1E0912974D048
:1045600008DC7F296ED080296DD083296CD08D29FD
:1045700007D1B2E0932905D0972970D09F2900D1A7
:1045800035E039E120793649487035E1211D34485C
:10459000801C0D9A19F024F800213148801C0D9AD6
:1045A000815429E13AE108E044E00BE0211D324862
:1045B000801C0D9A19F014F81EE12079284981F821
:1045C0000E0119E1211D2C480F300D9A19F008F841
:1045D00012E107E0B2E0211D274814300D9A18F0CF
:1045E000FFFF09E120791E4981F8280104E12079C3
:1045F0001B4981F82901FFE0CCE0D0E006E051E062
:10460000AFE02079164981F82A01F5E020791449B4
:1046100081F82B01F0E02079114981F82C01EBE0C1
:10462000C9E0CDE001E07FE037E020790C4981F876
:104630002D01E1E0211D10482E300D9A18F0D0FF19
:10464000DAE002E097E09BE022E02079044981F87B
:104650004201D1E02079024981F84301CCE094E0A5
:104660008C9900103A9900105C990010A8C60010AF
:1046700055000020089900108C9A00105C00002062
:1046800020000020FE040010AECA001042000010FE
:104690002079FE4981F84401AEE02079FB4981F898
:1046A0004501A9E02079F94981F84601A4E0211DDE
:1046B000F7480D9A18F094FF0021F5480D9A81549F
:1046C0009AE0211DF24814300D9A18F089FF00215C
:1046D000EF4814300D9A81548EE0211DEC4854307F
:1046E0000D9A18F07DFF87E0211DE94860300D9A92
:1046F00018F076FF0021E64860300D9A81547BE087
:10470000211DE4480D9A18F06BFF0021E1480D9A35
:10471000815471E0211DE0480D9A18F061FF0021DD
:10472000DD480D9A815467E0211DDC480D9A18F090
:1047300057FF0021D9480D9A81545DE0211DD748CB
:1047400040300D9A18F04CFF56E0211DD3484C30F4
:104750000D9A18F045FF0021D0484C300D9A815435
:104760004AE0211DCE480D9A18F03AFF0021CC48AE
:104770000D9A815440E02079C44981F8FB053BE063
:104780002079C24981F8FC0536E0A088BF49A1F82C
:10479000FE0531E0BD496068C1F800062CE0211D2E
:1047A000BF4811300D9A18F01BFF0021BC48113092
:1047B0000D9A815420E0B5496068C1F814061BE0E9
:1047C000241D66883246211DB548273018F008FFA1
:1047D0000021B34827308155301D04446688324695
:1047E000211DAF48313018F0FBFE0021AC483130BC
:1047F0008155301D044400BF00BF208840F23C4179
:10480000884202D00D98001D0444DDE90C10001D03
:10481000081A0C900C9800287FF44BAEA14B002294
:104820001146104601F0E6FB9F49088007E09D4BCA
:1048300000221146022001F0DDFB9B49088047E081
:104840009A480079162804D0182803D0192834D1A2
:1048500023E000BF1E2240F24121954802F094FC63
:104860001E2240F24121934802F0B9FC052240F299
:104870006921914802F088FC052240F269218F48A5
:1048800002F0ADFCFBF750FE864B002211461046AD
:1048900001F0B0FB8449088018E0002088490870C6
:1048A0000120884908807F4B0846028884490020FF
:1048B00001F0A0FB7C49088008E07A4B00221146F9
:1048C000104601F097FB7849088000BF00BF00BF89
:1048D00000BF01217C4804F0D0FF01217A4804F098
:1048E000F8FF4FF0000B02E04FF0000B00BF00BFDD
:1048F0000A2007F06DFEFCF75DBE00BF0100A0F1CD
:104900000100FBD1704707F072FE70A1764819F0E4
:1049100097FF07F074FE00240CE006F0C8F8734817
:10492000057806F0D3F805B106E04FF47A7007F089
:104930004FFE641C0F2CF0DB00BF0DB9082625E0EC
:1049400007F055FE6AA1684819F07AFF07F057FE94
:1049500007F04DFE69A1644819F072FF07F04FFEA1
:1049600000240CE006F0A3F86C48057806F0AEF8D9
:1049700005B106E04FF47A7007F02AFE641C142C8F
:10498000F0DB00BF05B134E0092600BF07F02FFEC1
:1049900063A1554819F054FF07F031FE28E00024C8
:1049A00012E06548408B40F0100063494883FA20CC
:1049B00007F00EFE6048008B40F010005E4908834F
:1049C000FA2007F005FE641CB442EADB5A48408B2B
:1049D00040F0200058494883FA2007F0F9FD564876
:1049E000008B40F0200054490883FA2007F0F0FDC6
:1049F000D5E707F0FCFD3EA13B4819F021FF07F089
:104A0000FEFD1BE04C48408B40F010004A494883B3
:104A10000846008B40F020000883962007F0D8FD60
:104A20004548008B40F01000434908830846408BFE
:104A300040F020004883962007F0CAFDE2E72DE908
:104A4000FC5F0746B94666E14FF4966506F02FF81D
:104A500000203A49086006F039F807F0C8FD38A18F
:104A6000214819F0EDFE07F0CAFD002001AB40F22D
:104A7000CF723E490090484611F063FC0446002C7A
:104A800076D101980C2874DD384873E08C990010B9
:104A9000D39A0010339C0010339D0010339E0010F9
:104AA0007F9F0010AECA001042000010A8C6001080
:104AB0004CF002085C9900107BF0020855000020C1
:104AC000FE04001020000020005400404C696E6B72
:104AD0002073746174652069732077616974696EED
:104AE000672E2E2E0D0A0000EC000010450000205D
:104AF000446F6E652E2E2E0D0A0000004950206670
:104B0000726F6D2044484350206973207761697447
:104B1000696E672E2E2E0D0A000000004600002050
:104B20004552524F523A2042616420726573756C4F
:104B300074210D0A00000000000002402C0000203B
:104B400057652061726520726561647920746F20F9
:104B50007265616420636F6D6D616E642066726F53
:104B60006D2050432E2E2E0D0A0000009D7A00105D
:104B7000C5E015E00078022812D10198401FFA49DB
:104B8000085C03280CD1881DFCF740FC804607F028
:104B90002EFD4246F5A1FE4819F052FE07F02FFD0A
:104BA00005F085FF0020FB49086005F08FFF4FF0FE
:104BB000000A019802281DD1EB480078102819D16D
:104BC00007F015FDF4A1F24819F03AFE07F017FDC1
:104BD00005F06DFF0120EF490860E348407800F0E0
:104BE0000F00F449085CF44908700020487005F093
:104BF0006DFF66E005F05BFFF0490198086005F085
:104C000065FFEF48007870282BD105F050FFEB4985
:104C10000198086005F05AFF0BE005F048FFE748EF
:104C2000006886B205F052FF06B907E0642007F07D
:104C3000CFFC2800A5F101018DB2EED100BF019893
:104C4000401EC949085C1B280AD10198801E085CD7
:104C50001B2805D14FF000080020D949087000E05A
:104C600059E020E005F023FFCA48006886B205F04D
:104C70002DFF06B11CE005F01AFFD048006886B28F
:104C800005F024FF66B9BAF1000F09D107F0AFFCB7
:104C9000CCA1BF4819F0D4FD07F0B1FC4FF0010AD8
:104CA000642007F095FC2800A5F101018DB2D9D14F
:104CB00000BF07F09CFCCBA1B54819F0C1FD07F07F
:104CC0009EFC65B1BC4818F0F2FC83460020034608
:104CD0005A46B9490090484611F0D9FA044607F0FF
:104CE00086FCC8A1AA4819F0ABFD07F088FCB449BE
:104CF00081F80080084600786D2800D10CE04CB1A6
:104D000007F075FC2246C6A1A14819F099FD07F0ED
:104D100076FC01E000BF97E600BF07F068FCC4A185
:104D20009B4819F08DFD07F06AFC0221484611F0FE
:104D300053FB07F05CFCC4A1954819F081FD07F016
:104D40005EFC484611F067FB07F051FCC4A1904897
:104D500019F076FD07F053FCC74807F0DAFCBDE810
:104D6000FC9F1FB5B5E00421C34807F0A6FC38B985
:104D700007F03DFCC1A1864819F062FD07F03FFC39
:104D80000621012011F03CF904463CB907F02FFC44
:104D9000C2A17F4819F054FD07F031FCC648B0F8B5
:104DA000F420C649204611F0CBF906463EB107F083
:104DB0001EFCC3A1764819F043FD07F020FC00213A
:104DC000204611F002FA06463EB107F010FCC4A1DD
:104DD0006F4819F035FD07F012FC0120C949087031
:104DE000012700BF07F003FCC7A1694819F028FD9F
:104DF00007F005FC07F0FBFBC5A1654819F020FD95
:104E000007F0FDFB0220BF49087003AA01A9204654
:104E100011F0F3F9054645B907F0E9FBC7A15C4875
:104E200019F00EFD07F0EBFB39E00021924807F086
:104E30005AFCA0B907F0DBFB002101A80CF0B5F982
:104E40008046BDF80C0043463A46C6A10090504843
:104E500019F0F6FC07F0D3FB01F0C6F81FE0CE48CE
:104E60000068401CCC49086007F0C1FB002101A884
:104E70000CF09BF98046BDF80C0043463A46C7A1AA
:104E80000090434819F0DCFC07F0B9FB2846FFF717
:104E9000D6FD4B4800786D2800D102E000BF7F1C92
:104EA000A0E700BF07F0A3FBCAA1394819F0C8FC6E
:104EB00007F0A5FB0221204611F08EFA07F097FBC0
:104EC000CCA1334819F0BCFC07F099FB204611F047
:104ED000A2FA48E7F8B500264AF6AA20CD490860AC
:104EE0001E21CD4818F0A4FBCC4800210160416090
:104EF0008160C16078221421C94818F092FB7822A1
:104F00000A21C84818F08DFBC7A1CA4818F0F1FB68
:104F10000020C9490870FBF750FA02F0D9FB0821BC
:104F2000C64804F0B2FB00281CD107F060FBC4A106
:104F3000174819F085FC07F062FB00249BE1BF488D
:104F4000408B40F01000BD4948830846408B40F03C
:104F500020004883C148FFF7D0FCB848008B40F0E0
:104F600010007DE182E200009D7A00105765206804
:104F700061766520636F6D6D616E642066726F6D22
:104F800020504320307825782E2E2E0D0A00000068
:104F9000EC0000103000002053686F7274207374AE
:104FA0006174757320726571756573742E2E2E0D84
:104FB0000A0000003D0000206D8200102C0000203F
:104FC00014000020436F6D6D616E64207761732063
:104FD00072656164696E67206279204543522E2EA6
:104FE0002E0D0A00416E737765722066726F6D2018
:104FF0004543522069732072656164792E2E2E0D0F
:105000000A000000416E7377657220776173207328
:10501000656E6420746F2050432E2E2E0D0A000002
:105020004572726F7220307825782E2E2E0D0A0070
:10503000477261636566756C2073687574646F7719
:105040006E2E2E2E0D0A0000436C6F73696E672062
:10505000636F6E6E656374696F6E2E2E2E0D0A007F
:10506000436F6E6E656374696F6E20636C6F7365FA
:10507000642E2E2E0D0A0000080000204661696C87
:10508000656420746F206372656174652073656D5B
:105090006170686F7265210D0A00000043616E6ED9
:1050A0006F74206F70656E2045435220736F636B81
:1050B0006574210D0A000000C89F0010A462030857
:1050C0004661696C656420746F2062696E64204576
:1050D000435220736F636B6574210D0A000000005A
:1050E0004661696C656420746F20656E746572201A
:1050F0006C697374656E696E672073746174652181
:105100000D0A0000900000200D0A0D0A00000000AA
:1051100057616974696E6720666F7220616E2069DD
:105120006E636F6D696E6720636F6E6E6563746921
:105130006F6E2E2E2E0D0A0D0A00000043616E6E5A
:105140006F7420616363657074206E657720636F90
:105150006E6E656374696F6E2072657175657374C8
:10516000210D0A00436F6E6E656374696F6E2023B4
:10517000257520726566757365642077697468208B
:10518000636C69656E7420257320706F72742025BE
:10519000752E2E2E0D0A000010000020436F6E6E3B
:1051A000656374696F6E2023257520657374616271
:1051B0006C6973686564207769746820636C6965DD
:1051C0006E7420257320706F72742025752E2E2E1C
:1051D0000D0A0000477261636566756C2073657225
:1051E0007665722073687574646F776E2E2E2E0D3F
:1051F0000A000000436C6F73696E672073657276F6
:10520000657220636F6E6E656374696F6E2E2E2EED
:105210000D0A0000003000405C9900107C990010DD
:10522000C0A00010E9A000104E6F206D657373617F
:105230006765730000A900109E0000200000024076
:105240000D0A466163746F7279206D6F6465206426
:1052500065746563746564210D0A000040420F00A7
:10526000FE4908830846008B40F020000883FC4874
:10527000FFF743FB641C0A2CFFF661AE07F0B7F999
:10528000F8A1FC4819F0DCFA07F0B9F902F084F84B
:10529000054605B1B7E007F0AAF9AFF2AC71F548E1
:1052A00019F0CEFA07F0ABF907F0A1F9F2A1F14835
:1052B00019F0C6FA07F0A3F94FF47A7001F0F3FE83
:1052C000F148FFF71AFB07F092F9AFF2DC71E948F9
:1052D00019F0B6FA07F093F907F089F9EBA1E54860
:1052E00019F0AEFA07F08BF90025002412E02846E9
:1052F0006D1CC1B2204601F009FF00B90DE0E0B21B
:10530000FF2806D1002C04DD601CC11700EB1161E1
:105310000D12641CB4F5006FE9DB00BFB4F5006F3B
:1053200001DA05256FE007F062F9AFF63C01D148DC
:1053300019F086FA07F063F907F059F9D9A1CD48B9
:1053400019F07EFA07F05BF900240DE0204601F029
:10535000E6FE0546E11704EB116104EB2121C9B219
:10536000A94200D003E0641CB4F5006FEEDB00BF7F
:10537000B4F5006F01DA062545E007F038F9AFF61D
:105380009001BC4819F05CFA07F039F90021CA48CD
:1053900001F061FF4FF48171C74801F05CFF00220A
:1053A000C549C64801F08EFF0B224FF40B71C4486B
:1053B00001F0BEFE0B224FF40B71C24801F0CFFE8C
:1053C00007F015F9C0A1AB4819F03AFA07F017F940
:1053D00002F037FA07F00BF9C0A1A64819F030FA2D
:1053E00007F00DF901204FF448730022AFF6E921D0
:1053F0000090C0A007F0C5F808B9072503E007F042
:10540000BCF800BFFEE707F0F2F8BEA1994819F01A
:1054100017FA07F0F4F828E0002412E08F48408BD8
:1054200040F010008D494883BC48FFF766FA8B486E
:10543000008B40F0100089490883B848FFF75DFAF7
:10544000641CAC42EADB8548408B40F02000834975
:105450004883B248FFF751FA8048008B40F02000A3
:105460007E490883AD48FFF748FAD5E7AC48FFF717
:1054700044FAAC480078A8B90421AB4802F09FFF79
:1054800040B107F0B4F8A9A17A4819F0D9F907F0AA
:10549000B6F807E007F0ABF8A9A1764819F0D0F903
:1054A00007F0ADF800228449844801F00BFFC8B929
:1054B0004FF481728049814801F004FF70B90021E6
:1054C0007E4801F0C8FE4FF481717C4801F0C3FEB4
:1054D00000227949794801F0F5FE03E00021774880
:1054E00001F0B9FE0B224FF40B71764801F037FE44
:1054F00058B90B224FF40B71714801F019FE0B22C1
:105500004FF40B716F4801F02AFE6B49D0316B48A4
:10551000D03018F0D3F878B1684890F8D0006649D8
:1055200091F8D010884207D1644890F8D1106248B1
:1055300090F8D10081422CD0FBF756F806465E4920
:10554000D0315E48D03018F0D4F8F0B25B49D93190
:10555000FBF734FF2D21594880F8DB1000F1DC0106
:10556000C6F30720FBF72AFF2D21544880F8DE10F0
:1055700000F1DF01C6F30740FBF720FF00214F4891
:1055800080F8E11001F067FE4FF481714B4801F0A3
:1055900062FE6448007890B907F029F86EA135489A
:1055A00019F04EF907F02BF802F04BF907F01FF84D
:1055B00070A1304819F044F907F021F842E01E22AA
:1055C00040F24121734801F00AFE58B91E2240F210
:1055D0004121714801F0D8FD1E2240F241216D4861
:1055E00001F0FDFD052240F269216C4801F0F7FD54
:1055F00058B9052240F26921694801F0C5FD05222C
:1056000040F26921654801F0EAFD12224FF41E7153
:10561000644801F0E4FD48B91221624818F008F826
:1056200012224FF41E715F4801F0AEFD5948007818
:10563000C0F3400030B157480078C0F3800008B98B
:10564000FAF72AFF584800684078574909680978EE
:105650000A2212FB010000F00F00A7E00000024048
:1056600040420F004932432070696E2074657374A4
:10567000210D0A00EC00001042656570207465730E
:1056800074210D0A00000000A0860100454550521B
:105690004F4D2077726974652074657374210D0A0B
:1056A00000000000454550524F4D20726561642056
:1056B00074657374210D0A0090F00208C89F0010F1
:1056C00062000020BC9F0010504859206D6F647527
:1056D0006C6520696E69740D0A0000004661637490
:1056E0006F7279205461736B2073746172740D0A48
:1056F00000000000466163746F7279205461736B1F
:10570000000000000D0A4552524F523A2042616497
:1057100020726573756C74210D0A0000404B4C00BB
:10572000001BB70043000020005C00400D0A20462B
:105730004E20697320636F6E6E656374656421002B
:105740000D0A20464E206973206E6F7420636F6EC1
:105750006E656374656421000D0A20496E69746981
:10576000616C697A696E672045746865726E6574EC
:105770002E2E2E000D0A20496E697469616C697ABB
:10578000696E672069732066696E69736865642154
:105790000D0A00005C9900104CF002085500002032
:1057A0007BF002083A990010780000208030EE4922
:1057B0000870EE48007860B900204FF44873024644
:1057C000EB490090EBA006F0DCFE10B9EEA019F05A
:1057D00045F801204FF448730022F2490090F2A0EE
:1057E00006F0CFFE10B9E8A019F038F8F44806F03A
:1057F00099FF38B906F0FBFEF2A1FA4819F020F83B
:1058000006F0FDFE002064230246F7490090F7A051
:1058100006F0B7FE10B9DCA019F020F800206423D0
:105820000246F4490090F4A006F0ABFE10B9D6A0F1
:1058300019F014F802204FF4FA730022AFF6DD21BC
:105840000090EFA006F09DFE38B906F0D0FECEA184
:10585000E44818F0F5FF06F0D2FE06F08EFE0020B8
:10586000F8BD10B582780A2392FBF3F403FB1422EF
:1058700030324A70827892FBF3F230320A702D2275
:105880008A70427892FBF3F403FB142230320A71DF
:10589000427892FBF3F23032CA702D224A710278BC
:1058A00092FBF3F403FB14223032CA71027892FBAC
:1058B000F3F230328A7120220A72C27892FBF3F43A
:1058C00003FB142230328A72C27892FBF3F2303238
:1058D0004A723A22CA72027992FBF3F403FB142251
:1058E00030324A73027992FBF3F230320A730022AB
:1058F0008A7310BD2DE9F04194B004460D466069ED
:10590000C66805F0D4F82022C04909A817F068FE3F
:105910001022BF4905A817F063FE05F0D7F8BDA116
:10592000284617F049FF60B9BE480068401CBD49D1
:1059300008600846BCA1026804F52B7018F09EFFB1
:105940007BE2BAA1284617F037FF28B9BA4904F517
:105950002B7017F0CEFE70E2B8A1284617F02CFF8E
:1059600028B9B94904F52B7017F0C3FE65E2B7A159
:10597000284617F021FF30B9B748016804F52B70AD
:1059800017F0B7FE59E2B5A1284617F015FF40B948
:1059900006F0EEFE804604F52B71404606F018FF37
:1059A0004BE2B1A1284617F007FF48B912A93046CB
:1059B00007F01CFF04F52B7112A809F041FB3CE233
:1059C000ACA1284617F0F8FE48B911A9304609F0F5
:1059D000D5FF04F52B7111980AF05BFC2DE2A8A10C
:1059E000284617F0E9FE48B911A9304609F0F2FF40
:1059F00004F52B7111980AF04CFC1EE2A3A1284675
:105A000017F0DAFE48B911A930460AF00DF804F58E
:105A10002B7111980AF03DFC0FE2A0A1284617F067
:105A2000CBFE50B911AA002130460AF02DF804F53A
:105A30002B7111980AF02DFCFFE19DA1284617F06B
:105A4000BBFE50B911AA012130460AF01DF804F539
:105A50002B7111980AF01DFCEFE19AA1284617F06E
:105A6000ABFE38B99DF824206FA104F52B7018F017
:105A700005FFE2E196A1284617F09EFE38B99DF891
:105A8000252069A104F52B7018F0F8FED5E194A14A
:105A9000284617F091FE38B99DF8262062A104F53A
:105AA0002B7018F0EBFEC8E190A1284617F084FE99
:105AB00038B99DF827205CA104F52B7018F0DEFEA4
:105AC000BBE18EA1284617F077FE38B99DF8282053
:105AD00055A104F52B7018F0D1FEAEE18AA128463D
:105AE00017F06AFE58B901A90DF12900FFF7B9FEB8
:105AF00001AA89A104F52B7018F0C0FE9DE187A1D1
:105B0000284617F059FE38B911220DF12E0104F57F
:105B10002B7017F039FE90E183A1284617F04CFE58
:105B200038B9DDF83E2040A104F52B7018F0A6FE30
:105B300083E180A1284617F03FFE38B99DF8142074
:105B400039A104F52B7018F099FE76E17CA1284666
:105B500017F032FE38B99DF8152033A104F52B70EB
:105B600018F08CFE69E1F1E03C00002043000020C9
:105B70000B0A01084F46442045786368616E6765EB
:105B8000205461736B0000004661696C6564207489
:105B90006F20637265617465207461736B210D0AF7
:105BA000000000009D1501084C697374656E6572F4
:105BB000204B4B5420493243205461736B0000004A
:105BC0000C0000204661696C656420746F2063726C
:105BD0006561746520464E206D75746578210D0AE7
:105BE00000000000EC000010A10601084C656431C3
:105BF00000000000030701084C656432000000004B
:105C000053534C2053657276657200005C99001006
:105C10007C990010504147455F434F554E544552C3
:105C20000000000094000020257500004543525FED
:105C30004E414D4500000000C0A000104543525F9A
:105C400053455249414C0000E9A000104543525FC2
:105C500056455253494F4E00780000205359535433
:105C6000454D5F54494D45004D41435F41444452C9
:105C700000000000495056345F4144445200000087
:105C80005355424E45545F4D41534B0044454641A8
:105C9000554C545F4741544557415900495056347B
:105CA0005F5052494D4152595F444E53000000002D
:105CB000495056345F5345434F4E444152595F4417
:105CC0004E530000464E5F504841534500000000CF
:105CD000464E5F444F435F5354415445000000001B
:105CE000464E5F444F435F4441544500464E5F5328
:105CF000484946545F53544154450000464E5F574F
:105D000041524E494E470000464E5F444154455F64
:105D100054494D450000000025730000464E5F4E7B
:105D2000554D424552000000464E5F444F435F4E82
:105D3000554D00004F46445F535441544500000008
:105D40004F46445F524541440000000052A128469E
:105D500017F032FD40B9BDF81620AFF2341104F54A
:105D60002B7018F08BFD68E04EA1284617F024FD3B
:105D700038B9AFF24C1104F52B70069A18F07EFD7D
:105D80005BE04AA1284617F017FD58B901A907A8FA
:105D9000FFF767FD01AAAFF2800104F52B7018F040
:105DA0006DFD4AE044A1284617F006FD38B9454A82
:105DB000AFF29C0104F52B7018F060FD3DE042A1AC
:105DC000284617F0F9FC50B93E485038B0F8E820A2
:105DD000AFF2AC1104F52B7018F050FD2DE03DA191
:105DE000284617F0E9FC38B93D4AAFF2D40104F572
:105DF0002B7018F043FD20E03AA1284617F0DCFC98
:105E0000B8B93B48007820B139480078C0F58070B7
:105E100001E03748007802463548007808B135A0DF
:105E200001E0AFF2FC10014604F52B7018F026FDDE
:105E300003E0EB2014B0BDE8F08104F52B7017F0FF
:105E400036FC07463A4604F52B71204610F0F6FD65
:105E5000F0E7024640F2051070472DE9F041064692
:105E60000F46904635460020287000240FE03CB1D4
:105E700004F00F0020B920A1284618F0FFFC0544CB
:105E80003A5D20A1284618F0F9FC0544641C4445FD
:105E9000EDD33046BDE8F0814F46445F434F554E49
:105EA000540000004F46445F4E554D004F46445F3E
:105EB00044415445000000004F46445F4144445271
:105EC0000000000018A000104F46445F504F52548D
:105ED000000000004F46445F4D4553534147450085
:105EE00000A900104F46445F4552524F5200000037
:105EF0009E0000202D2575000D0A20202020202046
:105F000020200000253032582000000070B50446E3
:105F10002146F9480BF038F90546002D1DD006F052
:105F200066FBF6A1FE4818F08BFC06F068FB00202B
:105F30002060606000232246EF49184610F046FBBF
:105F4000054655B106F053FBEB4AF6A1F44818F0AC
:105F500077FC06F054FB284670BD0020FCE77CB5BA
:105F60006846FFF7D3FF04460CB120467CBD0621EE
:105F7000012010F045F8F44908600846006848B967
:105F800006F035FBF1A1E64818F05AFC06F037FBA5
:105F9000C820EBE706F02BFB002168460BF005F963
:105FA0000546D5485038B0F8E8302A46EEA1DC481E
:105FB00018F046FC06F023FBCF485038B0F8E82034
:105FC0006946E148006810F0D0F8044614B16FF05B
:105FD0002400CBE706F00BFBEFA1D14818F030FC12
:105FE00006F00DFB0020C1E710B5D748006810F09F
:105FF00012FA10BD2DE9F04780460F4615461C46A3
:106000004FF0000904202070681C6070000AA07026
:1060100084F8038047B1002604E0B95D301D2154A7
:10602000701C86B2AE42F8DBE91C601C00F008FF71
:106030008146281D04F800904FEA2921681D21544B
:10604000A81D80B2BDE8F08770B50446002641F275
:10605000883509E022460421D54802F045F910B1FF
:10606000681E85B200E001E0002DF3D100BF0DB93C
:10607000002070BD6078A17800EB0120401D86B241
:106080003046F6E72DE9F04704460D460026002786
:10609000B046B1462078042803D06FF02200BDE856
:1060A000F087E91E601C00F0CBFE064606F0FF08F4
:1060B0003712681E205CB84203D1A81E205C404500
:1060C00002D06FF02300EAE7E07800F07F0948464D
:1060D000E5E72DE9F04704460D4600260027B046C7
:1060E000B1462078042803D06FF02200BDE8F08785
:1060F000E91E601C00F0A4FE064606F0FF083712F9
:10610000681E205CB84203D1A81E205C404502D026
:106110006FF02300EAE794F803904846E6E701466B
:1061200000208A79CB7902EB03207047FEB5054643
:10613000A04E6946304609F021FC06F058FA9EA1AF
:10614000774818F07DFB06F05AFA01A8FFF7DEFE4B
:1061500004460CB12046FEBD062101200FF050FF81
:10616000794908600846006848B906F040FA77A106
:106170006B4818F065FB06F042FAC820EBE706F022
:1061800036FA002101A80BF010F807465A4850389B
:10619000B0F8E8303A4690A1614818F051FB06F09B
:1061A0002EFA69480068856253485038B0F8E820F4
:1061B00001A9654800680FF0D8FF0446FFF714FFF7
:1061C00014B16FF01000C6E70020C4E710B500243A
:1061D0008D4B002211462220FFF70CFF8B490880CF
:1061E0008B4B8C4A084601888748FAF7DCFA8848C6
:1061F00001888848FFF746FF00280CD006DC10F124
:10620000240F1BD010F1230F38D10DE008282AD01D
:10621000112833D11CE07F4800797E49497900EB91
:10622000012084B2204610BD06F0E1F97AA13C4875
:1062300018F006FB06F0E3F90020F4E706F0D7F9C2
:1062400082A1374818F0FCFA06F0D9F90020EAE7F5
:1062500006F0CDF98CA1324818F0F2FA06F0CFF929
:106260006FF01000DFE706F0C2F996A12C4818F095
:10627000E7FA06F0C4F96FF00700D4E706F0B7F9C3
:106280006448C2789749264818F0DAFA06F0B7F958
:106290006048C07800F07F00032816D106F0A7F907
:1062A00091A11F4818F0CCFA06F0A9F9564B00222C
:1062B00011463520FFF79EFE54490880544B554A3D
:1062C000084601885048FAF76EFA06F090F98DA159
:1062D000134818F0B5FA06F092F94B4B002211461C
:1062E0003020FFF787FE49490880494B494A084654
:1062F0000188454814E1000018A000104661696C4F
:10630000656420746F20636F6E7665727420746F9D
:1063100020495020616472657373210D0A000000EA
:10632000EC0000104661696C656420746F2067653D
:10633000742049502061647265737320666F726DBA
:106340002025730D0A000000980000204661696C4A
:10635000656420746F206F70656E20736F636B656A
:1063600074210D0A000000000D0A53746172744319
:106370006F6E6E656374696F6E2E436F6E6E6563CC
:1063800074696E6720746F2073657276657220255C
:10639000732025640D0A000053756363657373668B
:1063A000756C20636F6E6E656374696F6E0D0A00A5
:1063B000005C0040F807002054727920746F20635D
:1063C0006F6E6E65637420746F207365727665728C
:1063D0002E2E0D0A0000000054657374536572760A
:1063E0006572436F6E6E6563742E436F6E6E656388
:1063F00074696E6720746F207365727665722025EC
:10640000732025640D0A0000F8000010220000200F
:1064100026000020E60800100D0A4552524F523A5D
:1064200020526573706F6E73652066726F6D2046C3
:106430004E20646F206E6F742073746172742077C5
:106440006974682030783034210D0A000D0A4552F5
:10645000524F523A20526573706F6E7365206672A8
:106460006F6D20464E20697320696E76616C696499
:106470002064756520746F20435243206D69736DED
:1064800061746368210D0A000D0A4552524F523A59
:1064900020436F6E6E656374696F6E2077697468F0
:1064A000204F464420536572766572206973206ED2
:1064B0006F742065737461626C6973686564210D23
:1064C0000A0000000D0A4552524F523A204E6F20EA
:1064D0007265717565737465642064617461210D02
:1064E0000A000000A4B203080D0A494E464F3A20A4
:1064F00052656164696E6720464E204572726F7204
:10650000730D0A000D0A494E464F3A2052656164E8
:10651000696E6720464E205374617475730D0A00CE
:10652000FAF741F900207EE6F8B506460C46154616
:10653000002000900420FB490880FB490C702012C9
:1065400048708D702812C870F84BF64802882320D6
:10655000FFF750FDF64908806B4632460846018831
:10656000F248FAF720F9BDF800103046FFF78AFD2F
:1065700001283ED008DC10F1240F18D010F1230FB1
:106580000AD0002840D104E0022827D011283BD1AE
:1065900018E0BDF80000F8BD06F029F8AFF2881148
:1065A000E44818F04DF906F02AF80020F3E706F069
:1065B0001EF8AFF26811DF4818F042F906F01FF834
:1065C0000020E8E706F013F8AFF24411D94818F0BC
:1065D00037F906F014F86FF01000DCE706F007F862
:1065E000D5A1D44818F02CF906F009F86FF0010095
:1065F000D1E705F0FCFFD8A1CE4818F021F905F04D
:10660000FEFF4FF0FF30C6E705F0F1FFDC48C2782F
:10661000DC49C84818F014F905F0F1FF0020BAE78A
:106620002DE9FE4304460D46174601A8FFF76EFC10
:106630008046B8F1000F02D04046BDE8FE83002F2F
:1066400026D12A20D049087008204870412088703F
:106650000A20C87081200871A2204871002088712A
:106660000120C871002606E0C848815DC64A06F1CF
:1066700008001154761C102EF6DB2078C2490876EB
:1066800060784876142088760020C87608774877A6
:1066900005F0ADFF002101A80AF087FD8146BC4846
:1066A000B0F8E8304A46BBA1A24818F0C9F805F096
:1066B000A6FFB748B0F8E82001A9C04800680FF06D
:1066C00054FD8046B248B0F8EE00BC4909688862C3
:1066D00057B9002003461E22AB490090B748006816
:1066E0000FF0D5FD804636E005F081FF3A46B4A1B3
:1066F000904818F0A5F805F082FF05F078FF2A46CB
:10670000B6A18C4818F09CF805F079FF05F06FFFF2
:10671000A078009063782278B5A1864818F090F8A8
:1067200005F06DFF05F063FF681E205C0090A81E59
:10673000235CE81E225CAEA17E4818F081F805F0CB
:106740005EFF002003462A46214600909B480068D1
:106750000FF09DFD8046B8F1000F02D06FF02400CD
:106760006BE7002069E7FEB5002002908848B0F88A
:10677000EC00924909688862002002AB40F20542B1
:10678000A14900908D4800680FF0DBFD0646FFF739
:106790002BFC26B1DB2E02D06FF02400FEBDDB2ED9
:1067A0000AD105F024FF99A1624818F049F805F0D4
:1067B00026FF6FF01100F1E7029800287ED005F067
:1067C00016FF9BA15B4818F03BF805F018FF002569
:1067D0000EE005F00CFF8C49485D01A9F9F7D3FFE5
:1067E00007463946534818F02BF805F008FF6D1C92
:1067F00002988542EDD300208349029A885402987A
:106800001E3882B2494B1E312620FFF7F3FB484960
:1068100008808B4B5A4A084601884448F9F7C3FF61
:10682000874801885648FFF72DFC022855D008DC20
:1068300010F1240F72D010F1230F70D000286FD107
:1068400006E0032854D004285DD02028F7D109E0C1
:1068500005F0CDFE7BA1374817F0F2FF05F0CFFE23
:1068600000209BE705F0C3FE80A1324817F0E8FF47
:1068700005F0C5FE05F0BBFE4148027989A12D480F
:1068800017F0DEFF05F0BBFE6D480088401E0828AB
:1068900020DD04F00CF93A4C641D208840F22B41B5
:1068A000884215D1A08840F2FB31884210D1E0889F
:1068B000402801DD4020E080E28800E054E104F15E
:1068C00008017D4816F08CFE0020E1887A4A505479
:1068D00004F0FCF86FF01F0060E705F088FE77A178
:1068E000144817F0ADFF05F08AFE6FF0010055E780
:1068F00005F07DFE7BA10F4817F0A2FF05F07FFE9B
:106900006FF002004AE705F072FE7CA1094817F01B
:1069100097FF05F074FE6FF003003FE70CE1FFE026
:1069200016E1000024000020FE040010F800001012
:1069300022000020EC0000100D0A4552524F523A3E
:106940002057726F6E67207374617465206F6620C4
:10695000464E210D0A0000000D0A4552524F523A90
:1069600020496E636F727265637420636F6D6D6131
:106970006E6420666F7220464E210D0A00000000F2
:10698000E6080010A4B20308FAA40010EC0C0010F2
:10699000C89F001073656E644F46442E436F6E6E41
:1069A000656374696E6720746F20736572766572B3
:1069B0002025732025640D0A0000000098000020A7
:1069C0000D0A53656E6420746F207365727665726C
:1069D0003A256420626C6F636B0D0A0053697A6517
:1069E0003A2025642062797465730D0A0000000066
:1069F00042797465733A20307825582030782558CC
:106A000020307825580D0A00F4A000100D0A4D45DD
:106A100053534147453A204E6F20616E737765723C
:106A20002066726F6D20736572766572210D0A00A3
:106A30000D546F207365727665722D3E0000000064
:106A4000260000200D0A4D4553534147453A204149
:106A5000636B6E6F6C65646765207761732061633B
:106A6000636570746564210D0A0000000D0A4552CB
:106A7000524F523A20526573706F6E736520667282
:106A80006F6D204F4644205365727665722069739E
:106A900020696E61636365707461626C65210D0AC3
:106AA00000000000524541534F4E3A20436F646549
:106AB0003A307825580D0A0000A900100D0A4552F9
:106AC000524F523A20464E20697320696E207468F6
:106AD000652077726F6E67207374617465210D0A8B
:106AE000000000000D0A4552524F523A20464E20F7
:106AF0006572726F72210D0A000000000D0A455286
:106B0000524F523A2043727970746F636F70726F94
:106B1000636573736F72206572726F72210D0A0064
:106B200005F065FDAFF21071114817F089FE05F010
:106B300066FD6FF0220031E605F059FDAFF2F46119
:106B40000B4817F07DFE05F05AFD6FF0230025E697
:106B500005F04DFD0748C27807A1054817F070FE03
:106B600005F04DFD00BF00BF6FF0100016E60000FD
:106B7000EC000010E60800100D0A4552524F523A40
:106B800020436F6465206F6620726573706F6E734B
:106B9000652066726F6D20464E206973206E6F6EA1
:106BA000206E756C6C3A20307825580D0A00000074
:106BB00000B587B00121880303F087F90121062081
:106BC00003F050F902208DF818008DF8190000200C
:106BD0008DF81A008DF81B000C20059005A995482A
:106BE00002F0EEFC02208DF818008DF8190000204C
:106BF0008DF81A008DF81B004FF48060059005A9F0
:106C00008D4802F0DDFC01208DF8180002208DF87F
:106C1000190000208DF81A004FF40070059005A9A6
:106C2000854802F0CDFC05220221824802F056FD83
:106C3000052203217F4802F051FD05220A217E48EA
:106C400002F04CFD4FF400717B4802F038FD00204B
:106C5000ADF80000ADF80400ADF80600ADF808008E
:106C60004FF40070ADF80A002020ADF80C000020B1
:106C7000ADF80E004FF48270ADF8020069466F481F
:106C800003F0A4FA01216D4803F083FB4FF48071F7
:106C90006A4803F0ADFB07B000BD10B5044600BF65
:106CA0000221664803F02DFC0028F9D021466348F4
:106CB00003F0F0FB00BF0121604803F022FC002834
:106CC000F9D05E4803F0E3FBC0B210BD2DE9F041FE
:106CD00004460E4617464FF40071574802F0F1FC87
:106CE0000620FFF7DAFF4FF40071534802F0E7FC8B
:106CF00042F6E060FDF701FE4FF400714E4802F0ED
:106D0000E0FC0220FFF7C9FF2012FFF7C6FFE0B248
:106D1000FFF7C3FF002506E016F805804046FFF7A1
:106D2000BCFF681C85B2BD42F6DB4FF400714248DF
:106D300002F0C5FCBDE8F08170B504460D464FF485
:106D400000713D4802F0BDFC0620FFF7A6FF4FF49E
:106D50000071394802F0B3FC42F6E060FDF7CDFD6A
:106D60004FF40071344802F0ACFC0220FFF795FFAD
:106D70002012FFF792FFE0B2FFF78FFF2846FFF7E0
:106D80008CFF4FF400712C4802F099FC70BD2DE986
:106D9000F04104460E4617464FF40071264802F0B3
:106DA00090FC0320FFF779FF2012FFF776FFE0B297
:106DB000FFF773FF002505E00020FFF76EFF705519
:106DC000681C85B2BD42F7DB4FF400711A4802F02F
:106DD00076FCBDE8F08170B504464FF400711648AA
:106DE00002F06FFC0320FFF758FF2012FFF755FF5A
:106DF000E0B2FFF752FF0020FFF74FFF05464FF4C8
:106E000000710D4802F05BFC284670BD10B54FF4D0
:106E10000071094802F055FC0520FFF73EFF0020F5
:106E2000FFF73BFF04464FF40071034802F047FCB4
:106E3000204610BD00080240000402400038004017
:106E400070B502460B4641F221054FF6FF70002156
:106E500017E0565C80EA062000240EE000F40046AD
:106E60002EB141F2210686EA4006B0B203E04FF6A9
:106E7000FF7606EA4000661CB4B2082CEEDB4E1C1E
:106E8000B1B29942E5DB70BD10B50BE010F8014BD3
:106E9000138884EA23230F4C34F81330147883EAE0
:106EA000042313800B00A1F10101EFD110BDF8B54F
:106EB00004460D464FF6FF7000902646E81C87B248
:106EC000761C791E6A463046FFF7DEFFBDF80000EB
:106ED000F8BD000080F2020870B504460D46E1B22C
:106EE000144803F090FC00BF4021124803F03BFD22
:106EF0000028F9D0204670BD70B5054600BF0120BE
:106F000000F075FF0446601C0028F8D021460120DF
:106F100000F025FF204670BD10B504462146012033
:106F200000F01DFF10BD01464FF0FF30704700BF5D
:106F3000FEE700000010014000B52DED048B81B08C
:106F40000121084602F0C1FF0121022002F0BDFF2D
:106F50006748006816F04BFE41EC190B9FED650B7E
:106F600053EC102B16F051FD41EC180B16F06BFE94
:106F70004FF0804108853220C8624007808940F088
:106F8000010088810846008840F0010008805848C8
:106F9000006816F02CFE41EC190B9FED560B53ECDC
:106FA000102B16F032FD41EC180B16F04CFE534935
:106FB00008800820091D086050481C38008840F0EF
:106FC00001004E491C3908804C482838008840F0A0
:106FD00001004A49283908801C208DF8000007204C
:106FE0008DF801000F208DF8020001208DF80300BC
:106FF000684601F0AEFF1D208DF800000F208DF8CF
:1070000001008DF8020001208DF80300684601F0B0
:10701000A0FF01B0BDEC048B00BD002013E0384997
:1070200011F8301069B9364901EBC001496841B126
:10703000334901EBC0014968491E314A02EBC002E5
:107040005160411CC8B20628E9DB704710B54FF00B
:107050008040008A20F001004FF080410882FFF755
:10706000DCFF00F085FF2748006820B12548006854
:10707000401E2449086010BD10B52048183800880B
:1070800020F001001D49183908801E48006820B111
:1070900049151D4802F01EFB04E04FF400711A4828
:1070A00002F00FFB10BD1749086070470122144B16
:1070B00003F830201A4602EBC0025160002203F8A8
:1070C0003020704701460E4800EBC100406808B907
:1070D000012070470020FCE710B50446214601203E
:1070E000FFF7E4FF00BF0648C0680028FBD110BDD1
:1070F00000000010F168E388B5F8E43E2804004081
:1071000044A90010180000100010024070B5044699
:107110000D46A0B22946FFF70FFE012070BD70B5E5
:1071200004460025A0B2FFF756FE0546284670BD6E
:107130002DE9F04105460E461746B04600240AE008
:10714000295D404608F10108FFF7E0FF10B9002073
:10715000BDE8F081641CBC42F2D30120F8E72DE9C0
:10716000F04105460E461746B046002407E040466B
:1071700008F10108FFF7D3FF2855601C84B2BC4218
:10718000F5DB0120BDE8F0812DE9F0470546884692
:1071900091464646002700240CE0285D0744295DFF
:1071A0003046761CFFF7B2FF10B90020BDE8F0872B
:1071B000601C84B24C45F0DBF9B23046761CFFF718
:1071C000A5FF08B90020F1E73046761CC7F3072178
:1071D000FFF79CFF08B90020E8E70120E6E72DE96A
:1071E000F04705460F4690463E464FF00009002402
:1071F00008E03046761CFFF792FF2855285D814451
:10720000601C84B24445F4DB3046761CFFF787FFF0
:1072100004463046761CFFF782FF04EB002084B260
:1072200089EA040010B90120BDE8F0870020FBE7DF
:1072300070B504460D460020A4F8F600F82120465B
:10724000FFF7FEFD0646A4F8F660F8222146284620
:1072500016F0C6F970BD2DE9F04106460D462F46E1
:107260002D493046FFF7E4FF00240BE02A4A115D68
:1072700038467F1CFFF74AFF10B90020BDE8F081B7
:10728000601C84B2F82CF1D30120F7E72DE9F0411E
:1072900004460E46F8223146204616F0A1F9B4F80D
:1072A000F6500020A4F8F600F8212046FFF7C8FDAC
:1072B0000746A4F8F650AF4202D10120BDE8F081A4
:1072C0000020FBE72DE9F04106460F461446A04694
:1072D000002508E0404608F10108FFF720FF0E49AD
:1072E0004855681C85B2F82DF4D30B493046FFF79A
:1072F000CDFF18B109A017F0B1FA0BE0F82239461A
:10730000304616F06DF921463046FFF7A4FF002005
:10731000BDE8F0810120FBE774A900105265737489
:107320006F72652073657474696E6773206F6B216B
:107330000D0A00001CB504468DF804404FF480701F
:10734000009000208DF8060014B901208DF8070088
:1073500002208DF805006946D84802F031F94FF453
:10736000007000906946D64802F02AF91CBD1CB591
:1073700004468DF80440C020009000208DF80600DF
:1073800014B901208DF8070002208DF80500694628
:10739000CC4802F015F91CBD2DE9F0410120FFF7A2
:1073A000C9FF0020FFF7E3FFC448408B40F4807022
:1073B000C24948830846008B40F480700883C04867
:1073C0001A30008840F40070BD491A310880881EC8
:1073D000008840F40070891E0880012453E004F006
:1073E000010030B1B548008B40F48070B349088388
:1073F00005E0B248408B40F48070B049488304F007
:10740000020040B1AE481830008840F40070AC492A
:107410001831088007E0AA481A30008840F400704C
:10742000A7491A3108804021A64802F02EF90646E5
:107430008021A44802F029F9054604F0010030B18A
:10744000012E01D1012000E00020074604E00EB922
:10745000012000E00020074617B90120BDE8F081B7
:1074600004F0020030B1012D01D1012000E0002024
:10747000074604E00DB9012000E0002007460FB9DF
:107480000220EBE7641C032CA9DB0120FFF76FFF50
:107490000020FFF74FFF012458E004F0010040B145
:1074A00088481830008840F040008649183108802C
:1074B00007E084481A30008840F0400081491A31C2
:1074C000088004F0020040B17E481830008840F087
:1074D00080007C491831088007E07A481A3000881B
:1074E00040F0800077491A3108804FF4807173486A
:1074F00002F0CBF806464FF40071714802F0C5F86F
:10750000054604F0010030B1012E01D1012000E058
:107510000020074604E00EB9012000E000200746E5
:107520000FB903209AE704F0020030B1012D01D118
:10753000012000E00020074604E00DB9012000E032
:10754000002007460FB9042088E7641C032CA4DB45
:10755000002083E71CB501208DF804001020009066
:1075600000208DF8060002208DF80500694653487A
:1075700002F026F8202000906946504802F020F8DA
:107580001CBD1CB504460CB9012000E000208DF89C
:1075900004000820009000208DF806008DF80700F8
:1075A00001208DF805006946444802F009F81CBD29
:1075B0000EB501208DF808000002019000208DF822
:1075C0000A0001208DF80B008DF8090001A93B4845
:1075D00001F0F6FF3948408B40F48070374948830A
:1075E00049F64040009002E00098401E009000984C
:1075F0000028F9D14FF40071314802F046F808B97B
:10760000012000E000203049087008460078D0B121
:107610002A48008B40F480702849088349F640408E
:10762000009002E00098401E009000980028F9D1D8
:107630004FF40071224802F028F808B1012000E060
:107640000020214908700EBD1CB501208DF80400F2
:107650004002009000208DF806008DF80500694674
:107660001A4801F0ADFF1CBD1CB501208DF80400C7
:107670004020009000208DF8060001208DF80700C2
:1076800000208DF8050069460C4801F099FF402163
:107690000A4802F014F81CBD10B54021074802F05A
:1076A00010F8642004F094FF4021044802F007F829
:1076B0004FF4FA6004F08CFF10BD0000000002409F
:1076C0000008024000040240430000200010024075
:1076D00008B50121084602F0C5FB0121022002F095
:1076E000C1FB0121042002F0BDFB0121082002F0B2
:1076F000B9FB0121102002F0B5FB0121202002F08E
:10770000B1FB0121402002F0ADFB0121802002F0FD
:10771000A9FB0121080202F0A5FBFFF71BFF0120D6
:10772000FFF72FFFFFF790FFFFF79EFF00F094FA9F
:10773000A848009002E00098401E009000980028A1
:10774000F9D104F054FFA4A1A44817F079F804F08B
:1077500056FF04F04CFFA2A1A04817F071F804F006
:107760004EFF04F044FFA7A19C4817F069F804F00D
:1077700046FF04F03CFF9AA1984817F061F804F026
:107780003EFF04F034FFA8A1944817F059F804F024
:1077900036FF04F02CFFADA3AFA2B2A18F4817F0C3
:1077A0004FF804F02CFF04F022FFB348B3A10268A5
:1077B0008A4817F045F804F022FF04F018FFB3A13F
:1077C000864817F03DF804F01AFF04F010FFB0A14E
:1077D000824817F035F804F012FFFFF7ADFB04F014
:1077E00006FFB2A17D4817F02BF804F008FFFFF761
:1077F000DFF90821B54801F048FF002820D0B4483F
:10780000007850B904F0F3FEB2A1744817F018F8EC
:1078100004F0F5FE00F026FC07E004F0E8FEB5A158
:107820006E4817F00DF804F0EAFE04F0E0FEB8A18F
:107830006A4817F005F804F0E2FE042000F0DCFDD1
:1078400008BD30B587B000200090019002900390F1
:10785000B7A1684615F04DFFB749684615F0F3FE2D
:1078600005F031FF04463CB104F0C1FEB3A15B4812
:1078700016F0E6FF04F0C3FEBA4DBBA1284606F0A1
:1078800029F86946284606F03AF8B949284606F02C
:1078900062F8B849284606F074F805A9B64807F01A
:1078A00067FB05A9284605F086FF284606F0E0F8A4
:1078B00004464CB104F09BFE06F10C02AFA1474810
:1078C00016F0BEFF04F09BFEAB48D038B0F8F200D3
:1078D000002819D0B2480DF0F3FAB1480560002035
:1078E000AF494861AF480DF04FFD044614B1AEA05A
:1078F00016F0B4FFAB480DF091FD0446002C32D0D9
:10790000B2A016F0ABFF2EE004A99B48D03808F0D7
:107910007AFC2846049908F00DF804A99648C03866
:1079200008F071FC2846049908F043F804A992482D
:10793000B03808F068FC2846049908F05EF804A9FD
:107940008D48A03808F05FFC00212846049A08F012
:107950007EF804A98848903808F055FC0121284693
:10796000049A08F074F8A1480EF078FF7D489F490A
:107970000860502088800420C8609D4808619DA14F
:107980009A48143015F0B5FE9CA19848343015F093
:10799000B0FE9D48954948659C48C8659C480EF0D6
:1079A00075FF04463CB104F022FE9AA10B4816F084
:1079B00047FF04F024FE96480FF065FA04463CB1F8
:1079C00004F015FE9CA1054816F03AFF04F017FEDE
:1079D00007B030BD801A0600200D0A00EC00001030
:1079E0002A2A2A2A2A2A2A2A2A2A2A2A2A2A2A2AF7
:1079F0002A2A2A2A2A2A2A2A2A2A2A2A2A2A0D0A24
:107A0000000000002A2A2A2A2A2A2A2A2A20495340
:107A10004B524120555044202A2A2A2A2A2A2A2A0F
:107A20002A2A0D0A00000000436F707972696768A6
:107A3000743A20323031362D32303138204F4A43BB
:107A40002049534B52410D0A0000000031303A35B5
:107A5000333A313200000000536570203237203253
:107A600030313800436F6D70696C65643A2025735E
:107A70002025730D0A0000007800002056657273FF
:107A8000696F6E3A2025730D0A0000000D0A000090
:107A90000D0A20496E697469616C697A696E6720A4
:107AA00054696D6572732E2E2E0000000D0A204958
:107AB0006E697469616C697A696E67204652414DDE
:107AC000206D656D6F72792E2E2E00000000024031
:107AD000430000200D0A20496E697469616C697A5F
:107AE000696E6720493243204D41535445522E2E32
:107AF0002E0000000D0A20456D756C6174696F6E73
:107B000020464E206465746563742E2E2E0000009E
:107B10000D0A20496E697469616C697A696E672023
:107B200049324320534C4156452E2E2E0000000072
:107B300049534B5241000000BC9F00104661696CE4
:107B4000656420746F20696E697469616C697A6517
:107B5000205443502F495020737461636B210D0AE8
:107B600000000000F8070020657468300000000085
:107B700010620308BC62030898A000104661696C9B
:107B8000656420746F20636F6E6669677572652027
:107B9000696E74657266616365202573210D0A0044
:107BA0006CAA001098AA00104661696C6564207484
:107BB0006F20696E697469616C697A652044484315
:107BC0005020636C69656E74210D0A004661696C12
:107BD000656420746F20737461727420444843504C
:107BE00020636C69656E74210D0A000028AB0010DB
:107BF000F8AB00102F7777772F000000696E64656F
:107C0000782E7368746D0000F5580108535E010802
:107C100088AB00104661696C656420746F20696EE2
:107C2000697469616C697A652048545450207365A1
:107C300072766572210D0A004661696C6564207474
:107C40006F207374617274204854545020736572AD
:107C5000766572210D0A000000B587B00121102061
:107C600002F044F90121084602F0FCF805A801F0F1
:107C7000F2FC02208DF818000002059002208DF819
:107C8000190000208DF81A0001208DF81B0005A9AD
:107C9000E54801F095FC02208DF81800400205909F
:107CA00002208DF8190000208DF81A0001208DF8AF
:107CB0001B0005A9DC4801F083FC07220921DA48F2
:107CC00001F00CFD07220A21D74801F007FD002230
:107CD00040F22551D54802F021FE0021D34802F0A0
:107CE00067FDD24802F08EFC0121102002F0FEF860
:107CF0004FF4612001900020ADF80800ADF80A00B3
:107D0000ADF80C00ADF810000C20ADF80E0001A984
:107D1000C64802F0C5FC4FF4A06001F015F925201B
:107D20008DF8000005208DF801008DF8020001207B
:107D30008DF80300684601F00CF90121BB4802F000
:107D400037FD012240F22551B84802F0E7FD01223B
:107D500040F22551B54802F0E1FD07B000BD70B515
:107D600005460C46012D19D1B148026810308454E3
:107D700010380068401CAE49086008460068C0B270
:107D800008600846C06838B10020C860012240F28F
:107D90002771A64802F0C2FD204670BD4FF0FF30AB
:107DA000FBE7014601291FD1A2484068A14B1B688F
:107DB000984204D100209F4B9860401E70479D4818
:107DC0008068401E9B4B9860184643681030C25C28
:107DD00010384068401C974B58601846406800F0C7
:107DE000010058601046E9E74FF0FF30E6E770B554
:107DF00005462846FFF7D5FF044606E0052003F0B8
:107E000023FD2846FFF7CDFF0446002CF6DB204675
:107E100070BD2DE9F04107460D4614462E460CB9BB
:107E2000BDE8F08104E016F8011B3846FFF797FF24
:107E30002000A4F101018CB2F5D100BFF0E70246A9
:107E4000012A1FD17B4840687A4B1B68984203D1B6
:107E50000020784B9860704776488068401E754BCC
:107E60009860184643681030C05C087071484068DC
:107E7000401C704B58601846406800F00100586084
:107E80000120E8E74FF0FF30E5E778B506460C46FD
:107E9000002504E09DF8002028466D1C2254694608
:107EA0003046FFF7CCFF0128F4D00020605528466B
:107EB00078BD2DE9F84107460D461646002400BF5F
:107EC00069463846FFF7BBFF80460DE09DF800206D
:107ED0002046611C8CB22A54B44200DB07E069469C
:107EE0003846FFF7ACFF8046B8F1000FEED100BF77
:107EF000002028552046BDE8F8810146012913D10C
:107F00004C4800684B4A5268904205D34948006883
:107F1000484A5268801A704746484068454A126885
:107F2000801AC0F10200F6E70020F4E701460129BB
:107F300002D14048C06870470020FCE7012805D105
:107F400000213C4A91605160116000BF00BF704742
:107F500010B503461846FFF7D0FF80B2040005D0E5
:107F60001846FFF7E3FF08B9204610BD0020FCE7E4
:107F70003048C06820B12F48C068401E2D49C860F5
:107F8000704710B540F22551284802F002FDE0B1DB
:107F900040F22551254802F033FD244802F037FC19
:107FA000C1B2244802681030815410380068401C67
:107FB000204908600846006800F001000860084693
:107FC0008068401C88601E20C86040F227711748F6
:107FD00002F0DFFC30B340F22771144802F010FDCC
:107FE0001348006812494968884212D01048426814
:107FF0001030815C0D4802F006FC0D484068401CC2
:108000000B49486008464068C0B248600020C8601C
:1080100008E001200649C860002240F227710348A9
:1080200002F07CFC10BD0000000002400010014086
:10803000A0000020C006002010B5044608492046D4
:1080400001F041FD208B10BD10B5044604490E31EE
:10805000204601F038FD0121204601F00EFC10BD44
:108060000200001000B587B00121C80501F02DFF06
:10807000DB498868012101F0F5FED94988690121B1
:1080800001F0F0FE0121C80501F087FF00214FF447
:10809000000001F082FFD24A117B1068042201F037
:1080A0001DFBCF4A117F1069042201F017FB02204B
:1080B0008DF818008DF8190001208DF81A008DF840
:1080C0001B00C74880880590C549086805A901F0CC
:1080D00077FAC348808A0590C149086905A901F06B
:1080E0006FFAC04801F024FB0121BE4801F020FCDA
:1080F0000021BC4801F01CFC0020ADF808004BF644
:10810000FF70ADF80A004FF48060ADF80E0000017A
:10811000ADF81000B44801900121B24801F0D9FB3C
:1081200001A9B04801F02DFB0121AE4801F00BFC84
:108130000121AC4801F0A1FB07B000BD2DE9F041E1
:1081400006460F4615464FF47A7400BF06E00CB1A0
:10815000641E03E06FF00100BDE8F0814FF40031D0
:10816000304601F0B0FC0028F1D10121304601F089
:1081700090FB4FF47A7405E00CB1641E02E04FF0FE
:10818000FF30E9E79949304601F07BFC0028F3D045
:108190002A463946304601F094FB4FF47A7475B99B
:1081A00000BF04E0601E040001D10120D4E7904923
:1081B000304601F088FCA0B9002CF3D111E0012D6C
:1081C0000FD14FF47A7404E0601E040001D1012045
:1081D000C2E78649491C304601F053FC08B9002C1F
:1081E000F2D1308B0020B7E770B505460E464FF44C
:1081F0007A7405E00CB1641E02E04FF0FF3070BDF0
:108200007C49284601F03DFC0028F3D03146284641
:1082100001F0DBFB4FF47A7405E00CB1641E02E060
:108220004FF0FF30EBE77349091D284601F029FCA8
:108230000028F2D00020E2E770B505464FF47A74CA
:108240000121284601F045FB05E00CB1641E02E067
:108250004FF0FF3070BD65493F31284601F011FCF9
:108260000028F2D0284601F0B2FB06463046F1E77E
:1082700070B505464FF47A740021284601F029FBB9
:108280000121284601F011FB05E00CB1641E02E05B
:108290004FF0FF3070BD55493F31284601F0F1FBEA
:1082A0000028F2D0284601F092FB06463046F1E75E
:1082B00070B505464FF47A7409E00CB1641E06E00F
:1082C0000121284601F0F1FA4FF0FF3070BD494915
:1082D000091D284601F0D5FB0028EED001212846D3
:1082E00001F0E3FA0020F1E72DE9F04780468946E6
:1082F000154600260527012249464046FFF71EFF86
:10830000401C30B90121404601F0CFFA701EBDE893
:10831000F087002415E0032C04D16878A97800EBDD
:10832000012007444046FFF787FF0646701C30B91E
:108330000121404601F0B9FA4FF0FF30E7E72E5532
:10834000641C781EA042E6DC4046FFF791FF06461B
:10835000701C30B90121404601F0A7FA4FF0FF3000
:10836000D5E72E550020D2E72DE9F0410746884693
:1083700015461E46002241463846FFF7DFFE401CE8
:1083800038B90121384601F090FA4FF0FF30BDE8CE
:10839000F08100240DE0295D3846FFF725FF401CE1
:1083A00030B90121384601F080FA4FF0FF30EEE796
:1083B000641CB442EFDB3846FFF77AFFE7E770B59D
:1083C00004460D460026002229462046FFF7B6FE49
:1083D00000B901262046FFF76BFF304670BD000054
:1083E00020000010005C0040A08601000100030096
:1083F000020000108000070010B588B0044601217B
:10840000480501F062FDB5498868012101F02AFDA7
:10841000B2498869012101F025FD0121480501F0DB
:10842000BCFD00214FF4001001F0B7FDAB4A117BF9
:108430001068042201F052F9A84A117F1069042241
:1084400001F04CF902208DF81C008DF81D00012070
:108450008DF81E008DF81F00A048808806909F4967
:10846000086806A901F0ACF89C48808A06909B49F0
:10847000086906A901F0A4F8994801F059F9012109
:10848000974801F055FA0021954801F051FA002073
:10849000ADF808004BF6FF70ADF80A00ADF80C40DF
:1084A0004FF48060ADF80E000001ADF810008D486B
:1084B000019001218A4801F00CFA01A9884801F0D5
:1084C00060F90121864801F03EFA0121844801F05B
:1084D000D4F91F208DF8140000208DF815008DF8B8
:1084E000160001208DF8170005A800F032FD2020AD
:1084F0008DF8140000208DF815008DF8160001206D
:108500008DF8170005A800F024FD012251027448DF
:1085100001F0AEFA01221102714801F0A9FA08B087
:1085200010BD38B56E4801F0C1FA00900098B0F166
:10853000021F19D009DC022815D0102836D0502887
:108540001FD0B0F5806F6ED168E0A0F500304038E4
:10855000C8B1042816D0A0F58020423800283DD0AC
:10856000022860D14BE000BF5D48FFF765FD0020A9
:108570005D49086001205D49087000205C49088061
:1085800051E000BF00BF5948007801280AD1544883
:1085900001F01DFA56490C88611C554A1180554955
:1085A000085502E04E4801F012FA3CE04C48143005
:1085B000008800904A48008840F00100484908803F
:1085C0004A48007810B10120474908600020474917
:1085D00008700021424801F07CF924E04048FFF790
:1085E0002BFD00204449088008460488601C0A4688
:1085F00010804248015D3A4801F0E7F913E03E4837
:108600000488601C3C4A10803C48015D344801F0FD
:10861000DCF93B49324801F056FA04E03949304868
:1086200001F094FA00BF00BF07E02D481430008825
:1086300000902B481830008800902948143000889A
:1086400000F002000228F0D038BD10B52E492448B1
:1086500001F05CFA20B12C49214801F077FA3CE0A6
:108660002A491F4801F052FA20B128491C4801F05C
:108670006DFA32E026491A4801F048FA20B124493F
:10868000174801F063FA28E02249154801F03EFA44
:1086900020B12049124801F059FA1EE0194910484A
:1086A00001F034FA20B117490D4801F04FFA14E0F7
:1086B00019490B4801F02AFA20B11749084801F07E
:1086C00045FA0AE04FF00121054801F01FFA20B1F8
:1086D0004FF00121024801F039FA10BD48000010A6
:1086E00000540040A0860100440000106800001003
:1086F00040000010A8C6001042000010AECA0010D2
:10870000040000100004000100800001004000018E
:1087100000100001000800010002000110B5014630
:1087200000200022314B1B6803F0005333B10120BD
:108730002E4B1B6843F080732C4C236045F255533D
:108740002B4C23600B2902DB0723636002E0032329
:10875000274C6360FF2901D101223CE009B90522C1
:1087600039E0012901D10A2235E0022901D10F2285
:1087700031E0032901D11F222DE0042901D13D223E
:1087800029E0052901D17B2225E0062901D1FF221C
:1087900021E0072902D140F2FF121CE0082902D192
:1087A00040F2FF3217E0092902D140F2FF7212E0D5
:1087B0000A2902D140F6FF720DE00B2902D140F2E6
:1087C000FF3208E00C2902D140F2FF7203E00D29CC
:1087D00001D140F6FF72064B9A604AF6AA23044C78
:1087E00023604CF6CC43236010BD00007438024077
:1087F0000030004070B50546284614F058FF064684
:1088000000242FE0285DB82803D1F12066490855DF
:1088100027E0285DA82803D1F0206349085520E00F
:10882000285D802803DA285D5F49085518E0285D37
:10883000C02807DB285DEF2804DC285D40385A4952
:1088400008550DE0285DF02807DB285DFF2804DCD3
:10885000285D10385449085502E0285D52490855F2
:1088600000BF641CB442CDDB002427E04E48005D0D
:10887000802800DA21E04C48005DA02808DB4A4847
:10888000005DAF2804DC4848005D203846490855A3
:108890004548005DE02808DB4348005DEF2804DC24
:1088A0004148005D5038404908553F48005DF12877
:1088B00002D1F0203C49085500BF641CB442D5DB0E
:1088C00000203949885570BD10B503E03220207072
:1088D0003020607035A1344814F0C1FE0400F5D199
:1088E00010BD70B50546002407E0314830F834006B
:1088F000A84200D103E0601C84B2822CF5DB00BFEB
:108900002B4901EBC4014868FFF774FF284830F891
:10891000340028490880264800EBC400807888701D
:108920002148486070BD2DE9F04106460F46224DB2
:10893000002408E004EB440035F82000B04200D1E8
:1089400003E0601C84B2EF2CF4DB00BF07F00100F1
:1089500050B9B6F5A04F07DC04EB440105EB8101EB
:108960004868FFF747FF06E004EB440105EB81018F
:108970008868FFF73FFF04EB440035F820000F49FB
:10898000088004EB440005EB80004088488007F035
:10899000020020B1B6F5A04F01DAFFF795FF0248BB
:1089A00006494860BDE8F0813007002031380000FA
:1089B00080F40208F005002098F80208240700203F
:1089C0002DE9F74F84B016464FF0000ADDF81090FD
:1089D00038E00921684614F02BFE00241FE0305DCA
:1089E000401E87B2FD1007F007010120884080B2C9
:1089F000039019F805100398014071B14FEAE4089B
:108A000004F00701012088401FFA80FB1DF80800D0
:108A100040EA0B00C0B20DF80800601C84B2305D63
:108A20000028DCDCE410002505E01DF8050009F84D
:108A30000500681C85B2A542F7DBA1440AEB0400DF
:108A40001FFA80FA05988245C3DB07B0BDE8F08FB6
:108A500070B504460B4600251D60002025E000EBA4
:108A6000400545F39C02A65C551C655D06EB05259B
:108A7000A9B200EB40056D00A5EBC205294101F04C
:108A80003F0101F0010201F0200505B1921CC1F384
:108A9000430102EB800501EB0515B34E755D8600C1
:108AA000B5401E6835431D60401C0828D7DB70BDEB
:108AB0002DE9F04104464FF0000CC1F800C0A1F8C8
:108AC00004C0002028E0DFF8A4C21CF800C0ACF10C
:108AD000010C0CF0FF03DF1003F007084FF0010C4E
:108AE0000CFA08FC0CF0FF0514F807C00CEA050CA2
:108AF000BCF1000F0FD0C0F3C70200F007084FF021
:108B0000010C0CFA08FC0CF0FF0611F802C04CEA4C
:108B1000060C01F802C0401C3028D4DBBDE8F0810F
:108B200073B50E46924D29466846FFF7C1FF0024F3
:108B300004E0285D315D48402855641C062CF8DBB4
:108B40008C498B48FFF784FF8B4A04218948FFF743
:108B500037FF884800687CBD2DE9F04104460E4689
